:020000040800F2
:10000000E0BE00205D3C0008AB5B0308493C0008F3
:10001000493C0008493C0008493C0008493C0008AC
:10002000000000000000000000000000493D000842
:10003000493C000800000000E13C000895A60008CB
:10004000E93E0008E93E0008E93E0008E93E0008F4
:10005000E93E0008E93E0008E93E0008E93E0008E4
:10006000E93E0008E93E0008E93E0008E93E0008D4
:10007000E93E0008E93E0008E93E0008E93E0008C4
:10008000E93E0008E93E0008E93E0008E93E0008B4
:10009000E93E0008E93E0008E93E0008E93E0008A4
:1000A000E93E0008E93E0008E93E0008E93E000894
:1000B000E93E0008E93E0008E93E0008E93E000884
:1000C000E93E0008E93E0008E93E0008E93E000874
:1000D000E93E0008E93E0008E93E0008E93E000864
:1000E000E93E0008E93E0008E93E0008E93E000854
:1000F000E93E0008E93E0008E93E0008E93E000844
:10010000E93E0008E93E0008E93E0008E93E000833
:10011000E93E0008E93E0008E93E0008E93E000823
:10012000E93E0008E93E0008E93E0008E93E000813
:10013000E93E0008E93E0008E93E0008E93E000803
:10014000E93E0008E93E0008E93E0008E93E0008F3
:10015000E93E0008E93E0008E93E0008E93E0008E3
:10016000E93E0008E93E0008E93E0008E93E0008D3
:10017000E93E0008E93E0008E93E0008E93E0008C3
:10018000E93E0008E93E0008E93E0008E93E0008B3
:10019000E93E0008E93E0008E93E0008E93E0008A3
:1001A000E93E0008E93E0008E93E0008E93E000893
:1001B000E93E0008E93E0008E93E0008E93E000883
:1001C000E93E0008E93E0008E93E0008E93E000873
:1001D000E93E0008E93E0008E93E0008E93E000863
:1001E000E93E0008E93E0008E93E0008E93E000853
:1001F000E93E0008E93E0008E93E0008E93E000843
:10020000E93E0008E93E0008E93E0008E93E000832
:10021000E93E0008E93E0008E93E0008E93E000822
:10022000E93E0008E93E0008E93E0008E93E000812
:04023000E93E00089B
:1002380081F0004102E000BF83F0004330B54FEA8F
:1002480041044FEA430594EA050F08BF90EA020FFC
:100258001FBF54EA000C55EA020C7FEA645C7FEA8F
:10026800655C00F0E2804FEA5454D4EB5555B8BFB2
:100278006D420CDD2C4480EA020281EA030382EA23
:10028800000083EA010180EA020281EA0303362DB5
:1002980088BF30BD11F0004F4FEA01314FF4801C88
:1002A8004CEA113102D0404261EB410113F0004F9A
:1002B8004FEA03334CEA133302D0524263EB430351
:1002C80094EA050F00F0A780A4F10104D5F1200EEF
:1002D8000DDB02FA0EFC22FA05F2801841F100014A
:1002E80003FA0EF2801843FA05F359410EE0A5F11E
:1002F80020050EF1200E012A03FA0EFC28BF4CF04F
:10030800020C43FA05F3C01851EBE37101F0004504
:1003180007D54FF0000EDCF1000C7EEB00006EEB11
:100328000101B1F5801F1BD3B1F5001F0CD349089B
:100338005FEA30004FEA3C0C04F101044FEA4452F2
:1003480012F5800F80F09A80BCF1004F08BF5FEA79
:10035800500C50F1000041EB045141EA050130BD59
:100368005FEA4C0C404141EB0101013C28BFB1F56B
:10037800801FE9D291F0000F04BF01460020B1FAB6
:1003880081F308BF2033A3F10B03B3F120020CDA89
:100398000C3208DD02F1140CC2F10C0201FA0CF067
:1003A80021FA02F10CE002F11402D8BFC2F1200CCC
:1003B80001FA02F120FA0CFCDCBF41EA0C01904082
:1003C800E41AA2BF01EB0451294330BD6FEA0404CB
:1003D8001F3C1CDA0C340EDC04F11404C4F12002B6
:1003E80020FA04F001FA02F340EA030021FA04F3C8
:1003F80045EA030130BDC4F10C04C4F1200220FA1F
:1004080002F001FA04F340EA0300294630BD21FA5C
:1004180004F0294630BD94F0000F83F4801306BF22
:1004280081F480110134013D4EE77FEA645C18BF16
:100438007FEA655C29D094EA050F08BF90EA020FAD
:1004480005D054EA000C04BF1946104630BD91EAA5
:10045800030F1EBF0021002030BD5FEA545C05D1A8
:100468004000494128BF41F0004130BD14F58004E7
:100478003CBF01F5801130BD01F0004545F0FE415B
:1004880041F470014FF0000030BD7FEA645C1ABF90
:10049800194610467FEA655C1CBF0B46024650EAC7
:1004A800013406BF52EA033591EA030F41F40021F3
:1004B80030BD00BF90F0000F04BF0021704730B579
:1004C8004FF4806404F132044FF000054FF000014E
:1004D80050E700BF90F0000F04BF0021704730B50F
:1004E8004FF4806404F1320410F0004548BF4042E4
:1004F8004FF000013EE700BF42004FEAE2014FEA39
:1005080031014FEA02701FBF12F07F4393F07F4F13
:1005180081F06051704732F07F4208BF704793F016
:100528007F4F04BF41F40021704730B54FF4607429
:1005380001F0004521F000411CE700BF50EA01022C
:1005480008BF704730B54FF000050AE050EA0102D5
:1005580008BF704730B511F0004502D5404261EB45
:1005680041014FF4806404F132045FEA915C3FF486
:10057800D8AE4FF003025FEADC0C18BF03325FEA23
:10058800DC0C18BF033202EBDC02C2F1200300FAD4
:1005980003FC20FA02F001FA03FE40EA0E0021FAF9
:1005A80002F11444BDE600BF70B54FF0FF0C4CF4E7
:1005B800E06C1CEA11541DBF1CEA135594EA0C0F99
:1005C80095EA0C0F00F0DEF82C4481EA030621EAD4
:1005D8004C5123EA4C5350EA013518BF52EA03350F
:1005E80041F4801143F4801338D0A0FB02CE4FF0C1
:1005F8000005E1FB02E506F00042E0FB03E54FF0F1
:100608000006E1FB03569CF0000F18BF4EF0010EE8
:10061800A4F1FF04B6F5007F64F5407404D25FEAE4
:100628004E0E6D4146EB060642EAC62141EA555197
:100638004FEAC52040EA5E504FEACE2EB4F1FD0CD9
:1006480088BFBCF5E06F1ED8BEF1004F08BF5FEA57
:10065800500E50F1000041EB045170BD06F0004609
:1006680046EA010140EA020081EA0301B4EB5C04B6
:10067800C2BFD4EB0C0541EA045170BD41F48011AE
:100688004FF0000E013C00F3AB8014F1360FDEBFD3
:10069800002001F0004170BDC4F10004203C35DAAF
:1006A8000C341BDC04F11404C4F1200500FA05F332
:1006B80020FA04F001FA05F240EA020001F00042D3
:1006C80021F0004110EBD37021FA04F642EB060149
:1006D8005EEA430E08BF20EAD37070BDC4F10C0473
:1006E800C4F1200500FA04F320FA05F001FA04F237
:1006F80040EA020001F0004110EBD37041F1000123
:100708005EEA430E08BF20EAD37070BDC4F120052D
:1007180000FA05F24EEA020E20FA04F301FA05F295
:1007280043EA020321FA04F001F0004121FA04F23D
:1007380020EA020000EBD3705EEA430E08BF20EA0D
:10074800D37070BD94F0000F0FD101F00046400047
:1007580041EB010111F4801F08BF013CF7D041EAC9
:10076800060195F0000F18BF704703F000465200CD
:1007780043EB030313F4801F08BF013DF7D043EA9E
:100788000603704794EA0C0F0CEA135518BF95EA54
:100798000C0F0CD050EA410618BF52EA4306D1D1DB
:1007A80081EA030101F000414FF0000070BD50EAFA
:1007B800410606BF1046194652EA430619D094EA84
:1007C8000C0F02D150EA013613D195EA0C0F05D16E
:1007D80052EA03361CBF104619460AD181EA0301C2
:1007E80001F0004141F0FE4141F470014FF000007A
:1007F80070BD41F0FE4141F4780170BD70B54FF015
:10080800FF0C4CF4E06C1CEA11541DBF1CEA135594
:1008180094EA0C0F95EA0C0F00F0A7F8A4EB050476
:1008280081EA030E52EA03354FEA013100F088806D
:100838004FEA03334FF0805545EA131343EA126336
:100848004FEA022245EA111545EA10654FEA0026EB
:100858000EF000419D4208BF964244F1FD0404F5A4
:10086800407402D25B084FEA3202B61A65EB030500
:100878005B084FEA32024FF480104FF4002CB6EBBD
:10088800020E75EB030E22BFB61A754640EA0C003D
:100898005B084FEA3202B6EB020E75EB030E22BF7D
:1008A800B61A754640EA5C005B084FEA3202B6EBBE
:1008B800020E75EB030E22BFB61A754640EA9C007D
:1008C8005B084FEA3202B6EB020E75EB030E22BF4D
:1008D800B61A754640EADC0055EA060E18D04FEA0B
:1008E800051545EA16754FEA06164FEAC30343EAAB
:1008F80052734FEAC2025FEA1C1CC0D111F4801F78
:100908000BD141EA00014FF000004FF0004CB6E770
:1009180011F4801F04BF01430020B4F1FD0C88BF0F
:10092800BCF5E06F3FF6AFAEB5EB030C04BFB6EB1A
:10093800020C5FEA500C50F1000041EB045170BD0D
:100948000EF0004E4EEA113114EB5C04C2BFD4EB3A
:100958000C0541EA045170BD41F480114FF0000EBE
:10096800013C90E645EA060E8DE60CEA135594EA3A
:100978000C0F08BF95EA0C0F3FF43BAF94EA0C0F3D
:100988000AD150EA01347FF434AF95EA0C0F7FF4B2
:1009980025AF104619462CE795EA0C0F06D152EA06
:1009A80003353FF4FDAE1046194622E750EA4106EA
:1009B80018BF52EA43067FF4C5AE50EA41047FF4FB
:1009C8000DAF52EA43057FF4EBAE12E74FF0FF3C60
:1009D80006E000BF4FF0010C02E000BF4FF0010C31
:1009E8004DF804CD4FEA410C7FEA6C5C4FEA430CAA
:1009F80018BF7FEA6C5C1BD001B050EA410C0CBFF9
:100A080052EA430C91EA030F02BF90EA020F00205A
:100A1800704710F1000F91EA030F58BF994208BFC1
:100A280090422CBFD8176FEAE37040F0010070477E
:100A38004FEA410C7FEA6C5C02D150EA013C07D1D5
:100A48004FEA430C7FEA6C5CD6D152EA033CD3D020
:100A58005DF8040B704700BF8446104662468C461A
:100A68001946634600E000BF01B5FFF7B7FF00284D
:100A780048BF10F1000F01BD4DF808EDFFF7F4FF76
:100A88000CBF012000205DF808FB00BF4DF808ED01
:100A9800FFF7EAFF34BF012000205DF808FB00BF24
:100AA8004DF808EDFFF7E0FF94BF012000205DF846
:100AB80008FB00BF4DF808EDFFF7CEFF94BF0120FB
:100AC80000205DF808FB00BF4DF808EDFFF7C4FFF4
:100AD80034BF012000205DF808FB00BF4FEA410247
:100AE800B2F1E04324BFB3F5001CDCF1FE5C0DD984
:100AF80001F0004C4FEAC0024CEA5070B2F1004FCE
:100B080040EB830008BF20F00100704711F0804FD0
:100B180021D113F13872BCBF01F00040704741F495
:100B280080114FEA5252C2F11802C2F1200C10FA99
:100B38000CF320FA02F018BF40F001004FEAC1237D
:100B48004FEAD32303FA0CFC40EA0C0023FA02F321
:100B58004FEA4303CCE77FEA625307D150EA0133F7
:100B68001EBF4FF0FE4040F44000704701F00040C7
:100B780040F0FE4040F40000704700BF80F00040A5
:100B880002E000BF81F0004142001FBF5FEA41035D
:100B980092EA030F7FEA226C7FEA236C6AD04FEA5D
:100BA8001262D2EB1363C1BFD218414048404140A2
:100BB800B8BF5B42192B88BF704710F0004F40F454
:100BC800000020F07F4018BF404211F0004F41F470
:100BD800000121F07F4118BF494292EA030F3FD03C
:100BE800A2F1010241FA03FC10EB0C00C3F120034F
:100BF80001FA03F100F0004302D5494260EB4000DE
:100C0800B0F5000F13D3B0F1807F06D340084FEA48
:100C1800310102F10102FE2A51D2B1F1004F40EB3D
:100C2800C25008BF20F0010040EA030070474900A5
:100C380040EB0000013A28BFB0F5000FEDD2B0FA42
:100C480080FCACF1080CB2EB0C0200FA0CF0AABF65
:100C580000EBC25052421843BCBFD0401843704703
:100C680092F0000F81F4000106BF80F40000013209
:100C7800013BB5E74FEA41037FEA226C18BF7FEAE0
:100C8800236C21D092EA030F04D092F0000F08BF22
:100C98000846704790EA010F1CBF0020704712F009
:100CA8007F4F04D1400028BF40F00040704712F148
:100CB80000723CBF00F50000704700F0004343F0AD
:100CC800FE4040F4000070477FEA226216BF0846E3
:100CD8007FEA23630146420206BF5FEA412390EAA6
:100CE800010F40F4800070474FF0000304E000BF9C
:100CF80010F0004348BF40425FEA000C08BF70474D
:100D080043F0964301464FF000001CE050EA010210
:100D180008BF70474FF000030AE000BF50EA010225
:100D280008BF704711F0004302D5404261EB410112
:100D38005FEA010C02BF84460146002043F0B64337
:100D480008BFA3F18053A3F50003BCFA8CF2083A5C
:100D5800A3EBC25310DB01FA02FC634400FA02FC65
:100D6800C2F12002BCF1004F20FA02F243EB02006C
:100D780008BF20F00100704702F1200201FA02FCCE
:100D8800C2F1200250EA4C0021FA02F243EB0200C1
:100D980008BF20EADC7070474FF0FF0C1CEAD05205
:100DA8001EBF1CEAD15392EA0C0F93EA0C0F6FD0C6
:100DB8001A4480EA010C400218BF5FEA41211ED0A4
:100DC8004FF0006343EA501043EA5111A0FB013190
:100DD8000CF00040B1F5000F3EBF490041EAD37165
:100DE8005B0040EA010062F17F02FD2A1DD8B3F1E1
:100DF800004F40EBC25008BF20F00100704790F050
:100E0800000F0CF0004C08BF49024CEA502040EAA1
:100E180051207F3AC2BFD2F1FF0340EAC250704767
:100E280040F400004FF00003013A5DDC12F1190FA5
:100E3800DCBF00F000407047C2F10002410021FA17
:100E480002F1C2F1200200FA02FC5FEA310040F12F
:100E5800000053EA4C0308BF20EADC70704792F0A8
:100E6800000F00F0004C02BF400010F4000F013AE0
:100E7800F9D040EA0C0093F0000F01F0004C02BFDB
:100E8800490011F4000F013BF9D041EA0C018FE74A
:100E98000CEAD15392EA0C0F18BF93EA0C0F0AD050
:100EA80030F0004C18BF31F0004CD8D180EA010076
:100EB80000F00040704790F0000F17BF90F0004F0F
:100EC800084691F0000F91F0004F14D092EA0C0FF1
:100ED80001D142020FD193EA0C0F03D14B0218BF84
:100EE800084608D180EA010000F0004040F0FE40CA
:100EF80040F40000704740F0FE4040F44000704766
:100F08004FF0FF0C1CEAD0521EBF1CEAD15392EAE4
:100F18000C0F93EA0C0F69D0A2EB030280EA010CD4
:100F280049024FEA402037D04FF0805343EA11116D
:100F380043EA10130CF000408B4238BF5B0042F1CB
:100F48007D024FF4000C8B4224BF5B1A40EA0C0070
:100F5800B3EB510F24BFA3EB510340EA5C00B3EBA2
:100F6800910F24BFA3EB910340EA9C00B3EBD10F90
:100F780024BFA3EBD10340EADC001B0118BF5FEAE2
:100F88001C1CE0D1FD2A3FF650AF8B4240EBC2500B
:100F980008BF20F0010070470CF0004C4CEA5020CC
:100FA8007F32C2BFD2F1FF0340EAC250704740F41B
:100FB80000004FF00003013A37E792F0000F00F00D
:100FC800004C02BF400010F4000F013AF9D040EA8B
:100FD8000C0093F0000F01F0004C02BF490011F41F
:100FE800000F013BF9D041EA0C0195E70CEAD15317
:100FF80092EA0C0F08D142027FF47DAF93EA0C0FFE
:101008007FF470AF084676E793EA0C0F04D14B02E1
:101018003FF44CAF08466EE730F0004C18BF31F093
:10102800004CCAD130F000427FF45CAF31F000438D
:101038007FF43CAF5FE700BF4FF0FF3C06E000BF26
:101048004FF0010C02E000BF4FF0010C4DF804CD49
:101058004FEA40024FEA41037FEA226C18BF7FEA59
:10106800236C11D001B052EA530C18BF90EA010F5B
:1010780058BFB2EB030088BFC81738BF6FEAE170EA
:1010880018BF40F0010070477FEA226C02D15FEA86
:10109800402C05D17FEA236CE4D15FEA412CE1D0F2
:1010A8005DF8040B704700BF844608466146FFE7B9
:1010B8000FB5FFF7C9FF002848BF10F1000F0FBD9B
:1010C8004DF808EDFFF7F4FF0CBF012000205DF894
:1010D80008FB00BF4DF808EDFFF7EAFF34BF012019
:1010E80000205DF808FB00BF4DF808EDFFF7E0FFB2
:1010F80094BF012000205DF808FB00BF4DF808ED03
:10110800FFF7D2FF94BF012000205DF808FB00BF65
:101118004DF808EDFFF7C8FF34BF012000205DF847
:1011280008FB00BF4FEA40024FEA41037FEA226C06
:1011380002D15FEA402C08D17FEA236C02D15FEA32
:10114800412C02D14FF0000070474FF0010070476A
:101158004FEA4002B2F1FE4F0FD34FF09E03B3EBBC
:1011680012620DD94FEA002343F0004310F0004FFC
:1011780023FA02F018BF404270474FF00000704752
:1011880012F1610F01D1420205D110F0004008BFF1
:101198006FF0004070474FF00000704742000ED2D9
:1011A800B2F1FE4F0BD34FF09E03B3EB126209D49A
:1011B8004FEA002343F0004323FA02F070474FF050
:1011C8000000704712F1610F01D1420202D14FF0C5
:1011D800FF3070474FF00000704700BF7BB972B90D
:1011E8000029BEBF00204FF0004106E008BF0028DC
:1011F8001CBF6FF000414FF0FF3000F077B8ADF141
:10120800080C6DE904CE002909DB002B1ADB00F07D
:10121800A9F8DDF804E0DDE9022304B07047404294
:1012280061EB4101002B1BDB00F09CF8DDF804E0CA
:10123800DDE9022304B0404261EB4101524263EB15
:1012480043037047524263EB430300F08BF8DDF829
:1012580004E0DDE9022304B0404261EB410170473C
:10126800524263EB430300F07DF8DDF804E0DDE96A
:10127800022304B0524263EB4303704753B94AB99F
:10128800002908BF00281CBF4FF0FF314FF0FF3086
:1012980000F02CB8ADF1080C6DE904CE00F062F84E
:1012A800DDF804E0DDE9022304B07047D0B5FFF7AC
:1012B80023F900220B4B06460F46FFF775F900F09D
:1012C80017F80446FFF7F6F80022074BFFF76CF90A
:1012D80002460B4630463946FEF7AEFF00F008F8E6
:1012E8002146D0BD0000F03D0000F041704700BF2E
:1012F8004A0011D212F5001211D20DD56FF478738D
:10130800B3EB62520ED44FEAC12343F0004343EAE1
:10131800505323FA02F070474FF00000704750EA2C
:10132800013002D14FF0FF3070474FF00000704796
:1013380010F8012B11F8013B012A28BF9A42F7D077
:10134800D01A7047034611F8012B03F8012B002A25
:10135800F9D17047034613F8012B002AFBD1181A5C
:10136800013870472DE9F04786468C460846089EA6
:10137800154674461946002B40F0C1808542B2FAE2
:1013880082F245D94AB1C2F1200300FA02FC954025
:1013980094402EFA03F343EA0C0C4FEA154EA8B218
:1013A800230CBCFBFEF80EFB18CC08FB00F943EA43
:1013B8000C43994528D9EB1808F1FF3704D2994511
:1013C80002D9A8F102072B44A3EB0903A4B2B3FB8B
:1013D800FEFC0EFB1C330CFB00F044EA0344A04265
:1013E80014D92C190CF1FF3304D2A04202D9ACF164
:1013F80002032C44241A43EA07401EB1D4400023B8
:1014080034607360BDE8F0874746DDE76346F1E77F
:1014180092BB431B01214FEA154EAFB2200CB3FB20
:10142800FEFC0EFB1C330CFB07F840EA034398450F
:1014380061D9EB180CF1FF3004D2984502D9ACF110
:1014480002002B44A3EB0803A4B2B3FBFEFC0EFB83
:101458001C330CFB07F744EA0344A7424DD92C1967
:101468000CF1FF3304D2A74202D9ACF102032C4499
:10147800E41B43EA0040C0E7C2F1200395409440D2
:1014880020FA03F12EFA03F34FEA154E9040AFB25B
:101498000343B1FBFEFC0EFB1C10190C0CFB07F8F8
:1014A80041EA0041884522D969180CF1FF3004D27D
:1014B800884502D9ACF102002944A1EB08019BB28E
:1014C800B1FBFEFC0EFB1C110CFB07F743EA0143C2
:1014D8009F420ED9EB180CF1FF3104D29F4202D97A
:1014E800ACF102012B44DB1B41EA004193E7604663
:1014F800E3E76146F7E76046A4E76346B8E7834257
:1015080006D916B9002108467CE7C6E900E0F9E7E4
:10151800B3FA83F78FB9834201D3724508D8BEEB7B
:10152800020460EB030301209C461EB9002169E711
:101538003846FAE7C6E9004CF8E7C7F1200CBB408B
:101548000EFA07F522FA0CF42EFA0CF1BA401C43F5
:1015580020FA0CF3B8404FEA144901431FFA84FEFD
:10156800B3FBF9F809FB18300B0C08FB0EFA43EA39
:1015780000439A4540D9E31808F1FF3004D29A4550
:1015880002D9A8F102002344A3EB0A0389B2B3FBF2
:10159800F9F809FB183308FB0EFE41EA03418E45B2
:1015A8002CD9611808F1FF3304D28E4502D9A8F16D
:1015B8000203214443EA0040A1EB0E01A0FB02987C
:1015C8004145CE46434602D306D14D4504D20138A3
:1015D800B9EB020E68EB0403002EA7D0B5EB0E02A0
:1015E80061EB030101FA0CFC22FA07F3F9404CEA1B
:1015F8000303C6E9003199E74046C5E74346D9E702
:101608002DE9F04390F8A53004460D4685B023B97E
:101618004FF07E50FFF7B6FA0546D4F884202E4BDB
:101628009A4212D12846FEF767FF29A3D3E900237F
:10163800FFF74AFA011E18BF012104F184000FF0D8
:101648001DFA0120C4F8985005E0B4F89C30B3F5B1
:10165800807F03D1002005B0BDE8F08304F1500974
:10166800484626F0CFFD0028F4D01C492846FFF74D
:1016780093FBFFF793FD94F88080C3B294F89C60C5
:10168800276E206DB8F1000F0DD08DF80D300223B4
:101698000122002100938DF80C6003ABB84748463F
:1016A80043F0F1F9CDE78DF80B600126414632464B
:1016B8008DF80C3000960DF10B03B84700964246A2
:1016C8003146276E206D03ABE8E700BFAFF300801B
:1016D800AE47E17A14AEEF3FBC22050800007F4315
:1016E80030F0004201462DE9F84F034604D10120AD
:1016F800BDE8F84F32F052BC002803DABDE8F84FD5
:1017080032F054BCB0F1FF4F03DBFFF73DFABDE800
:10171800F88FB0F5000F35DA4FF09841FFF73CFB32
:101728006FF018020346C3F31604DE15764B4FF02C
:101738007E517F3E2344164403F4000006EBD35643
:1017480080F07E502043FFF71DFA04F10F026F4B23
:1017580005461340002B3ED10021FFF7B1FC98B19C
:10176800002E00F0C8803046FFF7C2FA68490546E7
:10177800FFF712FB044667492846FFF70DFB0146B1
:101788002046C2E70022CEE75DA1D1E90001FFF7BC
:10179800A5F92946FFF700FB01464FF07C50FFF7FB
:1017A800F1F9044629462846FFF7F6FA014620468D
:1017B800FFF7F2FA04460EB921466FE03046FFF70C
:1017C80097FA07465249FFF7E7FA5249064638465C
:1017D800FFF7E2FA72E04FF08041DFF83CB1FFF723
:1017E800D3F901462846A344FFF78AFB81463046D1
:1017F800FFF77EFA494680464846FFF7CDFA01468C
:101808008246FFF7C9FA45490746FFF7C5FA444932
:10181800FFF7BAF93946FFF7BFFA4249FFF7B4F9BB
:101828003946FFF7B9FA4049FFF7AEF95146FFF7D5
:10183800B3FA3E4982463846FFF7AEFA3C49FFF70D
:10184800A3F93946FFF7A8FA3A49FFF79DF939464F
:10185800FFF7A2FA01465046FFF796F9C4F5571369
:10186800074603F5227343EA0B03002B30DD4FF0E4
:101878007C512846FFF790FA2946FFF78DFA014672
:1018880004463846FFF780F94946FFF785FA0746C8
:1018980046B901462046FFF775F901462846FFF785
:1018A80071F934E71A494046FFF776FA19490646AE
:1018B8004046FFF771FA3946FFF766F901462046B8
:1018C800FFF760F92946FFF75DF901463046E6E77C
:1018D80001462846FFF756F94946FFF75DFA0446E0
:1018E800002E3FF469AF0A494046FFF755FA094907
:1018F800064640466CE7002009E700BFAFF30080CA
:10190800555555555555D53F20FB4A00F0FF7F00EA
:101918008071313FD1F71737305CCFFF9788173E7A
:1019280025333A3E2549923EABAA2A3F4FD01C3E6A
:10193800298E633ECDCCCC3E31F000432DE9F04FEB
:10194800804687B00F4681460C460ED180F4800948
:101958004FEA490919F5000F40F2668239464046B8
:10196800FFF712F907B0BDE8F08F20F00046B6F196
:10197800FF4F02D8B3F1FF4F08D9B9F17E5FEDD11F
:1019880084F48004640014F5000FE5E7002832466B
:101998003DDAB3F1974F1BD3B3F1FF4F3AD002258D
:1019A800B4F17C5F4DD1B9F1000F80F29780B6F1A8
:1019B800FF4F28F0004040F04F82A6F17E562E439C
:1019C80040F0A080404607B0BDE8F04F32F0EEBAD4
:1019D800B3F17E5F2ED3D915C1F1960143FA01F513
:1019E80005FA01F18B423BD1B3F17E5F4AD1002C5D
:1019F80080F2938000214046FFF762FB00284FD019
:101A08004FEAD97007B0BDE8F04F32F0C7BAB3F16A
:101A1800FF4F3CD1B6F17E5F00F0068204D9002C5E
:101A2800C0F2058238469DE7002C80F2008207F15B
:101A3800004097E7B1F1804F38D0B1F17C5F53D0C7
:101A4800002529F0404128F00040B1F17E5F3BD1EC
:101A5800002C32DA01464FF07E50FFF751FA2CE0A5
:101A6800B3F17E5FC3D00025B4F1804FE9D1B6F160
:101A7800BF4F1DD2B6F1D05F24D941464046FFF78B
:101A88008BF96FE705F00105C5F10205ECE7B3F145
:101A98007E5FACD0B1F1804F4FF00005E7D07FE713
:101AA80041464FF07E50FFF72BFA5BE70025DEE753
:101AB800B6F1FF4F28F0004031D1B9F1000FBFF661
:101AC80051AF7AE728F000404EBB002C22DAB9F17A
:101AD800000F1DDA6B1E5842584193E7404607B085
:101AE800BDE8F04F48F0F0BFB6F1FF4F20F00040DE
:101AF8003FF438AFB6F17E5F3FF464AF002E3FF499
:101B080031AF5FE7012D7FF42DAF00F1004029E7E9
:101B1800304677E7012D7FF425AF404622E74FEAAC
:101B2800D9710139029129433FF44CAFB3F19A4F6F
:101B380040F29F81604B9E4207D8002C0ADA0020B1
:101B480007B0BDE8F04F32F021BA5C4B9E4207D98E
:101B5800002CF4DC002007B0BDE8F04F49F016B8BF
:101B68004FF07E51FFF70EF806465549FFF714F976
:101B7800544980463046FFF70FF981464CA1D1E918
:101B88000001FEF7ABFF82464FF07A513046FFF76F
:101B980003F901465046FEF7F5FF3146FFF7FCF81A
:101BA80001464FF07C50FEF7EDFF82463146304645
:101BB800FFF7F2F801465046FFF7EEF84249FFF703
:101BC800EBF801464846FEF7DDFF0146064640466B
:101BD800FEF7DAFF20F47F6B41462BF00F0B5846D7
:101BE800FEF7D0FF24F47F6401463046FEF7CAFFB3
:101BF800013D029B24F00F04064638461D4321464A
:101C080014BF4FF07E55314DFEF7BCFF5946FFF724
:101C1800C3F8804639463046FFF7BEF801464046CD
:101C2800FEF7B2FF064621465846FFF7B5F80146CB
:101C380007463046FEF7A8FF00280446804620F0F5
:101C4800004320DDB3F1864F0BD900212846FFF76A
:101C580041FA003818BF012072E7002114E101227F
:101C680027E139D11A493046FEF78EFF81463946B9
:101C78002046FEF787FF01464846FFF749FA002845
:101C8800E3D186232DE0134A934207D90021284641
:101C9800FFF720FA003818BF01205CE71CD139464D
:101CA800FEF770FF3146FFF729FA0028E9D0EDE783
:101CB800E13D55555555D53FF3FF7F3F0700803F20
:101CC80000AAB83F70A5EC363BAAB83F000080BF19
:101CD8003CAA383300001643B3F17C5F40F2A08081
:101CE800DB157E3B4FF400045249B8F1000F44FA6B
:101CF80003F438464444C4F3C753A3F17F0341FABD
:101D080003F1C3F1170301EA0401C4F3160444F410
:101D1800000444FA03F4B8BF6442FEF733FF0746F1
:101D280031463846FEF730FF20F47F68424928F0F4
:101D38000F084046FFF730F8394681464046FEF71F
:101D480021FF01463046FEF71DFF3C49FFF724F806
:101D580006463B494046FFF71FF801463046FEF766
:101D680013FF074601464846FEF70EFF494606465A
:101D7800FEF708FF01463846FEF704FF3146804665
:101D88003046FFF709F82F490746FFF705F82E49AF
:101D9800FEF7F8FE3946FEF7FFFF2C49FEF7F4FE82
:101DA8003946FEF7F9FF2A49FEF7ECFE3946FEF7F9
:101DB800F3FF2849FEF7E8FE3946FEF7EDFF014636
:101DC8003046FEF7DFFE074601463046FEF7E4FFE1
:101DD80081464FF080413846FEF7D4FE014648461A
:101DE800FFF78EF8414607463046FEF7D5FF4146D5
:101DF800FEF7CAFE01463846FEF7C4FE3146FEF736
:101E0800C1FE01464FF07E50FEF7BCFE00EBC45306
:101E1800B3F5000F06DA214632F05AF829462EE6C5
:101E280000247DE71846F9E74FF07E509AE5002038
:101E380098E500BF000080FF0072313F1872313F03
:101E48008CBEBF354CBB31330EEADD3555B38A380D
:101E5800610B363BABAA2A3EB6F17E5F3FF4ADADCF
:101E6800002E3FF457AE002D3FF4ACAD0023022501
:101E7800029319F0FF4F7FF4F0AE4FF09741FEF751
:101E88008BFF6FF017010246D315C2F316027F3B92
:101E980042F07E560B4403937E4B9A4208DD7E4BFC
:101EA8009A427FF7DCAE039BA6F500060133039345
:101EB80000227A4B30460492B24653F822B0594673
:101EC800FEF760FE314681465846FEF75DFE014644
:101ED8004FF07E50FFF714F8014605904846FEF78C
:101EE8005BFF6F49019001EA6606019B049A46F080
:101EF800005623F47F6806F5800628F00F0806EBE5
:101F0800425641463046FEF747FF01464846FEF72F
:101F180039FE594681463046FEF734FE01465046A2
:101F2800FEF730FE4146FEF737FF01464846FEF70A
:101F380029FE059B1946FEF72FFF0199834608469F
:101F4800FEF72AFF57490646FEF726FF5649FEF7D1
:101F58001BFE3146FEF720FF5449FEF715FE3146B9
:101F6800FEF71AFF5249FEF70FFE3146FEF714FF3F
:101F78005049FEF709FE3146FEF70EFF4E49FEF7BF
:101F880003FE814631463046FEF706FF01464846C5
:101F9800FEF702FF414606460198FEF7F5FD594651
:101FA800FEF7FAFE3146FEF7EFFD41468146404610
:101FB800FEF7F2FE41498246FEF7E6FD4946FEF786
:101FC800E3FD20F47F66414626F00F063046FEF713
:101FD800E3FE3A4980463046FEF7D4FD5146FEF707
:101FE800D1FD01464846FEF7CDFD0199FEF7D4FE26
:101FF800814631465846FEF7CFFE01464846FEF771
:10200800C3FD824601464046FEF7BEFD20F47F66CA
:102018002B4926F00F063046FEF7BEFE41468146A4
:102028003046FEF7AFFD01465046FEF7ABFD2549A9
:10203800FEF7B2FE804624493046FEF7ADFE014663
:102048004046FEF7A1FD049A204B019253F8221056
:10205800FEF79AFD06460398FEF74AFE1C4B019AC6
:1020680080463146484653F822A0FEF78DFD51467A
:10207800FEF78AFD4146FEF787FD20F47F6B414657
:102088002BF00F0B5846FEF77DFD5146FEF77AFD03
:102098004946A5E571C41C00D6B35D00B8500508D3
:1020A80000F0FFDF42F1533E55326C3E05A38B3EF4
:1020B800ABAAAA3EB76DDB3E9A99193F0000404093
:1020C8000040763F4F38763FC623F6B8A85005083B
:1020D800B05005082DE9F04F91B0009302F00403C9
:1020E8000293C2F3C2030133840705460E46DDF8A6
:1020F80068800392059340F0BB81041D30B1072925
:1021080009D86FF01B0011B0BDE8F08F01F0070689
:102118003444C6F10806009B4FF000094FF0040A4A
:10212800591E4FF0FF334F460193CB465346CDF827
:1021380010900DB1009A22600598002800F3E880FD
:102148009848009A824203D397488242C0F0E080C0
:10215800039AA4EB050E92074FEA9E0000F1038153
:102168000F2F00F2B180002D00F0058107F1400229
:102178000DEB020C019A0CF8200C0CF8102C0498AA
:1021880001300490E7E07A285DD84B280ED847281C
:1021980059D829282DD8252852D054D820287AD083
:1021A8002338D0F1000B4BEB000B74E04C382E2891
:1021B80049D8DFE800F07048484848484848484847
:1021C80048484B484848484848484859484B4B595C
:1021D8005959704B6D487048184B184848827F4BC6
:1021E80048484B487F0000204FF0000B4FF0040A8E
:1021F80038E001222A38C0B202FA00F010EA0E0FC5
:1022080049D110F0625C2FD110EA020B43D060462E
:10221800013C5444B4FBFAF40AFB04F4002D61D0E9
:10222800A3EB050CA444B4453FF66BAF002868D176
:10223800042B47D158F8043B2360042304342AE0D4
:10224800019A013A01924FF0000B24E011F8010CB9
:102258006C2834D1002011F8023C83466C2BC5D180
:102268004FF0080A5346D3E708F1070828F0070893
:10227800073424F00704F8E802AB35B10698204487
:10228800B0423FF63EAFC4E900AB4FF0000B083454
:102298004FF0080A534611F8010F002878D0BBF117
:1022A800000F7FF470AF2528F5D14FF0010B019B8B
:1022B800013301934FF0040AECE7584694E70020F5
:1022C8008346A5E7082B02D06FF015001BE708F13D
:1022D800070828F00708F8E80223C4E900230823C0
:1022E8000834D8E768B9042B02D108F10408A4E738
:1022F800082BE9D108F1070828F0070808F10808B1
:10230800EDE7059A013A059258F8042B009210E778
:10231800039A900720D54FF0010CA4EB050E4FEA65
:102328009E00BEF5007FCFD20F2FCDD8F5B107F1B3
:1023380040020DEB020E019AC0B20EF8200C0EF806
:10234800102CBCF1000F3FF41AAF60F07F000EF8BC
:10235800200C09F101090137C5F108024FF6DA7EB0
:102368000434069297E74FF0000CDAE7BCF1000F4F
:1023780001D00136EFE7029802360028EBD1009829
:10238800CDE90631FEF7E6FFDDE906310644E2E76E
:10239800631BB3F5806F97D245B9A6F10804E0181E
:1023A800B1E600BFB8AB040824DA0508029A9B0816
:1023B80028602B709DF81030C2B1EB7085F8029040
:1023C800B9F1000F05D0002208A8C5F1010C974209
:1023D8000ED14FF0000AC5F101030DF12008019359
:1023E8000DF1300B574512D1601B8CE66B70E5E799
:1023F80010F8013B190608D50CEB040EB64503F09E
:102408007F033FF67EAE04F8013B0132DFE7B9F106
:10241800000F03D098F90020002A17DB029BD3B1E4
:102428001AF80B2004F8012B0022019B18191044FC
:10243800B0423FF666AE98F80000009904F8010B28
:102448002046039248F061FA039A14440AF1010AFB
:1024580008F10108C6E798F8002055F822300093E3
:10246800029B009845F82230FEF774FF421CDCE717
:102478006FF00D0047E600BF2DE9F04F97B000AFB1
:10248800D7F880B03B62CBF3C0030446894690F886
:1024980002A0FA62BB6141B9457800780AEB800076
:1024A80020444D4517D8A0EB0409E378FB61BAF145
:1024B800000F02D01BF0010F16D1FB6953BBFB6A5A
:1024C8001BB1494620463A6A98474D4628465C372C
:1024D800BD46BDE8F08F461C3046FEF73BFF013095
:1024E800304409F10109DCE7626823787A62FA6A04
:1024F8009900796104EB8301002A40F001810E46BE
:102508004FF000084D4601EB0A094E454CD101EB4E
:102518000A0610E01BF0020FD1D023789A007A61E6
:10252800626804EB83017A62FA6A002A77D14D4621
:10253800904601EB0A061BF0050F0CBF022301238E
:10254800FB62FB6906EB430A0BF00203BB625645CC
:10255800BCD016F8021B16F8013C54F82390994B8E
:10256800994502D3984B994536D3BB69002B40D087
:10257800786A32F08FFD00283BD0E9468AB06A4677
:10258800924B53617B6AC2E906314FF4007313849E
:102598008F4B42F8103F00234FF412518D4800F042
:1025A8009DFC023DCD46D2E716F8013BF96254F88E
:1025B8002300FEF7CFFED7F88430F96A01304BB11B
:1025C800D7F8883098453EBFD7F8843023F81800EC
:1025D80008F10108054498E7BB6923B1786A32F02D
:1025E80059FD0028C9D11BF0010F05D1FB6AED1A6E
:1025F800ADE7BB6A002BAAD04846FEF7ABFED7F87A
:10260800843053B1D7F8883098453FBFD7F8842035
:10261800431C22F8183008F10108054497E7BAF17D
:10262800000F73D01BF0040673D0D046002607F1C4
:10263800480052463B61B96248F067F9B96A3B699C
:1026480001EB0A02BA62FA69F9695200FA60BA6AD9
:1026580002EB41023A610BF00202BA603A69B96AC8
:102668008A4258D162781BF0020F18BF00217A62A3
:1026780008BF4FEA5801B2181BF0010FD2B240F060
:102688009F801BF0040F14BF40460020BB6162709E
:10269800A070E17020463A6A7969FB6A9847051E7E
:1026A800FFF614AFBB69414623707B6A3A6A6370D0
:1026B800FB6984F802A0E37007F14800FB6A9847B9
:1026C800B0F10008C0F2BA807B69A9EB0A01C91A07
:1026D800FB683A6AC91AD7E90A0398470028C0F282
:1026E800AF804FF0000BA84408EB000507F1380A4B
:1026F800B34571D300213A6A0846FB6A9847E5E674
:1027080056464FF0000807F1380092E75646D04683
:1027180096E7B04694E7BA6A12F8021B12F8015C11
:10272800BA6254F82500274A904202D3264A9042BA
:102738001ED3BA6932B1786A7B6032F0ABFC7B6831
:1027480000288BD1BA6802BB08F1280207F1300CC7
:1027580008F10100944407F1580208F1020852FAFE
:1027680080F00CF8101C5FFA88F800F8105C75E728
:10277800BA693AB1786A7B6032F08CFC7B680028D1
:102788007FF46CAF1BF0010F09D006F1280207F1A6
:102798003000711C161806F8205CCEB25EE71BF0FC
:1027A800040F3FF45BAF08F1280207F1300008F18D
:1027B800010102EB000808F8105C5FFA81F84DE7A8
:1027C800002063E7B8AB040824DA0508B45A050802
:1027D80004000001CCB004081BF80A3054F8239018
:1027E80087F83730D7F884302BB3D7F888309B4533
:1027F80021D2D7F8843033F81B8001213A6AFB6A6A
:1028080007F13700984700281ADB0544B8F1000F94
:1028180006D14846FEF79EFD00F101081FFA88F828
:10282800414648463A6AFB6A9847002808DB05444F
:102838000BF1010B5CE74FF00008DEE7454645E683
:10284800054643E6014B1860704700BF8001002031
:1028580080B505460E46174698460BF007F903461D
:1028680001F050FB0446DFF81890424649F8003062
:1028780039463046A84754F8090001F017FA00BF56
:1028880008000000044608B5EFF31183102383F312
:102898001288BFF36F8F35F0A0FE204601F0F4F9DF
:1028A800024832F01EFC33F09EF9FCE7685B05082D
:1028B800034A0020536823F002035360704700BFA7
:1028C800004004E010B5EFF31184102383F312885D
:1028D800BFF36F8F084803683BB9084A916A41F013
:1028E80001019162916AC907FCD50133036084F341
:1028F8001188BFF36F8F10BDEC320020000802462C
:1029080010B5EFF31184102383F31288BFF36F8F90
:1029180011490B68A3B90122104BD3E8EF1F002916
:1029280003D1C3E8E02F0028F7D104D102210C4AD3
:102938000C4832F099FF84F31188BFF36F8F10BDF4
:10294800012B08BF084803F1FF3302BF826A22F057
:10295800010282620B60EEE7EC320020E8320020D0
:102968009C5B050874B104080008024607B505F029
:1029780067FD0E4B0E4A1A600E4BD3F8942042F0B6
:102988000402C3F89420D3F8943003F004030193AD
:10299800019B094BDA6A42F00102DA629A6822F076
:1029A80002029A6003B05DF804FB00BF3006002005
:1029B80000093D00000C0246000802462DE9F047D8
:1029C800044607464FF00109DFF8508014B938462D
:1029D800BDE8F08794FAA4F5B5FA85F509FA05F388
:1029E8002E0108EB05156FEA030A24EA03042B7B82
:1029F800002BEBD058F806301B694BB94644736876
:102A080002222846196807EA0A0732F0BDFEDDE708
:102A1800284698470028D9D1F0E700BF04B2040837
:102A280030B5002289B00F490F4837F001F800226D
:102A380000230024CDE906230E230C4DCDE90334F1
:102A48004FF440722846CDE90144094B09490094E6
:102A58000AF042FD0849284636F038FE204609B0FB
:102A680030BD00BF852A00082826002080210020CC
:102A7800892D0008C0470020DD5B050801480AF0E1
:102A880089BA00BF341000202DE9F047804620485D
:102A98000F4632F055FE0646002832D0002528465B
:102AA800BDE8F087237B83B12368DB680BB1204640
:102AB8009847636883F8069023681B69CBB96368F5
:102AC80002222046196832F05FFE01361034544560
:102AD800E8D3B8F1000FE2D0002DDFD02846FFF789
:102AE8006DFF0546002FF7D00021642036F0A2FEC6
:102AF800F2E7204698470028E1D009FA06F31D437B
:102B0800E3E705464FF00109024CDFF80CA0DEE7C9
:102B18000033002004B2040814B20408014B53F82F
:102B28002000704734B2040808B5034608462BB1A4
:102B3800044A136000F068FC002008BD6FF015001F
:102B4800FBE700BF8401002010B5044C237813B9BB
:102B580003480AF01FFA0123237010BD3A3F0020F2
:102B68003410002010B50446094832F0E9FD3CB1A4
:102B7800084BD3E8EF1F0139C3E8E21F002AF8D158
:102B8800054836F061FFBDE8104004480AF002BA73
:102B9800F8320020FC3200202826002034100020C3
:102BA80000200146034BD3E8EF0FC3E8E21F002AD9
:102BB800F9D17047F832002070B5FFF7F1FF0546EC
:102BC800074C084EB44200D370BD63685B792BB1E3
:102BD80023685B6813B12946204698471034F1E70B
:102BE80004B2040814B2040810B5044C0449204681
:102BF80032F089FB034B1C6010BD00BF4C0F002056
:102C080020B20408F032002000230D4A10B51370DA
:102C18000C4A4FF47A7113600B4A0C481360FFF7A3
:102C280083FFFFF7E1FF0A4B0A4918468B4200D39E
:102C380010BD1A1A5C681211013222711033F5E7BF
:102C48003B3F0020F8320020FC3200205B5703088D
:102C580004B2040814B20408014600220023014803
:102C680032F072BB4C0F0020014832F00BBC00BFA1
:102C78004C0F0020024B0146186832F05EBC00BFC2
:102C8800F0320020014832F093BC00BF4C0F002006
:102C980070B5244B1878002842D0FFF7E5FF0546A9
:102CA80000283AD1204B214C1B68002B12DD36F04E
:102CB80077FE0A220023FEF7E1FAD4E90032C01AAF
:102CC80040F2E93361EB0201984271F1000101D34E
:102CD800FFF772FFD4E9003213F57A7342F100026C
:102CE800C4E90032BDE87040FFF7CCBF63685B7988
:102CF80023B12368294620461B6898471034B442FC
:102D0800F4D32846FFF7B6FF094BD3E8EF1F013984
:102D1800C3E8E21F002AC5D0F7E7064C064EEEE7E7
:102D280070BD00BF3A3F0020F83200202026002066
:102D3800FC32002004B2040814B2040870B50D4D2A
:102D4800297861B90120FFF79FFE0B4C0B4EB44266
:102D580006D3FFF79DFF0028FBD101232B7070BD20
:102D680063685B791BB1236820469B6898471034D9
:102D7800EDE700BF3B3F002004B2040814B204088A
:102D880000212DE9F0470846FFF77EFE044658B3B8
:102D98004FF4FA784FF0000901F0B4F81B4B1C4AC5
:102DA8001B58136033B11B4B1B68092B02DD1A48F3
:102DB8000AF0F0F80025194FDFF85CA044B120466E
:102DC800FFF7FCFD044618B94FF0FF384FF0FF3904
:102DD800FFF75EFF064628B9B5B942464B4650464E
:102DE8000AF012F93546E9E74FF0FF384FF0FF399E
:102DF800D2E72B689B691BB10022284611469847E9
:102E08001035BD42F5D3E8E7054DFAE708000000A4
:102E1800F4320020FC3200203410002014B20408E0
:102E280004B2040813B5184832F08AFC174B1B7813
:102E380073B1EFF31184102383F31288BFF36F8FFC
:102E4800FFF726FF84F31188BFF36F8F02B010BD20
:102E58000F4B1B68002BF9D050B9002200230D48F6
:102E6800CDE9002342F2107200230BF00FF9EDE7D1
:102E78000928EBD1074836F0E7FD074802B0BDE85E
:102E880010400AF087B800BFFC3200203B3F00200A
:102E9800F4320020282600203410002010B5064BFC
:102EA80004461B6898472146A060044832F0CBFAD4
:102EB800BDE81040FFF7B6BF840100204C0F00208A
:102EC800044A054B9B1AB1EBD30F34BF52F83100BB
:102ED80000207047BCB0040804B204082DE9F04F84
:102EE8008FB0C1F34A2804AF0D469146B8607B60A5
:102EF8000C0DB8F1000F63D000264FF0040B4FF013
:102F08000A0A07F11403C7F80C80C7E907667E624E
:102F18000193CDF808B0CDF800A007F11C033246A4
:102F28004846F968FFF7A8FAB0F5006F03461CD3C6
:102F38006C468AB0D9F8041004AB26481A46C3E98F
:102F4800050140F2FF71D9614FF400711984224BD9
:102F580042F8103F4FF4125133462048FFF7BEFFA6
:102F6800A5462C37BD46BDE8F08FC0F30A0804F12A
:102F78001700184420F0070080083B60FFF76CFE3C
:102F880068F35325044690B13B6800F11001C7E986
:102F9800083607F11403F961CDE900A3CDF808B0AC
:102FA80048460F4AF96807F11C03FFF765FA68F30A
:102FB80053252A4620467B68B96832F005FCD0E7DD
:102FC80004F1170020F007008008FFF745FE0446CB
:102FD800EDE700BFEE5B05080400000124B104081A
:102FE800A35703082DE9F04F87B00446DDE9105ACE
:102FF800DDE91279934698460391BFB13B465246A4
:1030080010210020CDF80090CDF81490FFF762F859
:10301800B0F5006F06460AD340F2FF730221174A43
:10302800174807B0BDE8F04F32F027BC3E4605F11F
:103038001700304420F007008008FFF70DFE04F069
:1030480007040BF0070BE40044EA8B1444EA462417
:1030580044EA0554054640B13FB13B465246314625
:10306800CDF800901030FFF735F843462246284641
:10307800039907B0BDE8F04F32F0A6BB2D5C0508F8
:1030880024B10408406820B1034BC01A40F3CF00B4
:1030980070474FF0FF307047BCB004080EB403B55A
:1030A80003AB53F8042B01460448019301F062F97D
:1030B80002B05DF804EB03B0704700BFE5580308A1
:1030C800CA0605D48B064CBF02490349FFF7E6BF81
:1030D800704700BFBDB705083B7905082DE9F04FDB
:1030E80089B09B46149B9DF84CA00693159B0446FB
:1030F8000593169B0D469046179E0493BAF1000F50
:1031080000F09D8006F48073079332F03BFB06F0D5
:103118000209024600283ED020469149FFF7BEFF2B
:103128000746B9F1000F08D016F0440F35D12A46EA
:1031380020468C49FFF7B2FF074406F0010353B15C
:10314800894B204653F82A20884B8949002A08BF12
:103158001A46FFF7A3FF06F48073002B49D006F048
:103168000803002B63D1B8F1000F66D04246204611
:103178008049FFF793FF0546069B3D44002B6DD120
:10318800049B002B73D1F30700F1E48031462046FD
:10319800FFF796FFD8E00746C3E7774B1868002883
:1031A800CAD0764B4FF47A791B684FF03C0CB5FBCC
:1031B800F3F5B5FBF0F14FF4616300FB115509FB22
:1031C80005F5B1FBF3F2B5FBF0FE03FB121100FBB2
:1031D8001E55B1FBFCF309FB05F5B5FBF0F50CFB3F
:1031E800131120460091CDE901E56549FFF756FF27
:1031F800A2E706F00803EBB1624B204653F82A20F9
:103208006149FFF74BFF0546B8F1000F05D042466C
:1032180020465849FFF742FF0544BBF1000FABD0E9
:103228005A4620465949FFF739FF0544A4E74FF0AD
:10323800000BE1E706F00805E6E745469CE7BBF129
:10324800010F069B06D1002B64D1049B002B7BD079
:1032580000250CE0002BF8D04D485CE04D48069B5B
:1032680022464D4931F0E5FE049B002B68D0DFF87B
:103278002C81DFF82C91049F3146102F204628BF5F
:1032880010274FF0000BFFF71BFF5D4545DC059B42
:10329800494620461A78FFF701FF4FF0010B1BF053
:1032A800070F03D141462046FFF7F8FE5F453BD99B
:1032B800059B4946204613F80B20FFF7EFFE0BF15C
:1032C800010BBBF1100FEAD14FF0000B2046354936
:1032D800FFF7E4FE5A46059B20469A5CA2F12001BE
:1032E8005F2928BF2E223049FFF7D8FE0BF1010BCA
:1032F800BBF1100F1DD01BF0070F03D1414620462C
:10330800FFF7CCFE5F455A46E5D841462046FFF711
:10331800C5FEEBE71F485546A1E741462046FFF7A3
:10332800BDFE0BF1010BB0E720462049FFF7B6FEC2
:10333800C5E7059B3B440593049BDB1B04939AD18B
:10334800BAF1000F7FF41FAF204609B0BDE8F04F77
:1033580032F0B7BA2046054A0549FFF79FFE15E740
:103368006A5C05086E5C050844B20408655C0508DB
:10337800FFB90508935C05080833002004330020D2
:10338800775C050858B20408975C05089D5C050839
:1033980013590308E55803087D43000899D0050828
:1033A800A25C0508A85C050852B6050897D0050870
:1033B80042F20F7373B58B4228BF0B46056804466B
:1033C800052168460D4A2FF001F90646636828462C
:1033D8000B225B680A4932F066FA6368324669462E
:1033E80028465B6832F05FFA63681B2228465B68F0
:1033F800044932F058FA02B070BD00BFA170050848
:10340800C65C0508AA5C050800210123064A90420B
:1034180006D8064A01B901231360054B18607047A6
:10342800012140085B00F2E740420F00043300200E
:1034380008330020F8B50D460446064F4618B44236
:1034480001D12846F8BD14F8011BBB6801485B6828
:103458009847F4E7A4AE0408014B036000207047C6
:10346800A0B204082DE9F34205460E4600244FF0A9
:103478001409084B084F1B680193019BA34202DC07
:1034880002B0BDE8F0823868314609FB0400A8475D
:103498000134F2E7A0B204089001002070B5104B87
:1034A8000D461C68B4B10F4B196800238B4202DB30
:1034B8006FF0010070BD224612F8146B864202D0EC
:1034C80014460133F2E7E06835F071FE28B10020B8
:1034D8002C60EFE76FF00C00ECE76FF01200E9E703
:1034E80090010020A0B2040810B5436888B0029388
:1034F80083680C46CDE9033200230A68C068CDE929
:103508000623054901AA059334F077F9079808B905
:10351800059B236008B010BDAD5A03082DE9F84398
:103528000646FDF717FF0546EFF31188102383F3CE
:103538001288BFF36F8F114B1C68D3F804909C421C
:1035480008BF002434B988F31188BFF36F8F204671
:10355800BDE8F883A7683846FDF7FCFEA84206D107
:103568002A463946304647F01CFA0028EBD04C452D
:1035780001D02468E6E70024E5E700BF94010020B5
:103588002DE9F0410E461546FFF7C8FF044628B35B
:10359800C3681BB35F690FB3062E07D0072E20D070
:1035A8002A4631463B46BDE8F0411847838A3BB975
:1035B8002A463146B84750B9A38A0133A38206E0A8
:1035C8004FF6FF72934204D00133A3820020BDE876
:1035D800F0810121114A124832F046F96FF01500C6
:1035E800F5E745B12A7832B10022828231462A466F
:1035F8005B699847EAE7A38A012B08D12A46072185
:103608002046B8470028E2D1A38A013BD6E70BB190
:10361800013BDAE70221034ADDE700BF245D050824
:10362800DCB00408465D050810B5044608B180689A
:1036380038B9104A1048012132F016F96FF0150018
:1036480010BDFFF76BFF08B10C4AF3E7A082EFF358
:103658001181102383F31288BFF36F8F084B5A68C8
:10366800C4E9003214605C6081F31188BFF36F8F86
:10367800E6E700BF645D0508DCB004087D5D050869
:103688009401002008B50348034A0021121A32F0B9
:1036980080FA08BD40120020B4430020074808B54E
:1036A800074A0849121A32F076FABDE80840064877
:1036B800064A0749121A32F06EBA00BF000000200D
:1036C8001812002024DA050800000020000000205D
:1036D80024DA05082DE9F04706460C4600AF002914
:1036E80036D0D1E90012E9468AB06D46A3684FF09A
:1036F800050AA8461F48C5E90723C5E9050148F892
:1037080010AF002342464FF421511B48FFF7E6FB58
:10371800D4E90312CD466369AD461848C5E90723C5
:10372800C5E90501C5F810A0002342464FF4215110
:103738001148FFF7D3FBCD46E3690121104A0E4833
:1037480032F09BF8A36901210E4A0B4832F095F834
:10375800012E07D1EFF305830B4A31460648103B8B
:1037680032F08BF82146304609F062F8BD46BDE8D4
:10377800F08700BFAC5D050854B10408DB5D05089F
:103788000A5E0508195E0508475E050830BFFFF7A1
:10379800FDBF00BF2DE9F04105460B4EDFF82C8038
:1037A800324606EB0807CC1B2046094947F0ADF81E
:1037B800A01942460021083C47F0CEF8C5F89040D1
:1037C80007F10800BDE8F0810000000008000000D3
:1037D80014B20408054B5A699B689A421FBF044AF1
:1037E800536843F080535360704700BF4C37002044
:1037F80000ED00E070B52A4C06460D4629482A49D6
:1038080032F0D6F9A36ADB0647D52648274932F0B5
:10381800CFF91120A36A1C0704D52248244932F0A5
:10382800C7F912201E4CA36A990712D521491D48D1
:1038380032F0BEF9636BA26A120609D501211E4A4D
:10384800184832F01AF81EB1A36A23F08003A36265
:103858001320134CA36ADE0704D51248174932F027
:10386800A7F91420A36A9C0604D50E48144932F01F
:103878009FF915200A4B9A6AD10658BF9A6A9A6A24
:10388800920642BF5A6A22F400525A629A6A42F079
:10389800FF029A6200232B7070BD1020BAE700BFA8
:1038A80000ED00E054B104085A5E0508705E050892
:1038B800A35E0508B65E0508CE5E0508E45E050849
:1038C800035F050810B5244C2449254832F070F9E7
:1038D800A36A99013ED52248224932F069F91E208F
:1038E800A36ADA0104D51E481F4932F061F91F2086
:1038F800194CA36ADB0204D519481C4932F058F95F
:103908000220A36A1C0304D51548194932F050F95E
:103918002120114CA36A590304D51148154932F0E6
:1039280047F92220A36A9A0304D50D48124932F0B8
:103938003FF92320084CA36ADB0304D508480F4944
:1039480032F036F92420A36A6FEA03436FEA13437F
:10395800A36210BD1D20C3E700ED00E0325F05083B
:1039680054B104084A5F05085D5F0508775F0508DC
:10397800A15F0508BF5F0508E45F0508FE5F05084D
:1039880070B5294C06460D462848294932F010F9E9
:10399800A36AD9043CD52548264932F009F91720ED
:1039A800A36A1A0504D52148234932F001F91820E1
:1039B8001D4CA36A9B0512D51C48204932F0F8F823
:1039C800A36BA26A100409D501211D4A174831F0DA
:1039D80054FF1EB1A36A23F40043A3621920124CBA
:1039E800A36A590504D51148164932F0E1F81A209E
:1039F800A36ADA050ED50D48134932F0D9F81B2011
:103A0800094A936A43F47F43936200232B7070BD85
:103A18001620C5E7A36A9B04F2D504480B4932F087
:103A2800C7F81C20ECE700BF00ED00E054B1040823
:103A3800296005083F600508A35E05085060050871
:103A4800696005087E60050899600508035F050838
:103A58002DE9F0418AB0654B0446D3F8048000266E
:103A680000AFC8F3080586F31188BFF36F8F02F023
:103A78007F43B3F17F4F07D102F00C03082B12D11B
:103A88005B495C4832F094F8002634460023FB7109
:103A9800EB1E092B00F28980DFE803F00A7F827BA6
:103AA80087878787878510074CBF0C460126EDE777
:103AB8005149504832F07CF800234C4DFB71EB6AB9
:103AC8009A0705D54D494B4832F072F8002331E08A
:103AD800EB6A002B01DA4A49F5E7EB6A5B00F5D59A
:103AE8004849444832F064F86B69A26943F480732A
:103AF8006B61BFF34F8FBFF36F8F6B6932F8022C86
:103B080023F480736B61BFF34F8FBFF36F8F4DF654
:103B180002739A4207D0AB6ADBB26BB30120F91D7E
:103B2800FFF768FE37E023680121374A314831F052
:103B3800A4FE2368FA79DAB907F1080504F1200C24
:103B48002A4620686168083403C264451546F7D1DF
:103B58007A6A002E45D0C2F3080121B96FEA5222D1
:103B68006FEA42227A62184607F10801FFF7B2FDB0
:103B78002837BD46BDE8F081AB6A13F47F4F04D007
:103B88000120F91DFFF7FCFE05E0AB6AB3F5803FA5
:103B98009CD3FFF797FE0346CCE70020F91DBFE74B
:103BA8000020F91DEEE719498DE7194A18F4F87F46
:103BB800E8468AB0174B18BF13466A461649103DA7
:103BC800C2E905134FF400731384144BD56142F80E
:103BD800103F00234FF411510648FFF77FF9C546FF
:103BE80074E722F4FF7222F00102BBE700ED00E067
:103BF800DF60050854B104080A6105082161050859
:103C080042610508506105086F6105088B61050868
:103C1800C6600508B1600508AF6105080400000129
:103C2800064B5A6942F010025A615A6942F480629E
:103C38005A615A6922F008025A61704700ED00E0A3
:103C4800EFF30880EFF3098101B57246FFF700FF33
:103C580001BD00BF0A4880F30888102080F311884E
:103C680008484FF40061401880F30988EFF3148086
:103C78000221084380F31488BFF36F8F00F0C4F863
:103C8800E0BE0020C0560020BFF34F8F0549064B09
:103C9800CA6802F4E0621343CB60BFF34F8F00BFE2
:103CA800FDE700BF00ED00E00400FA05084B9B6843
:103CB80083420BD1EFF3058343B1064B5A6842F0B8
:103CC80080525A605A6A22F400425A6209F0D4BEFD
:103CD8004C37002000ED00E016498A684FF03000AC
:103CE8001044EFF3098C80E8F01F102080F312884D
:103CF800BFF36F8F104F4FF000664A698A603E60CD
:103D0800D2F890000D4C2060D2F894000023C2F83D
:103D1800943080F3118802F1300090E8F01F8CF3A2
:103D2800098802F1000004B531F04EFFBDE80440F7
:103D3800704700004C37002004ED00E038330020C5
:103D48001EF0040F0CBFEFF30880EFF309808169C0
:103D580011F8021C0229FFD001B5724631F01DFF8F
:103D680001BD00BF0028ACBF00F16040064B4FEA20
:103D78000111C9B2ABBF00F5614000F00F0080F837
:103D880000131954704700BF14ED00E040B200283A
:103D980007DB01234109034A00F01F00834042F872
:103DA8002130704700E100E040B200280CDB01221E
:103DB8000649430900F01F008240203341F82320C0
:103DC800BFF34F8FBFF36F8F704700BF00E100E074
:103DD800054B420953F82220012300F01F0003FA83
:103DE80000F01040704700BF00E100E0044B054AB6
:103DF80023F07F039360BFF34F8FBFF36F8F70473C
:103E08000000000800ED00E008B5FFF7EFFF0B4ADF
:103E1800D2F8883023F47003C2F88830EFF31483A3
:103E280023F0040383F31488BFF36F8FFFF72AFC92
:103E3800FFF734FC00F048F808F01AFE00ED00E047
:103E480042F8203C009B0B4942F81C3C019B21F0A6
:103E5800010142F8183C029B42F8081C42F8143C45
:103E68004FF0807342F8043C0023203A0265C0F802
:103E7800943070475928000800B50E4B15469860D5
:103E8800D0F890200C4B0E461A60D0F8803083F39F
:103E98000B882C4686F309880020044B9847204657
:103EA800002100220023024C20470000E15B0308A8
:103EB800592800084C370020383300201022014BC5
:103EC8001A61704700ED00E0002310210348C21872
:103ED80001337D2B82F80013F9D1704700E100E02F
:103EE80008B5EFF30583064A103B02EBC30152F80D
:103EF800330049688847BDE80840FFF76BBC00BF3E
:103F0800340B002001480068704700003833002057
:103F18001FB5094C094A23460121094800F012F946
:103F280000230393074B0121E41A01A8019302948B
:103F380000F012F904B010BD00000C2000000020B1
:103F4800F4B204084012002010B50C7A0B6804F093
:103F58001F0223F01F031A43CB68640923F01F03D1
:103F6800054943EA440343F00103C1F89800C1F846
:103F78009C20C1F8A03010BD00ED00E010B50A4B40
:103F8800D3F89030C3F30723013B984208D90121A5
:103F98000346064A064831F070FC6FF0150010BD64
:103FA800FFF7D2FFFBE700BF00ED00E0C6610508A0
:103FB8003CB104082DE9F04F8946144606464FF0F7
:103FC8000008514D85B0C84527DAD6F804A0BAF1E3
:103FD800000F44D0BAF11F0F17D91AF01F0F14D1D0
:103FE800D6F800B01BF01F0F0FD1584631F008FE6D
:103FF80007460AEB0B00013831F002FE874210D069
:104008006FF01507414A3B4601E04346404A01210B
:10401800404831F032FC6FF01504204605B0BDE889
:10402800F08F17F1160FEDD0BC42EBDDC5F8987094
:10403800D5F89C10C5F89870D5F8A03021F01F016C
:1040480043F01F0BD6E900321A44994202F1FF3AB5
:104058001DD1D34507D13146F8B231F0DAFD08F168
:1040680001080C36AFE73146C5F89870D5F89C3092
:1040780022F01F0203F01F031343C5F89C30E0B27F
:1040880031F0C7FD10F1160FC5D0441CE7E7C5F89D
:104098009870D5F8A020013B23F01F0302F01F02FF
:1040A8001343D3453146E0B2C5F8A030E8D031F02B
:1040B800B0FD10F1160FAED0C5F89870D5F89C2059
:1040C8009DF808300BF1FF3B62F304038DF80830CC
:1040D800D5F8A0309DF808205B0863F347128DF8E7
:1040E8000820D6E900321344009323F01F035B44F1
:1040F800A3EB0A03013023F01F036946C0B2039300
:10410800FFF73CFFBEE700BF00ED00E012620508C4
:10411800EC6105083CB104080522044BC3F894205F
:10412800BFF34F8FBFF36F8F704700BF00ED00E004
:10413800BFF35F8F0022024BC3F89420704700BF83
:1041480000ED00E010B5034C2278FFF733FF207034
:1041580010BD00BF3D3F00202DE9F74F294D8A468D
:1041680006464FF00008AB46274FD0451BDAD6F875
:104178000490B9F1000F3FD031680846019131F041
:104188003FFD0199044609EB0100013831F038FD83
:1041980084424FF014021D4B08D002FB08F36FF065
:1041A80015024BF8032003B0BDE8F08F14F1160F89
:1041B8002C60F8D01978A142F5DD02FB08B0C7F8E9
:1041C8009840C7F89840D7F89C4000F10801007B58
:1041D80064F304000871D7F8A0000C79400860F374
:1041E80047140C71D7F89C1021F01F016960D7F8AB
:1041F800A01021F01F01296108F1010814350C36BF
:10420800B3E700BF3C33002000ED00E03D3F002055
:10421800F0B55349534CD1F890302568C3F30723C0
:104228009D4287B000F299800020FFF781FF4E4B36
:10423800C1F8C030854216D14C4C01A82570FFF753
:104248000BF9002506464A4FAE4213D100202378C9
:104258004349D1F89020C2F30722934277DBFFF756
:104268005BFF002046E0616801EB0011FFF76CFE80
:104278000130DFE70199280101EB0513DA683A40BC
:10428800B2F1807F52D00AD8B2F5001F34D0B2F50F
:10429800800F3ED0B2F5801F12D00135D4E7B2F1BD
:1042A800006F43D0B2F1805FF7D15A689B68095814
:1042B800013B22F01F00034423F01F03012032E0DA
:1042C8005A689B680958013B22F01F0003440120EB
:1042D800844623F01F0340EA4C10CDE902218DF8F3
:1042E800100002A920780593FFF748FE00282ADA73
:1042F8006FF0150007B0F0BD5A689B680958013B7C
:1043080022F01F0003444FF0020C012023F01F038A
:10431800E1E75A689B680958013B22F01F000344F3
:10432800022023F01F034FF0000CD4E75A689B6863
:104338000958013B22F01F0003444FF0030C0120F1
:1043480023F01F03C7E7237801332370A5E7C1F8DB
:104358009830C1F8A00001337BE74FF0FF30C9E780
:1043680000ED00E000B30408AAFF44003D3F002030
:104378000000F0FFF0B587B007460E46144600214E
:10438800102268461D4646F0E7FA02238DF80230EF
:10439800054B2A4621466846CDE9047601932EF05E
:1043A8001BFA07B0F0BD00BF535C030808B5024B09
:1043B8001B689847002008BD50330020034B044A6F
:1043C8001860937843F002039370704750330020CD
:1043D8009C01002008B5054830F083FE002383F3D4
:1043E8001188BFF36F8F0423184602DF4462050863
:1043F80008B50649064821F00701C1F1005202F547
:10440800402230F0BEFD002008BD00BF3FD700208D
:10441800543300204FF0FF324FF0FF33014808F0CB
:10442800C3BC00BFAC010020014808F031BD00BF8B
:10443800AC01002038B50546FFF7ECFF2A460821F5
:10444800074830F0EAFC044628B925B1FFF75AFDC1
:104458000C22044B1A50FFF7E7FF204638BD00BF77
:10446800543300200C00000038B504460D46FFF711
:10447800D1FF21462B460822074830F04AFD044662
:1044880028B925B1FFF73EFD0C22044B1A50FFF75F
:10449800CBFF204638BD00BF543300200C0000007D
:1044A80010B50446FFF7B6FF2146034830F054FC28
:1044B800BDE81040FFF7B8BF5433002070B541691C
:1044C8000446867A0A4D59B1437ADB0706D42C2371
:1044D80003FB06535B6A1B689B689847002363616C
:1044E8002C20214606FB0050BDE8704035F053B83B
:1044F800881000202C22024B02FB0030704700BFBE
:10450800881000202C21827A054B01FB02339A6A1D
:104518001B7F801A1B3323F00303B0FBF3F07047B3
:104528008810002038B52C24827A064B04FB02330D
:104538005B6AD3E901240C601568FFF7E3FF04FB0D
:10454800005038BD881000202DE9F04385B005469D
:10455800684690461C46039135F024FADDE9006769
:10456800EFF31189102383F31288BFF36F8F6B8BDE
:10457800002B41D02A8B9A4225D9002200232846B5
:1045880008F0D6FC0446F0B189F31188BFF36F8FA9
:10459800039B002B41D032463B46684635F027FA4C
:1045A8002C21A27A254B204601FB02335B6A03A922
:1045B8001B681D68DDE90023A847606170BB2046C1
:1045C800FFF77CFF24E0698B4B1E6B8389F311880E
:1045D800BFF36F8F2B7F2A8BAC6A1B3323F0030347
:1045E800521A02FB0344154B154AEB1A9B1053430E
:1045F800A3722B7FE372CBE789F31188BFF36F8F28
:1046080023464246284608F093FC04460028BFD1BA
:104618000024204605B0BDE8F0836361012300252E
:104628002381039B29466382E27A656004F11800BE
:1046380046F092F963692582E360EAE78810002072
:10464800A38B2EBA70B52C250C4C00B970BD037A1B
:104658004668002BFAD0013BDBB20372002BF5D180
:10466800C3604360837A05FB03431B6A13B1984711
:104678003046EAE7FFF722FFFAE700BF881000207C
:10468800F7B506460D461446124F384634F08FFDEE
:10469800E0B1BB68314638461B68AAB29847002883
:1046A80002DB002003B0F0BD002CFBD1AC42F8D2F5
:1046B8002F1B042F28BF042706F0B4F83A460190B0
:1046C80001A9301946F021F93C44EFE76FF01200D8
:1046D800E8E700BF50AE040838B5044609F0BCF856
:1046E800204631F03EFBA069C8B194F87030DB0772
:1046F8000DD50221144A154831F031FB6FF07705CA
:10470800201D31F035FB09F0BBF8284638BD34F0E0
:104718004EFD38B901210E4A0C4831F020FB6FF0EC
:104728001205EDE7204601F02FF805460028E7D1ED
:1047380028220146A01846F00FF994F8703043F08B
:10474800010384F87030DBE764620508D4B104081B
:104758008E62050838B5054609F07EF8284631F01E
:1047680000FB95F87030DA070DD40221184A194871
:1047780031F0F5FA4FF0FF34281D31F0F9FA09F05D
:104788007FF8204638BD9B0707D50221124A1148F9
:1047980031F0E5FA6FF07704EEE7A86932F0FEFC35
:1047A800044628B101210D4A0A4831F0D8FAE3E756
:1047B800284631F067FC044618B1A86932F017FDA5
:1047C800DAE795F8703043F0020385F87030D3E7E4
:1047D800B1620508D4B10408D7620508FD6205086E
:1047E80038B590F8703004469B0708D40221144A63
:1047F800144831F0B4FA6FF07705284638BD31F027
:10480800B0FA0021204601F05DF920B101210E4ADD
:104818000C4831F0A4FAA06932F0E9FC054620B151
:1048280001210A4A074831F09AFA94F87030201D9D
:104838006FF3410384F8703031F09AFADDE700BF76
:1048480019630508D4B10408406305085E630508C8
:104858002DE9F04385B00746884614461E4631F0D8
:1048680089FA05468EB1384631F089FA012809D00F
:10487800FFF748FB6FF08502334B1A50002005B054
:10488800BDE8F083B5FA85F56D0901342946384647
:10489800E2B231F013FC814630B9012123462B4A9C
:1048A8002B4830F0EAFFE3E744684EB120686168BE
:1048B80001AB03C3227A01AC1A7007238DF80530C7
:1048C80008F10C06304631F039FA2278824203D9D1
:1048D800304631F033FA02462146304631F00CFAC0
:1048E800D9F80C90B9F1000F09D1B8F81010FB8D68
:1048F8009942C3D93046C91A31F019FABEE7D9F836
:10490800040083681B6B13B9D9F80090EAE72946BD
:1049180098470028F8D0041F54F8043F002BF3D020
:104928001B78002BF0D0304631F008FA23681A784B
:10493800824203D9304631F001FA82B2304621680A
:1049480031F0DAF9E8E700BF0C0000008E630508D3
:10495800B4B104082DE9F04190F82830044603F07A
:104968001F03012B0F4600F128061BD0022B05D090
:1049780043BB90F8291031F00EFC03E0818DC9B2D9
:1049880001F0FCF90546E8B1304631F02AFB024651
:1049980068688368A2B99B684BB13A463146BDE85E
:1049A800F0411847818DC9B231F0DCFBEAE76FF0BE
:1049B8008503FFF7A7FA0F4A13500020BDE8F081DE
:1049C800DB68E9E7204694F8291031F01FFA02461F
:1049D8000028ECD0304631F004FB40B91369002BB5
:1049E800E5D03A463146204698470346E1E7D36882
:1049F800F5E700BF0C0000002DE9F04F95B00D461B
:104A0800097E02AF00F1280331F080080446914680
:104A1800BB600BD00121A74AA74831F0F8FA6FF024
:104A2800040840464C37BD46BDE8F08F6B7E03F066
:104A38000102B9F1000F17D019F10C0F14D0B2B957
:104A480019F1710F03D12846FFF7FCFDE9E79B4AEE
:104A58000B4699480121CDF8009030F018FF284600
:104A6800FFF7F0FDC846DCE7002A00F0B284002911
:104A780040F072842B8A072B0FD9EA681368A36267
:104A88005368E362D5F804A0E28DBAF1000F17D19C
:104A98008B4A0121884831F0BAFA0121894A8648AF
:104AA80031F0B5FA2846FFF7CDFDB86831F099FA2C
:104AB8000346A069002B00F0A384802100F0A9BC64
:104AC80004F1280031F08DFAE0B99AF8193032B1C2
:104AD80098071DD46E4688B002AA7B4B05E05E0796
:104AE80016D46E4688B002AA784BC2E9053A032369
:104AF80042F8103F70480B464FF4C251FEF7EEF9EA
:104B0800B546CAE70AB9724AC3E79AF81930DFE727
:104B18002946002031F0D8F8054628B9684A01210D
:104B2800654831F074FAC0E7FFF7ECF9002394F810
:104B38002820684E12F0600F8351C2F3411307D04A
:104B4800032B40F0E981FFF7DDF96FF085033EE0C4
:104B580004F1280031F045FA94F82930002840F093
:104B68007781013B0A2BEED801A151F823F000BF51
:104B78003B4D00084F4B0008BF4D00084F4B000845
:104B8800A54B00084F4B00084F4B00084F4B00083F
:104B9800494C00084F4B0008ED4C0008A069618D96
:104BA80003697F29D3F88030CDD8A28D002ACAD1D5
:104BB800E28D002AC7D194F82820D206C3D194F8F0
:104BC8003420022A05D1FFF79DF94FF0FF33335007
:104BD80018E01A070BD5C9B231F03BFA804648B144
:104BE800638D01213C4A344830F047FE2BE701230E
:104BF80084F83D3094F83430012B1FD1638DEBB924
:104C080084F83430FFF77EF93358002B7FF44AAF2D
:104C18000123B868236331F0E4F9002840F0898360
:104C2800E38D002B00F085832946002031F04CF8F5
:104C38000546002840F07983284A70E70123DFE71A
:104C4800204631F097F8628D0146FF2A3FF67BAF88
:104C5800E38D002B7FF477AF94F82830DB067FF4E0
:104C680072AF94F83430002BADD02AB12046D2B2BE
:104C780031F04AFA0028A6D0618D94F83C308B4276
:104C8800C0D02046C9B200F01DFF638D804630B108
:104C980001210090124A084830F0F9FDD3E61A1EA7
:104CA80014BF022301230521204684F8343031F053
:104CB8009AFBA7E7B4630508B4B10408D5630508EF
:104CC8000464050867640508266405083564050852
:104CD800466405080C0000007E6405084865050860
:104CE800A064050894F8283003F01F03012B7FF413
:104CF8002AAFE38D002B7FF426AF628DFF2A3FF6A3
:104D080022AFA18DFF293FF61EAF94F83430022B55
:104D18007FF459AF2046D2B2C9B231F0A5FA10F1EA
:104D2800020F804640F04B81FFF7ECF846F8008010
:104D380068E7E38DA18D002B7FF405AF94F834303C
:104D4800002B3FF440AF012B10D100297FF43BAF7B
:104D580012F01F020DD1638D012B7FF453AF94F82D
:104D680070306FF3C30384F870304BE712F01F0202
:104D780017D0022A7FF446AFB4F82A80B8F1000FA2
:104D88007FF440AF5FFA81FA5146204601F05CF9A2
:104D98000346FFF7B7F83350013306D14FF0FF3819
:104DA80051E600297FF40FAFD5E742465146204629
:104DB80031F01DF926E7E38DA18D002B7FF4C3AEFA
:104DC800638D5FFA81F8022B13D194F8283003F031
:104DD8001F0358EA03037FF4B6AE0122A069090A4B
:104DE80031F017F900287FF4AEAE012384F83D3086
:104DF80008E794F8340000283FF4E5AE01280DD107
:104E080000297FF4E0AE12F01F020AD1012B7FF4D3
:104E1800F9AE94F8703043F00803A4E712F01F02CB
:104E280012D0022A7FF4EEAE002B7FF4EBAE41469F
:104E3800204601F0E7F80346FFF764F833500133E2
:104E4800ACD001224146B2E700297FF4BCAEDDE7D1
:104E58000A2B3FF678AE01A151F823F0914E0008D5
:104E68004F4B00084F4B00084F4B00084F4B0008B2
:104E78004F4B0008114F00084F4B0008CB52000859
:104E88004F4B0008F9520008E38DA18D022B7FF4E7
:104E98005AAE94F83430002B3FF495AE012B10D164
:104EA80000297FF490AE12F01F020DD194F87030F3
:104EB8004FEA930808F00208C3F3001348EA03080E
:104EC80006E012F01F0210D0022A12D04FF000089C
:104ED80005F10C0A504630F031FFE38D98420ED2AE
:104EE800FFF710F86FF00B0371E600297FF46BAE43
:104EF800DCE72046C9B231F055FA8046E8E741467A
:104F0800504630F00AFF7DE694F82810628DC806F6
:104F18004FEA1223D2B204D029462046FFF71AFDE1
:104F28004CE0013B0E2B3FF60EAE01A151F823F0E9
:104F3800754F0008BB4F0008D54F00084F4B0008BD
:104F48004F4B00082F510008D14F00084F4B000865
:104F58004F4B00084F4B00084F4B00084F4B0008C1
:104F68004F4B00084F4B0008C751000805F10C08CB
:104F78004046B4F82EA030F0E1FE82450AD2B4F8DB
:104F88002EA0204630F0F6FE48B101287FF4DBADB4
:104F9800A16F05E0404630F0D1FE8246F1E7616F2F
:104FA800002900F0DC800A78524528BF5246404666
:104FB80030E0002329462046FFF74AFC8046B8F136
:104FC800000F7FF440AD1DE60123F3E703212046DF
:104FD80030F05BFF824600283FF4B5AD30F0FCFFAF
:104FE800E38DF0B9BAF8142098463A85DAF810201B
:104FF80005F10C0A128850467A8530F09FFE8045EC
:105008000BD2E08D97F8282007F12801824228BFAB
:105018000246504630F070FEF4E5504630F08EFE01
:10502800F0E79B4600233B759AF81530DAF808201C
:105038007B75C34B1340C34A934263D1102107F1D8
:10504800180004F0F9F8002842DB07F128031028BB
:105058009E4628BF1020DFF8F0C207F118028045ED
:1050680003F102033DD3800002303875C7F80CE025
:1050780005F10C0A504630F061FE97F81480D845C7
:1050880028BFD846404503D2504630F057FE8046E8
:10509800B8F1020FC34628BF4FF0020B50465A46DC
:1050A80007F1140130F028FEA8EB0B08D7F80CB074
:1050B8004FEA58030BEB58025A452AD118F0010F52
:1050C8003FF4A0AD5046FA68D15C30F01EFE99E579
:1050D80058307FF438AD01219C4A9D4830F097FF45
:1050E80031E512F8011B08F101084FEA111A01F025
:1050F8000F011CF80AA01CF8011003F802AC03F811
:10510800011CACE79AF814303B75DAF81030FB60F4
:10511800AEE750461BF8011BC7E9002330F0FDFD40
:10512800D7E90023C8E7204630F024FED4E91D83E0
:10513800002808BF98460023C7F82A30C7F82E3041
:105148000A2387F828300623204687F8293030F0CC
:1051580016FE01287FF4F7ACB8F1000F02D16FF00A
:10516800150870E4B8F802307B8598F8043087F8A1
:105178002C3098F8053087F82D3098F8063087F8E5
:105188002E3098F8073087F82F3098F8113005F14D
:105198000C0887F830304046B4F82EA030F0CEFD29
:1051A800824508D2E08D97F8282007F1280182422D
:1051B80028BF0246FBE6404630F0C0FDF3E7204634
:1051C80030F0D8FD20B101287FF4BDACA36F00E01A
:1051D800636F002BC3D05B88B3F5007F7FF6B3AC59
:1051E8005C4B04F15002BB62002387F82C3004F1B9
:1051F8005003FB60236D9A4260D105F10C0A5046BA
:1052080030F09CFDB7F82A80E38D984528BF984672
:10521800404503D2504630F091FD804697F828204B
:105228005046424528BF424607F1280130F064FD48
:10523800B8F1050F94BFA8EB0808A8F10508B8F164
:10524800000F3FF4DFACD4F850B0FB689B453FF447
:10525800D9ACBBF1000F3FF4D5AC9BF815300F2B40
:1052680015D19BF814205046424528BF4246DBF82A
:10527800101030F041FD9BF81430434594BFA8EB63
:105288000308A8EB0808B8F1000F3FF4BBAC636D46
:105298005B453FF4B7ACDBF800B0DAE75A7D0F2A7C
:1052A80008D11A7D798D0A447A8597F82C20013225
:1052B80087F82C20626D9A429FD01B68002BEDD195
:1052C8009BE794F8343094F83CA0002B3FF47BAC77
:1052D800E38D012B7FF437AC05F10C08404630F024
:1052E8002DFDE38D9842FFF4FBAD51464046ECE6B8
:1052F80094F8283003F01F03012B7FF464AC204698
:1053080030F0F0FE00283FF45EACA38D4268FF2B1E
:105318003FF619AC12799A42FFF415AC0F2B3FF601
:1053280012AC234493F83EA0D2E76B7E59077FF571
:105338007BAC2946204600F01DFE8046FFF771BB76
:1053480000FF02000003020065650508C364050844
:10535800B4B10408050F05005A077FF5A6AB8029EC
:105368007FF4A3AB2846FFF76DF9256B012D40D1DB
:1053780094F83D30002B3FF454AB94F82930052BBA
:105388000CD1618DA069C9B230F063FE804628B1A6
:10539800638D234A2946234830F06FFA94F8293060
:1053A800032B11D1638D022B0ED1A18D00220D0A82
:1053B8002946A06930F02DFE804628B101212B46F0
:1053C800194A184830F059FA002384F83D30FFF79D
:1053D80028BB5B077FF569AB0029C0D1236B012B84
:1053E8003FF431AB0221114A0E4830F010FEFFF7AE
:1053F8002ABB02210E4A0B4830F009FEFFF711BB09
:10540800E38D002B3FF459AB19F10C0118BF0121B2
:10541800C90131F0F8FD002380462363FFF701BB83
:105428007E640508B4B1040806650508E564050846
:10543800246505080B7810B4062B14D10369D3F83A
:105448009C20EFF31184102383F31288BFF36F8F2E
:1054580000204B681860506A58B9C2E9083384F3D1
:105468001188BFF36F8F00220023034810BC33F06C
:1054780098BF03605362F2E70410002030B589B08A
:10548800002200230024CDE906236FF007034FF420
:105498008062CDE90334CDE90144154B15490094E8
:1054A800154808F019F81549134834F00FF9144B4A
:1054B80014498B4207D30020134B14498B420CD359
:1054C800002009B030BD03F11402D2E8EF0FC2E8A2
:1054D800E54F002DF9D11833EBE703F11402D2E8B8
:1054E800EF4FC2E8E50F002DF9D11833E6E700BF0A
:1054F8006D550008C04A002060260020B6800508C7
:1055080088110020D0110020D0110020181200208E
:1055180038B50D4630F0E6FD30B90121BDE8384018
:105528000E4A0F4830F0A0B9C46804B938BD2B78CA
:10553800032B07D0052B0CD0022B08D16068836899
:105548009B6902E0606883685B6903B198472468D7
:10555800EBE760688368DB69F7E700BF7F650508EC
:10556800C4B104082DE9F047102684B0DFF8FC81A7
:1055780000AF4FF0FF334FF0FF324046391D07F0C0
:10558800AFFBFB681B69D3F89C40236A73B1EFF348
:10559800118386F31288BFF36F8FD4F820A0BAF175
:1055A800000F1BD183F31188BFF36F8F3B79062B54
:1055B800DFD0072BDDD801A252F823F05B56000894
:1055C8004F5600088356000861560008B95600086F
:1055D800A55600087B55000863570008616ADAF889
:1055E80000208A45226208BF626283F31188BFF3F4
:1055F8006F8F9AF8183051465D062046DAF81E205B
:105608001ED1FFF7F9F905460028BED0E9468AB051
:105618006A469AF81830C2E9073A05235449C2E99C
:10562800051042F8103F00234FF421515148FDF76F
:1056380055FC2A46CD460721204630F0D4FEA4E783
:1056480030F0A0FDDFE700220121204630F0CBFE3C
:105658008FE700221146F8E794F8703043F004030E
:1056680084F8703094F83430022B03D12046391D69
:10567800FFF74EFF00220321E7E794F870306FF33D
:10568800820384F8703094F83430022B03D120461A
:10569800391DFFF73DFF00220221D6E794F8343088
:1056A800022B7FF466AF2046391DFFF731FF60E714
:1056B80094F87030D4F818906FF3820384F870303F
:1056C800D9F808A0D9F81030A033D3E8AF3F9A072B
:1056D8001BD54846DAF83C309847DAF824300021E0
:1056E800484698470546DAF84030484698477DB11D
:1056F800214A01211F4830F0B7F800220421204632
:1057080030F071FE2A4607219FE74FF0FF35EFE79B
:105718002946204600F0D6F9054608B1174AE8E7B9
:105728008021204630F03BFE20B10121144A114867
:1057380030F09AF8A06931F01BFD0022831E584210
:10574800584194F87030042123F0680343EA401369
:1057580084F8342084F8703077E70121094A054835
:1057680030F082F80621BA686FE700BF0410002005
:10577800AE650508C4B10408D865050806660508BD
:10578800326605084F66050838B5024605460C49D5
:10579800806931F04CFD044630B10121094A0A48BC
:1057A80030F062F8204638BD85F83C00284600F005
:1057B80047F904460028F5D0A86931F067FDF1E7FC
:1057C8003D5400085F660508C4B104082DE9F84394
:1057D8004FF0010805460C4646462068002840D090
:1057E80068F07F02D2B211465FFA88F730F050FCB9
:1057F800E0B1D5F800901146484630F049FC48B968
:10580800134619480121194A30F037F86FF015008E
:10581800BDE8F88322F08002103206FA02F229EA83
:1058280002032B60236823EA0203236039462068B9
:1058380030F02EFC80B12A683946104630F028FC3A
:1058480008B94346DDE706FA08F122EA01022A60B0
:10585800236823EA0103236008F10108B8F1100F57
:10586800BBD10020D4E700BFECB104088666050868
:105878002DE9F04F00268FB05368CDE90621D46892
:10588800099002930C96039674B9039B029A093304
:105898009BB293701B0AD370069B1671DC68002CB0
:1058A80040F0BC80A146A3E0002560680D958368A0
:1058B8001B6B002B00F0A38007999847002800F085
:1058C8009E80C4E903553546071F57F8043F0BB1BE
:1058D8001A789AB9B54240F28F80E3680D9A13435B
:1058E800E360606883689B6A002B00F08A809847B1
:1058F8008146002800F088804E4A75E05A780B2AC5
:1059080008BF9D703B685A78042A10D1E2680D9947
:105918000A43E260DA78002A59D101229D7023698E
:10592800AA40134301352361EDB200230D93D7F844
:10593800008098F80130052BC7D16FF012094FF09D
:10594800010B099B9B69089398F8051098F80420A7
:105958000C9B42EA0122ADF82E2098F902205FFA4A
:105968008BFA002AB8BF4AF0800A514618460493B9
:1059780030F08EFB90BB0D9B51461846059330F0D6
:1059880087FB58BB98F8063098F8032051460093D7
:1059980008980DF12E0331F0ADFA8146F0B90123D4
:1059A8001AF0800F1EBF2AF0800110318B40049836
:1059B800059908BF03FA0AF3BDF82E2019431843C6
:1059C800CDE90C0188F802A0A8F804207DE76A1E3A
:1059D8009A700DA90CA8FFF7F9FEA6E70BF1010BC9
:1059E800BBF1100FB0D1144A012114482FF03CFF2D
:1059F80048460FB0BDE8F08F6FF01509F3E735465C
:105A08006FE76FF0850977E76068079930F08AFBE0
:105A1800039B2E4603442468039335E7E36804F1A7
:105A28000C01A3600CA8FFF7D1FE81460028DFD146
:105A3800246834E7C7660508A3660508ECB10408BE
:105A480070B5836905461B69426F93F88030C3F3CC
:105A58004113022B0CD0032B0CD0012B0CBF1023AD
:105A68000823D3712E6E3EB9AE6DBEB9344611E02F
:105A78002023F6E74023F4E7324601212846FFF7C2
:105A8800F7FE044640B173685B790B4A01210B4865
:105A98002FF0F3FE204670BD3668E4E73246002159
:105AA8002846FFF7E5FE044618B173685B79044A97
:105AB800ECE73668D9E700BFEB660508ECB10408E7
:105AC8000E6705082DE9F04105460E4630F052F9FB
:105AD80095F83C30804633B3284630F003FB074640
:105AE800F0B10146284630F06DFB10220446002133
:105AF80005F13E0044F030FF002385F83C30FF6894
:105B08003FB984B119491A4830F0CBFA2046BDE8AC
:105B1800F081786883685B6A03B198473F68EFE76C
:105B28006FF03C04EEE71EB985F83C600024EDE711
:105B380032464146284630F0C1FA074690B102463F
:105B4800284630F069FB04460028DFD185F83C6020
:105B5800FC68002CEAD0606883681B6A03B1984728
:105B68002468F6E76FF03C04D0E700BF40630508FF
:105B7800ACB104082DE9F04105468846144657683B
:105B880030F093FA95F87030D8070BD54F49504844
:105B980030F087FA6FF00F08281D30F08DFA404674
:105BA800BDE8F081B8F1010F15D1284630F0E7F8CB
:105BB80030B94849464830F074FA6FF08508EBE789
:105BC800FB7999061AD5AB691B69D3F880309A0717
:105BD8000CD44149EEE7FB799B06F4D4B8F1000FE9
:105BE8000AD12B6E43BB05F158060BE0B8F1000F44
:105BF800F7D0B8F1010F01D03849DBE7AB6D83B9B5
:105C080005F1600600223368E3B96268B8F1000F55
:105C18003FD16B6F5B7C0133DBB253716A6F537496
:105C280022E0A34206D12E49294830F03AFA6FF013
:105C38001508B1E71B68E2E7A34201D12949F3E758
:105C48001B68CFE79C4221D12368CAB972683360C8
:105C5800944200D173600023236063685B7902215A
:105C6800214A1B482FF009FEA16819B3284630F0D5
:105C780026F98046D0B11D49154830F012FA8BE755
:105C8800136073689C4208BF7260E4E71A461B6899
:105C9800BAE7B8F1010F02D001235371E4E7AB6F03
:105CA8005B7C0133DBB25371AA6FB8E7A06830F0B0
:105CB80093F9B87100232360736823B9C6E90044D7
:105CC8004FF0000868E71C607460F9E75F67050833
:105CD800ACB10408816705083B6705089F6705089C
:105CE800BF670508DC670508F96705081668050831
:105CF800F8B5054600AF21B301290BD1184C194E50
:105D08002AE0636828461968FBF712FBB0B118341B
:105D1800B442F6D36C4688B06A46134BC2E90535DF
:105D28004FF400739383114B42F8103F00234FF454
:105D3800E2510F48FDF7D2F8A54600242046BD469B
:105D4800F8BD0C4C0C4EE3E7636828461968FBF76E
:105D5800EFFA0028F2D01834B442F5D3DAE700BFDE
:105D6800D0110020181200204D680508030000011A
:105D7800BCB1040888110020D011002070B501259D
:105D880001F07F0311F0800F18BF10339D4090F889
:105D980034300446022B06D001210C4A0C482FF05F
:105DA80063FD002070BD90F83C602FF0E3FF3246A1
:105DB8000146204630F082F90028F2D0C068002859
:105DC800EFD083681D42EDD10068F8E76B680508DD
:105DD800BCB104082DE9F8430546084611461646A5
:105DE8009846FFF785FF0446002843D0284630F040
:105DF80092F995F87030DA0702D5204A012109E0B6
:105E0800D4F8049004F11407D7E8AF3FDB070CD5AA
:105E180002211B4A1B482FF027FD6FF00F04281D95
:105E280007F036F82046BDE8F883D9F804301BB1EE
:105E3800AB4201D0144AE1E742463146284630F0E9
:105E48003DF9A0B10023236003696BB9C0E903449D
:105E5800D7E8EF3F43F00103C7E8E23F002AF7D154
:105E68000024C9F80450DAE71C600461F0E76FF019
:105E78003C04D4E76FF01204D4E700BF5F6705085D
:105E880090680508BCB10408B26805082DE9F04F10
:105E980083B000AF7B6097F830304C680E463B60AB
:105EA800814690462FF066FFA36801461B6B33B905
:105EB8006FF0150420460C37BD46BDE8F08F20462C
:105EC80098470028F4D00024051F06F10C0A55F85D
:105ED800041F09B10B782BB9002C0CBF6FF03C04E0
:105EE8000024E7E74B78042B0ED1002C3CD18B78AB
:105EF8007A689342EBD1CB783A689342E7D10B7931
:105F0800002BD7D00124E2E7052BE0D1002CDED00E
:105F1800B8F1010F91F802B009D0B8F1020FF1D130
:105F280052465946D9F8180030F004FA04E05246AF
:105F3800D9F8180030F0E2F904460028E2D06D469E
:105F48008AB06A46F368C2E907B306230749506274
:105F5800C2E9051842F8103F00234FF441510448A4
:105F6800FCF7BCFFAD46A5E70024A3E7F2680508E7
:105F7800E4B104082DE9F0410B7E05465E060C46A7
:105F880038D119062DD52FF035FF40B11B48012116
:105F98001B4A2FF069FC4FF0FF30BDE8F08128461E
:105FA800D5F87480268AEF8D2FF0E4FEF8B1421EF2
:105FB800534253419B01228A9AB1BE42324628BFBE
:105FC8003A46E98D91420CD9B2FBF3F103FB112259
:105FD8003AB994F91830002BBEBF637E43F008032A
:105FE80063762146A869BDE8F04131F068B898F8B1
:105FF8000730E0E76FF01500CFE700BFDCB1040819
:106008002E69050870B5064680690C4630F0FBFF1E
:10601800054638B102212346094A0A482FF02DFCCB
:10602800284670BD012214F0800F18BF24F08004A8
:10603800B36B18BF1034A2401A43B263F0E700BF35
:1060480042690508DCB1040870B5054680690E464A
:1060580031F004F8044638B102213346054A0648AF
:106068002FF00BFC204670BD314605F1380030F0AA
:1060780037F9F7E759690508DCB1040870B5064631
:10608800EFF31181102282F31288BFF36F8F1D4C3A
:10609800236881F31188BFF36F8F5B6893F87030C2
:1060A800DB0705D4BDE870400A22002307F0B8B921
:1060B800EFF3118382F31288BFF36F8F256865B9F8
:1060C80083F31188BFF36F8F2368D3B13046BDE8DF
:1060D80070400022002307F06FB961682A688D427A
:1060E80008BF6260226083F31188BFF36F8F68680E
:1060F80005F10801C36998472946034833F0EEF8CB
:10610800E2E770BD60330020900F002030B585B005
:106118006C46054684E8060000230022144803A9BB
:1061280006F040FD0246E8B994E80300039B5D6071
:10613800083383E80300EFF31180102383F31288F8
:10614800BFF36F8F039B1A600A4A516861B9C2E9AD
:10615800003380F31188BFF36F8F002200230648B5
:1061680007F02AF905B030BD0B605360F1E700BFB6
:10617800900F0020603300200000002038B54B78D5
:106188000469202B4568206908D0222B19D0FDF717
:10619800B9FE6FF08502104B1A5010E0CB88072B20
:1061A800F5D1D3681A6842609A8802819B79837214
:1061B80030F03EF922460821284630F022F9002026
:1061C80038BD4B880921C3F34002838103F00103E2
:1061D800027643762246EFE70C00000008B5134626
:1061E800026910694A78212A12D133B9FDF78AFE6B
:1061F8006FF00B02094B1A5008E0CA88011D072AE4
:1062080028BF072203F10C002FF076FD002008BDFF
:10621800FDF778FE6FF08502004BECE70C000000FC
:1062280038B5002405690E49EB6B05F14800C3E950
:106238000144DC606B6BC3E90144DC6033F034FA81
:1062480005F17800074933F003FA074905F12400FE
:1062580033F0FEF9284630F0EBF8204638BD00BF91
:106268007D63000821650008ED6500082DE9F3410C
:10627800036906460D46D0F804801C690F7E002A83
:1062880032D00B8A713238480BBF02210121374ABC
:10629800374A00933B462FF0FAFA30462F7E30F00B
:1062A8003BF9874204D1042104F1880030F0B5F9A4
:1062B80030462F7E30F03EF9874204D1052104F1A3
:1062C800880030F0AAF930462F7E30F017F987425F
:1062D80003D104F18C0006F0BDFE2946404602B009
:1062E800BDE8F04130F058B830F016F9874214D1C3
:1062F8002A8AE968606B2FF0C3F928B1E3691BB1FA
:1063080004F1240006F0E8FF04F18800042130F0CD
:1063180084F904F1780006F0DFFF30462F7E30F074
:1063280009F9874215D1E3691BB104F1240006F08D
:10633800D3FF052104F1880030F06FF9E36B5A8927
:10634800DB889A4205D00022002304F1480007F0B8
:1063580033F830462F7E30F0D1F88742BDD104F1B2
:106368008C0006F017FEB8E7A4B104088369050895
:10637800A76905082DE9F04750F8483C00F14006A8
:106388005B68074600213046D3F8008030F0B0F84B
:10639800002854D00121304630F0AAF800284ED108
:1063A800D6E8EF3F43F02002C6E8E12F0029F7D1F5
:1063B8009B0644D4404630F0BDF800220446002332
:1063C80020482FF04EFC054650B93046052130F0E4
:1063D80024F93846BDE8F0470A22002306F0ECBF4E
:1063E8008146047659F80C1F428A57F80C0C2FF096
:1063F80067F90446014648462FF078FC54B1D8F8AE
:10640800040030F001F9B4FBF0F303FB1044B4FAD4
:1064180084F464092946404607F82D4C2FF0A4FF60
:1064280068B10121084A09482FF01EFA2846FEF7EC
:1064380009F93046BDE8F047052130F0EEB8BDE86F
:10644800F08700BF88100020C8690508A4B10408B7
:1064580038B503461B6940685D68AC68A37A84F860
:10646800223094F82D3084F82330696849B1237CB0
:106478003BB92FF024FD30B10121054A05482FF022
:10648800F3F9002038BD68682FF0A6FD2074F8E7FE
:10649800DA690508A4B1040873B5102504698DF8F4
:1064A8000710EFF3118685F31288BFF36F8F01226F
:1064B800E06B0DF107012FF0E3F886F31188BFF3C5
:1064C8006F8F012814D033F0FBF808B9A37EBBB94D
:1064D80001220E4BD3E8EF1F002903D1C3E8E02FB8
:1064E8000028F7D104D10221094A0A482FF0BCF943
:1064F8000A22002304F1480006F05EFF02B070BDD6
:1065080000210A2033F096F9CBE700BF683300205A
:10651800046A0508A4B1040870B550F8782C00F195
:106528001004526803460021204615682FF0E0FF4A
:1065380000284DD0012120462FF0DAFF002847D14E
:1065480053F8442C68689388918916695B1A9BB242
:10655800F61A30F059F8B0423AD8D4E8EF3F43F091
:106568001002C4E8E12F0029F7D1DB0606D5BDE803
:1065780070400221174A18482FF076B928462FF0A4
:10658800CBFF00220646002314482FF06AFB04467E
:10659800F0B10676686830F037F8638A984203D21B
:1065A800686830F031F883B22146284663822FF0BC
:1065B800DBFE68B128462FF0AFFF034606480121ED
:1065C800074A2FF05AF92046BDE87040FEF73AB85E
:1065D80070BD00BF236A0508A4B104088810002014
:1065E800436A050838B550F8243C04465B681A68C5
:1065F80050F8083C33B9BDE838400121284A2948F9
:106608002FF032B9002300F16405838283830221CD
:1066180028462FF06DFFB8B154E902311069984748
:10662800637D1BB104F1540006F056FE052128468F
:106638002FF05EFF98B9637F6BB10022002304F14D
:10664800240006F0B9FE0AE0032128462FF050FF87
:106658000028E1D1E4E714F8093C002BEDD1022130
:1066680028462FF045FF38B123695A89DB889A42BA
:1066780002D0204606F030FE032128462FF038FFCE
:1066880060B1A2699388918912695B1A9BB29A4298
:1066980004D02046BDE8384006F01EBE38BD00BF15
:1066A800686A0508A4B10408D3B500260027044683
:1066B800CDE9006705482FF0D8FA28B1230658BF5E
:1066C8000023047658BF038202B0D0BDB410002066
:1066D8002DE9F04383B000234FF0010805691C4CF5
:1066E8001C4E02AF28602B7785F8203005F124096D
:1066F800B442234601D3002019E095F82020103435
:10670800CAB16C4688B01B6802AA1349C2E90513CE
:106718004FF400739383114B42F8103F1048002345
:106728004FF4E251FCF7DAFB6FF00B00A546043793
:10673800BD46BDE8F08385F8208054F8043C4846FF
:10674800009354F8101C54E9032330F004FACFE7FF
:106758003CEC05084CEC0508F36A05080300000149
:10676800F4B104081FB500230190CDE902334FF0BE
:10677800FF324FF0FF3301A9024832F012FE05B094
:106788005DF804FBD40F002008B54B78FF2B07D128
:106798004B882BB9CB881BB9FFF7E4FF002008BD55
:1067A800FDF7B0FB6FF08502014B1A50F6E700BF0A
:1067B8000C00000013B514464A780369FE2A14D168
:1067C8004A8892B9CA8882B193F820300BB1013B4C
:1067D800DBB201220DF1070104F10C008DF807303E
:1067E8002FF08AFA002002B010BDFDF78BFB6FF086
:1067F8008502014B1A50F5E70C0000001FB5CDE9E2
:10680800010103924FF0FF324FF0FF3301A9034813
:1068180032F0C7FD002005B05DF804FBD40F00205E
:106828002DE9F041044617460E46006830F01EF880
:1068380031463A468046FFF737FFD4F87B300546A5
:10684800DB1B0146C4F87B3020682FF08DFD88B132
:106858000B4A434601210B482FF00FF831462046DA
:1068680030F0AAF82846FDF7EDFE2046BDE8F041D5
:1068780030F06EB8A37F0133A377BDE8F08100BF85
:10688800436A0508F4B104082DE9F74F0446006887
:1068980030F001F8302706464FF02408E37F012B3B
:1068A8001FD82368D3F810A0D3F804909AF8611081
:1068B80017FB01810AEB010B584630F072F9594673
:1068C8000246019048462FF0FCFF9AF81F30054613
:1068D80033B1019A5946121A48462FF0F2FF05467D
:1068E80015B903B0BDE8F08F20462FF0A7FF2A4660
:1068F800014681463046FFF7D7FE05460146206827
:106908002FF032FD88B10B4A334601210A482EF098
:10691800B4FF2846FDF796FE4946204630F04CF86D
:1069280003B0BDE8F04F30F013B8E37F0133E377ED
:10693800B4E700BF436A0508F4B104082DE9F04F35
:10694800DFF8EC9289B04FF0FF324FF0FF33B948CF
:1069580005A906F0C5F9059E069D3469002D40F08D
:106968009080257704F1240694F820309D42C0F2E7
:10697800828004F11803D3E8EF2F22F00202C3E863
:10698800E12F0029F7D1D3E8EF1F21F00401C3E874
:10699800E21F002AF7D104F11803D3E8AF3FDB0761
:1069A800D1D5237F022B00F09581032B00F08E8137
:1069B80053BBDDF814A0DAF81050EB7F23BB504628
:1069C8002FF069FF804628462FF038FF4FF40072F9
:1069D800014606464046FFF767FE07460146504611
:1069E8002FF0C2FC002800F06D8101214346924A35
:1069F80092482EF042FF3846FDF724FE31462846DD
:106A08002FF0DAFF2FF0A4FFA37F002B9BD1237F69
:106A1800012B40F08481302304F1630694F861501F
:106A2800304694F8621003FB054500F06BFA2435F4
:106A3800024631462369284600F082FA0646C4F821
:106A48008400284630F0A3F88046284630F0A4F8A1
:106A58000746284630F0A5F8E26D3044002A40F099
:106A68004281002840F03A81284630F0C1F80038C9
:106A780018BF012033E1304630F080F80135303658
:106A880072E7079FD6F804A095F8188047B32B8AB9
:106A980071376A48009308BF0221434616BF012197
:106AA800674A684A2EF0F3FE30462F7E2FF0F3FE39
:106AB800874240F0F680E37F5A1EE2776A680AB19F
:106AC800023BE377204669692FF076FF6B6813B1C4
:106AD80059692FF071FF294650462FF05DFC5AE79F
:106AE80030462FF0D8FE804540F09480237FD5F8BB
:106AF8000C80B5F810B0002B49D1BBF11F0F42D163
:106B0800D8F800304B453ED1414604F1540308F112
:106B18001C0251F8040B914243F8040BF9D10A887E
:106B28001A808A7842219A70552384F87330532347
:106B380084F8743084F87630A36DE26DC4F8773049
:106B48000023C4F8803094F86030C4F87B209A069B
:106B580084F875100FD194F8612094F820309A4287
:106B680009D294F86230013B0F2B04D8012384F832
:106B78007F30237798E720682FF083FE022384F87C
:106B88007F300423F5E720462FF0E2FE8CE7032B45
:106B98008AD1302394F8617003FB0747D4F880301A
:106BA80024375B44C4F88030BBF1000F16D0384658
:106BB8002FF0F7FF90B141465A46384630F004F8B6
:106BC800804628B902215B461F4A1C482EF055FE14
:106BD800D4F87B30A3EB0803C4F87B30D4F88020CA
:106BE800E36D9A420DD238462FF0DBFF00287FF480
:106BF8005BAFD4F88020E36D9A4202D220682FF070
:106C080056FE38462FF0F4FF003818BF012084F8EC
:106C18007F00B6E7304695F818802FF027FE8045AC
:106C28007FF442AF237F2A8A052B0FD127773BE7D2
:106C380055534243D40F0020436A0508F4B10408B1
:106C480083690508A76905080A6B0508022B7FF404
:106C58002BAF4FF03008D4F8803094F861701344AB
:106C6800C4F8803023681969D3F804B091F861300A
:106C780008FB03112431084603912FF092FF039972
:106C8800024658462FF01DFE00287FF40DAFD4F8B9
:106C98007B3013B120682FF0F4FD08FB0740243047
:106CA800B0E730462F7E2FF0E1FD87427FF40AAF30
:106CB800A37F5A1EA2776A68002A3FF403AF023BFB
:106CC800A377FFE6EB7F0133EB779DE62046FFF7DE
:106CD800DBFD99E620462FF07FFE95E6022084F83A
:106CE8007F0004231AE094F9601040B90029206855
:106CF80002DA2FF0C6FDB7E62FF0D9FDB4E6002979
:106D080014DA904202D8B8F1000F06D120682FF0AB
:106D1800B8FD022384F87F30E3E702232377237F3B
:106D2800022B0CD120462FF057FE0CE6904200D8DB
:106D38001FB920682FF0BBFDEBE70323EEE7032B19
:106D480003D12046FFF7A0FDFDE5042B7FF4FBAD42
:106D5800A37F2BB101211D4A1D482EF085FDF2E5C8
:106D680020682FF083FD074620462FF067FD054673
:106D7800024604F1730304F17F0153F8040B8B42BC
:106D880042F8040BF9D11B782946137038460D22B6
:106D9800FFF78AFC0646014620682FF0E5FA78B12D
:106DA8000C4A3B4601210A482EF067FD3046FDF7A4
:106DB80049FC294620462FF0FFFD2FF0C9FDC2E50A
:106DC800A37F0133A37705232377BCE5306B050840
:106DD800F4B10408436A0508802938B50D461446FD
:106DE80021D083290DD019BB80235371832303201D
:106DF800117193710023E07023706570A3700430E3
:106E080038BD0223137101235371002393710A23A0
:106E1800D37108224168A01843F0D5FD064B0E2017
:106E28001B882382E6E7044B02201B889380E1E756
:106E38006FF08500E4E700BF98D005082DE9F04120
:106E48008769D0F82480BA4228BF3A46B2FBF8F5E1
:106E58000446C2692B4600682EF084FE064648B9EF
:106E6800B7FBF8F7AF4207D0E3692B44E361606AE8
:106E7800684312E000250126002205212068FCF75E
:106E88007FFB60B10121094A09482EF0EDFCE36956
:106E98002B44E3610020074BA362BDE8F081E3695E
:106EA8002B44E361002EF5D1E1E700BF516B0508E3
:106EB800F4B104080203000C81420B4607B509D35C
:106EC80002210D4A0D482EF0D8FC6FF0150003B0D2
:106ED8005DF804FB6AB101391144814201D28B4249
:106EE80007D90221009305481346054A2EF0CFFC26
:106EF800EBE70020EBE700BF686B0508F4B1040876
:106F08007F6B05080C290346084616D11B78252BEC
:106F180012D009D8122B10D8084A42FA03F313F0FA
:106F2800010F08BF0620704703F0FD02282A03D08E
:106F38005A2B08BF0A2070470A207047F6FFFBFF4C
:106F48002DE9F0411E4690F82C30062A23F00C0358
:106F580080F82C304FF00003C0E904338361044605
:106F680088460B7886B040F00C81D3B94D7915F07E
:106F7800040540F0168290F82C309B070AD40223AF
:106F88004FF468521D4684F8295084F828300025AB
:106F980062853AE02FF061FD0028F0D12B462A46A1
:106FA800F1E7032B35D14F7917F0040740F0F98149
:106FB80090F82C308DF8077043F0040380F82C30DB
:106FC8007023ADF8043090F829300D7903F00F03E1
:106FD8008DF806300A23122D28BF12258DF80B30A4
:106FE800438D2A465BBA304601A98DF808708DF8A2
:106FF80009708DF80A700397ADF81030ADF812706B
:10700800ADF8147043F081FCA762284606B0BDE8CD
:10701800F081122B4BD14B795F0700F1C28190F8B8
:107028002C3043F0040380F82C304B7813F002071F
:1070380023D113F0010F8B7819D0B1F803503246E1
:107048001946FFF7C9FE6DBAADB2854206DAB8F83F
:10705800030040BA80B200231A4613E032462046A5
:1070680098F80210FFF7B8FE0028F4DA05E083B1BB
:107078000221AB4AAB482EF000FC022305274FF44F
:1070880010520020054684F8283084F8297062855B
:10709800BBE7B1F8035031462FF015FD6DBAADB21C
:1070A8008542D4DB314620462FF00DFDDCE71A2B54
:1070B80027D14D7915F0040540F0738190F82C30F4
:1070C80043F0040380F82C308B783F2B14D1CF7811
:1070D80097B90D790323042D28BF042530462A4685
:1070E80001A9019343F011FC3A463B4684F8282055
:1070F80084F82970638588E7022205274FF4105326
:10710800F4E71B2B23D14D7915F0040540F0498194
:10711800097990F82C200809C2F340030AD18E0798
:1071280008D5C80711D402F00302032A00F03E81F3
:10713800002301E0002BF6D094F82C2063F34102E1
:1071480084F82C2000231A461DE70123F4E71E2BA0
:1071580040F022814D7915F0040540F022810B7929
:1071680013F0030306D0012BECD190F82C3043F038
:10717800010303E090F82C3065F3000384F82C3009
:10718800E0E70A2A40F00881232B40D14B7A13F01C
:10719800040340F00681ADF804308DF8063008236A
:1071A80090F82C208DF8073042F0040280F82C204B
:1071B8002FF053FC0028B5BF4FF0FF330222032203
:1071C800236A8DF80C20A8BF1BBA0293636A304665
:1071D8001BBAC3F307228DF80D30C3F307438DF8AC
:1071E8000F3094F82C308DF80E2043F0040384F807
:1071F8002C30B8F8075001A96DBAADB20C2D28BFD4
:107208000C252A4643F081FB0023A362FDE6252BCB
:107218002ED14F7A17F0040740F0C38090F82C3035
:1072280043F00403990780F82C3006D402274FF462
:107238006853002584F828705AE72FF00EFC0028C0
:10724800F4D1236A93B1013B1ABA22F07F421B069C
:1072580094F82C00616A1A4309BA40F0040084F8D3
:107268002C000023082532607160E3E71A46EFE737
:10727800282B2BD14D7A15F0040540F0928090F818
:107288002C30D1F8027043F004039A07B1F8076074
:1072980080F82C307FF573AE2FF0DFFB00287FF4E9
:1072A8006EAE76BA3FBAB6B232463946206AFFF7B2
:1072B80003FE20B1022305254FF4045263E61A4B5E
:1072C800E7612361636A7343A36167E62A2B2FD1C1
:1072D8004D7A15F0040564D190F82C30D1F802707D
:1072E80043F00803B1F8076080F82C309B077FF55E
:1072F80046AE2FF0B2FB00287FF441AE76BA3FBA13
:10730800B6B232463946206AFFF7D6FD0028D1D1F9
:10731800064BE7616361636A7343A36112E700BFC9
:10732800A96B0508F4B10408316B0308456E000821
:107338005A2B31D14D7A15F0040532D190F82C3002
:1073480043F0040380F82C308B783F2B19D1CF7889
:10735800E7B94FF4C063CDE90135B1F807503046BD
:107368006DBAADB2082D28BF082501A92A4643F0F9
:10737800CCFA00231A4684F8283084F829706285EC
:1073880043E6022305274FF41052F4E702230527AA
:107398004FF410520025EEE70121074A07482EF066
:1073A8006CFA022305254FF41052ECE5022305255B
:1073B80045F20232E7E500BFC66B0508F4B10408E0
:1073C80007B56B46084A92E8030083E803000748BC
:1073D8008268126822B11946904703B05DF804FB31
:1073E8006FF05700F9E700BF14B20408C8AC0408EE
:1073F8001F2808B5034606D909480121094A2EF075
:107408003CFA002008BD0120074A00FA03F3D168BE
:1074180033EA0101F6D01269934318BF0020F1E75F
:10742800E4B00408E16B050800200246012100F0E1
:107438001F021F2808B501FA02F2034606D90648BA
:10744800064A2EF01AFA6FF0150008BD044B00200A
:10745800DA601A61F9E700BFE4B00408E16B0508D7
:10746800002002462DE9F041054600264FF00108AC
:107478000E4F6B78F4B2A34201D8BDE8F0812B78A7
:107488001C442046FFF7B4FF68B12046FFF7CEFF43
:1074980057F834303BB107EBC40204F01F045168BD
:1074A80008FA04F098470136E3E700BF6C33002080
:1074B800014B1954704700BFCF0A0020034670B132
:1074C800B0FA80F2C2F11F02D2B206498856064AC3
:1074D800D2F880100B43C2F88030FCF757BCFF226B
:1074E800F3E700BFCF0A002000200246034AD2F883
:1074F800803023EA0003C2F880307047002002463B
:10750800032921D8DFE801F0020C10190F4B1A6883
:1075180022EA00021A605A6822EA00025A6070479A
:107528000A4B1A680243F5E7084B5A6802435A6047
:107538001A6822EA00021A607047044B1A6802436C
:107548001A605A6810435860704700BF002002460E
:1075580030B5B0B1B0FA80F3C3F11F03DBB20B480A
:1075680050F833408C4204D100EBC3056D68954256
:1075780005D044B940F8331000EBC3004260002046
:1075880030BDFF23EBE76FF00F00F9E76C33002005
:1075980060B1B0FA80F3C3F11F03DBB20021044AE3
:1075A80042F8331002EBC30251607047FF23F5E73E
:1075B8006C330020C300074AC0F38100183052F82A
:1075C800202003F018000F238340134023FA00F013
:1075D800704700BF00200246F8B504690D4600AFA9
:1075E800A034D4E8AF3FC3F38003994217D1164AB9
:1075F800164B6E4688B0002908BF13466A461449E0
:10760800C2E905134FF400739383124B42F8103FFD
:1076180000234FF4E4511048FBF760FCB5464DB128
:10762800D4E8EF3F43F00403C4E8E23F002AF7D16F
:10763800BD46F8BDD4E8EF3F23F00403C4E8E23FB9
:10764800002AF5D0F6E700BF496C0508416C05082B
:10765800506C05080300000194B104082DE9F047B7
:107668000546894690461F46D0F808A02FF0C6FB6D
:107678000446D0B1067FF3070AD590F820301848A1
:107688000121184A2EF0F9F86FF07700BDE8F0876D
:107698003B46424649462FF071FB48B994F82030E2
:1076A8000121114A0E482EF0E8F86FF01200EDE7BC
:1076B8009DF8203026F0060684F82180678484F837
:1076C80024302677DAF81830214628469847B0FA49
:1076D80080F3227F5B0963F300022277D6E700BFBD
:1076E80094B10408626C05087C6C050870B5054601
:1076F80086682FF083FB0446D8B1037FDB0709D4E3
:1077080090F820300C4801210C4A2EF0B6F86FF0A2
:10771800770070BD0146F3692846984738B1237F42
:1077280003F00103227F63F300022277F1E70346A7
:10773800F8E76FF01200ECE794B104089E6C0508B6
:107748002DE9F3411746D0F808800546D8F83C30B3
:107758000E4698470022002339460B48FCF7F4FEF2
:10776800044670B901213B46084A094800962EF0A4
:107778008EF82846D8F840309847204602B0BDE831
:10778800F0810676F5E700BFE0100020B96C050827
:1077980094B1040870B50D460C7E497E0669C90788
:1077A800D6F88020D6F8A4301FD56CBBEA68D488F8
:1077B80043B1012B03D1D6F8A800FCF743FF0023FF
:1077C800C6F8A430C6F8A85064B3EB681C78E4097E
:1077D8000134D6F8A4309C4204D10221144A154839
:1077E8002EF042F8C6F8A44070BD6CB9012B1BD02E
:1077F800042B14D12B8A002BEBD002210E4A0D4802
:107808002EF032F80624E4E7052B0FD0022B04D122
:1078180082F0040303F00404DBE7032B06D0012104
:10782800064AECE70324D4E70524D2E70024D0E78E
:10783800106D050894B10408E36C0508F06C0508A0
:1078480013B503690C46D3F8AC0091F8201030F05A
:10785800DCFF94F8203048B101210090084A09481B
:107868002EF015F86FF0040002B010BD5B0601D1D0
:107878000020F9E7237F43F002032377F8E700BFEE
:10788800276D05089CB10408F8B503694768D3F863
:10789800AC4091F9203091F82060002B01DB0020EA
:1078A800F8BD7306FBD0488CB7F84830C0F30A001F
:1078B800834293BF033303308308C3F38D03402B04
:1078C80098BF5B00D4F8E8049D008AB9A84224BF99
:1078D800401BC4F8E80491F820100022204601F06B
:1078E8007F0131F02DF80028D9D06FF00400D7E7D8
:1078F800BA68121AAA4207D20A4832460A492FF031
:10790800F6FD6FF00B00CBE720469AB206F07F0138
:1079180031F016F80028E8D1D4F8E8342B44C4F83C
:10792800E834BCE79CB104084E6D0508F7B5466815
:1079380003697468D3F8AC5064009834A1B2074660
:10794800A400284631F01BF8C5F8E84401241022A9
:107958000021284630F0F4FFD5F8E8344033C5F864
:10796800E83473689C420ED3284630F054FE05462E
:1079780080B10246164917482FF0B9FD6FF004048C
:10798800204603B0F0BDE1B20022284630F0D8FF0F
:107998000134E6E702460146009040233846FFF7E7
:1079A8005DFE044628B12A460B490A482FF09FFD80
:1079B800E6E702460090402380213846FFF74EFE56
:1079C800044608B18022EFE73069FCF7DFF9D7E712
:1079D800716D05089CB10408866D050838B5044624
:1079E8000369D3F8AC5043681869FCF7DDF9002146
:1079F8002046FFF77BFE38B10C490D482FF07CFD7F
:107A08006FF00404204638BD20468021FFF76EFE43
:107A180004460028F0D1284630F01AFE0246002815
:107A2800F0D0044902482FF062FDE9E7A06D05088F
:107A38009CB10408C36D050838B503690546D3F839
:107A4800AC40204630F076FF024630B10D490E4872
:107A58002FF04DFD6FF0040038BD0021142031F0E7
:107A6800E9FE204630F069FF04460028F2D10146BD
:107A78002846FFF7B1FD2246022128462FF016FAC4
:107A88002046E9E7D76D05089CB1040870B503697D
:107A980045680446D3F8AC0030F0A8FD024618B19A
:107AA8001A491B482FF023FD6668F069D8B143686E
:107AB80098470446B8B10246164915482FF017FDF5
:107AC800002C19DB00F09CFC024618B11249104842
:107AD8002FF00DFD2869FCF77BF910B12869FCF738
:107AE80063F9002070BD0D48716983685B6843B90C
:107AF8000B4907482FF000FD0A4905482FF0FCFC08
:107B0800E0E798470028DDD0F2E700BFF86D0508E8
:107B18009CB104080E6E0508616E0508C8AC04081F
:107B28002C6E0508486E05082DE9F04103690646E4
:107B3800D3F8AC50476800F02FFC044638B1024631
:107B48002D492E482FF0D3FC2046BDE8F0817668F9
:107B58002B4896F84A307169012BD0F8088012D961
:107B6800D8F81830083153B9264924482FF0C4FCF6
:107B7800254922482FF0C0FC6FF00404E4E72246B0
:107B880098470028F0D1D8F8003071690BB91F491F
:107B9800EBE71B48984704460028F8D1F06950B134
:107BA80003689847064630B10246194913482FF032
:107BB8009EFC002EDCDB40F2E4420021284642F025
:107BC800CBFE3B6828462B607B682B7140232B72C9
:107BD8003B6B6B727B6BEB7102F0EEFE024620B1E1
:107BE8000C4906482FF083FCC6E7284630F030FDE4
:107BF8000028A9D0C0E700BF7F6E05089CB1040823
:107C0800C8AC04089C6E0508F66E0508BE6E05082B
:107C1800D96E05080E6F05082DE9F04F06464FF09E
:107C280000084FF0280A4FF0400BD0F81090446835
:107C3800D9F8AC708BB06368434559D84FF0000849
:107C48004FF0280A4FF0400B6368434500F29080DC
:107C580099F8803023F06E0343F06A0389F8803086
:107C6800636B2BB999F8803043F0010389F88030B1
:107C780007F5B86108230422C7F8E46407F5B26081
:107C880031F07CFBD4E9101207F59E654FF000082F
:107C98004FF000096FF0070301200027CDE90330FA
:107CA800CDE906892846CDE901775D4B009605F0B8
:107CB80013FC3168284631F009FDE36898473946D6
:107CC800A06909AA30F04EF9051E08DB099B3A465F
:107CD8001979186801F07CFC051E80F28480AB1CC1
:107CE80000F081802A464F494F482FF000FC21E0E0
:107CF8000AFB08F3E26B1A44917E41F04001917649
:107D0800E26BB8F1000F19D1917E41F00101917633
:107D1800E26BA2F818B0E26B30461A4482F8208071
:107D2800E16B19442FF07CF80546F0B13F493E4815
:107D38002FF0E2FB28460BB0BDE8F08F1A44917E85
:107D480041F004019176E26B1A44917E41F0020100
:107D58009176E26B1A44917E41F008019176E26BCC
:107D6800B4F848101A441183D5E708F1010862E70E
:107D78000AFB08F3A26B1A44917E41F02001917628
:107D8800A26BB8F1000F17D1917E41F001019176F5
:107D9800A26BA2F818B0A26B68F07F011A4482F8AF
:107DA8002010A16B304619442FF03AF805460028F8
:107DB800BCD108F1010847E71A44917E41F004015B
:107DC8009176A26B1A44917E41F002019176A26BE2
:107DD8001A44917E41F008019176A26BB4F84810DC
:107DE8001A441183D7E7A06A08B90025A2E7283406
:107DF80031F0DDF930B90E490B482FF07DFB6FF0FB
:107E0800150597E74FF4B01120462FF0FBFA00282C
:107E1800EBD0084904482FF06FFB6FF0040589E7A1
:107E2800157F00083E6F05089CB10408226F0508FD
:107E38005C6F0508786F050873B5D0F8AC60084624
:107E48000C4615462EF0E3FFB8B930466B8AEA684F
:107E580094F8201030F099FC58B194F820300121A2
:107E68000090074A07482DF012FD6FF0040002B099
:107E780070BD012120462EF0CEFF0020F7E700BF9D
:107E8800956F05089CB104082DE9F341036907467D
:107E980008460C461546D3F8AC802EF0B8FF78BBE0
:107EA80094F820102B8A80291E46EA6802D1402BBC
:107EB80028BF402691199B1B2B82E9603346404618
:107EC80094F8201030F087FC054660B194F8203013
:107ED800012100900B4A0C482DF0D9FC6FF00400EA
:107EE80002B0BDE8F081012120462EF094FF94F8FD
:107EF8002030802B04D11EB1294638462FF0A9FA2C
:107F08000020EDE7BB6F05089CB104082DE9F74F89
:107F18000369A04FD3F8AC50DFF87C824FF0FF32F2
:107F280001A94FF0FF3305F5B26004F0D9FE9DF8C2
:107F38000410012900F0C78002294CD00029EDD196
:107F4800D5F8E44405F29C4A20462EF057FF2EF05F
:107F580082FF08B1FCF776FB802120462EF04EFF09
:107F68002EF079FF08B1FCF76DFB082200212046AE
:107F78002FF0EEF8064620B9384688492FF0BCFAAB
:107F8800CCE72EF083FF0822514606F10C002DF0B5
:107F9800B3FE20463146FFF7FDFB20462FF00FFACF
:107FA80068B1F3682046D9882FF053FA10F10C0F06
:107FB8000246B3D1314620462EF084FFAEE7204674
:107FC8002FF004FA18B120462FF0ADF9A6E72046A5
:107FD8002FF0CFF9A2E79DF80590D5F8E46449F0B1
:107FE800800B594630462EF009FF824600212EF0BC
:107FF80012FF50462EF046FF044600288ED019F096
:108008007F0F18D1038A73B3402B28BF4023C2685F
:10801800594628461E4630F0DEFB024620B141464E
:1080280038462FF064FA79E7238A9B1B2382E3689A
:108038003344E36072E72EF030FF814678BB504648
:108048002EF005FF4A46214630462EF03BFF5046AB
:108058002EF018FF024600283FF460AF5146304624
:10806800FFF712FF5AE72EF018FFC0B950462EF05E
:10807800EEFE30462FF0B8F9F8B1214630462FF021
:1080880097F930462146FFF785FB30462FF0A5F9D2
:1080980000283FF443AF2046FCF7D4FA3EE72046D9
:1080A8002EF0FFFEE26800235946284630F093FB85
:1080B800024600283FF432AFB1E730462FF09BF973
:1080C8000028DAD1DDE79DF80590D5F8E464494643
:1080D8003046BDF806B02EF091FE04462EF0D2FED2
:1080E800824648B938464A462D492FF000FA51468B
:1080F80020462EF090FE11E759460C302DF0F6FD83
:10810800B9F1000F3CD130462FF067F9D8B12046BD
:108118002EF09DFE824601463046FFF73BFB514656
:1081280030462FF045F9002120462EF074FE2046F7
:108138002EF0A8FE024600283FF4F0AE2146306932
:10814800FFF77AFEEAE6BAF81020D5F8EC349A423E
:1081580009D2DAF80C1040230A44284694F8201073
:1081680030F013FBDAE620462EF071FE8246014617
:108178003046FFF70FFB514630462FF0AEF8D2E7F6
:1081880020462EF064FE0022014630462EF09AFE6C
:10819800C9E700BF9CB10408FF6F0508E26F050836
:1081A8001E700508F7B591F82150036905F003051D
:1081B800D3F8AC706B1E022B4FF001020C4688BF3F
:1081C8000025FFF761FB064698B9628C2B463846B6
:1081D80094F82010C2F30A0230F070FA48B194F80B
:1081E800203001210090044A04482DF050FB6FF024
:1081F8000406304603B0F0BD377005089CB104088A
:1082080013B503690C46D3F8AC0030F044FA40B11A
:108218000121009023460448044A2DF038FB6FF0F2
:10822800040002B010BD00BF9CB104085A700508D4
:1082380037B5036905460C46D3F8AC0091F8201011
:1082480030F075FA024630B92146284603B0BDE839
:108258003040FFF719BB94F8203001210090044A00
:1082680004482DF014FB6FF0040003B030BD00BFCC
:10827800807005089CB1040873B5036905460C466F
:10828800D3F8AC0091F8201030F0F6FA58B194F811
:10829800203001210090154A15482DF0F8FA6FF0AA
:1082A800040002B070BD237F60F3410323772046AA
:1082B8002EF0E8FD064608B90020F2E720462EF029
:1082C800A6FD94F92030002B07DA0028F4D13246B5
:1082D80021462846FFF7D8FDEEE70028ECD03246C5
:1082E80021462869FFF7A8FDE6E700BFA470050846
:1082F8009CB1040837B50D46044630F064FA0123F2
:108308008DF805508DF80430ADF8060000220023E2
:1083180001A904F5B26031F044F818B102490348E4
:108328002FF0EAF803B030BDCB7005089CB1040803
:10833800002307B5ADF8063002238DF805108DF837
:1083480004300022002301A900F5B26031F029F8B9
:1083580018B1034903482FF0CFF803B05DF804FBC8
:10836800CB7005089CB10408002307B501930022CF
:10837800002301A900F5B26031F013F8002803DAF0
:10838800034904482FF0B8F803B05DF804FB00BFB8
:10839800CB7005089CB1040838B54FF0FF324FF098
:1083A800FF33124804F030FE0446C0B9104D2B6864
:1083B8005A1C2A6083B90F4BDA6802F44032B2F5CE
:1083C800003F0ED26FF0040401210B4A0B482DF038
:1083D8004BFA2B68013B2B60044804F0DBFD204678
:1083E80038BD1A6942F080521A61F5E7641000201E
:1083F800CC35002000080246FE7005087CB1040850
:1084080010B54FF0FF324FF0FF330A4804F0FCFD7F
:10841800044660B9084A1368013B136023B9074A48
:10842800136923F080531361024804F0B3FD20461A
:1084380010BD00BF64100020CC35002000080246A3
:10844800074B1A6822F004021A605A68D207FCD453
:108458000222DA601A6842F001021A60704700BF0F
:1084680000040340044B1A6822F001021A601A68DB
:10847800D207FCD4704700BF000403400D4A0E49E0
:10848800936813F4000308D0936813F400030CD125
:10849800D2F8F42051F8230070479068000207D4FE
:1084A800D2F8F430C3F30333F4E793681B0FF1E712
:1084B8009268EFE7000C024634B8040838B5394B27
:1084C8000D4618680B881446C3F30B03112B31D8DB
:1084D80013B96FF0850040E0013B102BF9D801A2D9
:1084E80052F823F0658500083785000831850008B3
:1084F800DB840008DB840008878500087B8500088A
:1085080081850008578500085785000857850008A9
:108518005785000857850008578500088B8500088F
:1085280065850008658500084FF4FA400FE04FF4B0
:1085380000400CE0882B0AD003F67473C3F30B03D6
:108548001C2BC6D8184A22FA03F3DB07C1D52060D2
:108558002B68B3F5805F1ED2002038BDFFF78EFF71
:108568004FF42023A0FB0303400B40EAC34040081C
:10857800EDE7FFF783FFEAE70C4B1868E7E70C48DD
:10858800E5E7FFF77BFF4FF42023A0FB0303400B35
:1085980040EAC340DBE7C3F313330133B0FBF3F026
:1085A8002060D9E7300600201101111134B8040801
:1085B800006CDC0237B5A94CA94BE26902F00C0249
:1085C8001341D80700F14581FFF758FF236AA54AF0
:1085D80003F00F03D35C20FA03F5A34BDA6842F4E7
:1085E8004032DA60DA681104FCD5A048854201D22D
:1085F80003F056F8994CD4F8943043F00403C4F8C7
:108608009430D4F8943003F004030093009BFAF7F5
:1086180059F9D4F8F03023F0180343F01003C4F8E4
:10862800F030D4F8F03043F00103C4F8F030D4F857
:10863800F0309A07FBD5D4F8F03043F08003C4F843
:10864800F030864CD4F8F0301B05FBD5FAF758F912
:10865800A36843F40003A360A36823F0704343F0C6
:108668008043A360236843F040032360236843F0FA
:1086780008032360236843F001032360774B1A68DB
:108688005407FCD5D3F8942050070BD4D3F8942082
:1086980042F00402C3F89420D3F8943003F00403A2
:1086A8000193019B6D4CFAF70DF9D4F8F03043F0C3
:1086B8008063C4F8F030D4F8F0301901FBD5FAF72C
:1086C8001FF9236843F480532360644B1A689204AB
:1086D800FCD5DA6902F00C020C2A1AD11A68540582
:1086E80007D41A6842F480721A605C4A1368580505
:1086F800FCD55A4BDA6922F0030242F00102DA6132
:10870800DA6902F00C02042AFAD11A6A22F00F027E
:108718001A62524B1A6822F080721A609A6A22F022
:10872800030242F001029A624F4AD16821F4802183
:10873800D160D46814F48044FBD19A6A474922F482
:1087480070429A624A4B4B4A1B699342B6BF4A4AE7
:10875800102393FBF2F38A6A03EBD37322F470427B
:108768005B1042EA03338B623F4BDA6842F48022A3
:10877800DA60DA685104FCD5FFF780FE3F4AA0F5BD
:108788007413A3F51063934205D93D4B3A4A034449
:10879800934260D20C24314B9A6A22F470629A6236
:1087A8009A6A22F00C0222439A625A6B22F4FF72F0
:1087B80022F0010242F04F025A639A6A22F0100234
:1087C8009A625A6B22F4FE0242F480325A639A6A21
:1087D80042F400329A625A6B22F0FE4242F08072F2
:1087E8005A639A6A42F480229A621A6842F0807246
:1087F8001A601A689201FCD5DA6A22F00302DA627A
:108808001A6B22F003021A631A6A22F00F021A6224
:108818001A6A22F070021A621A6A22F4E0621A6274
:108828005A6A22F070025A62DA6942F00302DA6187
:108838000A4AD36903F00C030C2BFAD10B4CA5425E
:1088480002D3204602F02CFF00200E4B1C6003B020
:1088580030BD0020BAE66FF02100F8E7000C0246B0
:10886800FEEFFFFF587605080008024600688909F0
:1088780034B804080020A10700127A0000093D005E
:10888800FFED85FF30060020182808D8054BC340A7
:1088980013F0010F14BF00206FF0850070476FF0D0
:1088A80085007047CE7E030108B5074830F07FFC8D
:1088B80038B10648FBF782FD0448F9F7C3FF0020EA
:1088C80008BD6FF01200FBE7A4AE0408D9880008C1
:1088D8000A2838B50446074D04D1AB680D2128464F
:1088E8005B689847AB6803485B68E1B298472046E5
:1088F80038BD00BFA4AE0408064A11680B6823F00F
:1089080004030B605068044B196883685B6803B103
:1089180018477047EC0400205805002010B5094B93
:10892800D3E90040084B196883681B6803B198476E
:10893800236843F004032360236843F0080323609B
:1089480010BD00BFEC0400205805002008B5EFF367
:108958001181102383F31288BFF36F8F0120084B16
:1089680093F8482083F8480081F31188BFF36F8F8C
:1089780022B9FFF7D3FF5E20FBF708FA002008BDF5
:10898800EC040020F8B51646837890F803C0EFF39E
:108998001182102484F31288BFF36F8F077890F840
:1089A80001E0DB1B03EA0C039E4288BF9EB2BD199F
:1089B8000CEA05053C46057082F31188BFF36F8FFA
:1089C8008A198A421AD177450CD1EFF31182102106
:1089D80081F31288BFF36F8F0178417082F3118899
:1089E800BFF36F8F02799B1B9A4205D330F068FE64
:1089F80060B1084804F070FC3046F8BD05196D797F
:108A0800013401F8015B04EA0C04DAE7FFF79EFF82
:108A1800F2E700BF240500202DE9F8430D4614466F
:108A2800124F07F1560807F1180914B92046BDE896
:108A3800F8834FF0FF324FF0FF33384604F0E4FA82
:108A4800224629464046FFF79DFF064630B94FF0BB
:108A5800FF324FF0FF33484604F0D6FA3846A41BDD
:108A680004F098FAA4B23544DFE700BFF40400200C
:108A780010B54368046933486060196883681B68E7
:108A880003B19847012204F10800114630F091FD26
:108A98000122002104F1200030F08BFD04F13800A0
:108AA800294930F0D5FD072384F86130042384F880
:108AB80062300F23002284F84C300C23114684F8CE
:108AC8005E2084F85F2084F8602084F8492084F8C8
:108AD8004A2084F84B2084F84D305E202DF06CF845
:108AE8001A4B1B491B681A681C6922F07C4222F049
:108AF8007F028A42D86806D14AF2B0218C4202D15C
:108B08001449884211D0196821EA0201124A0A431D
:108B18001A604AF2B0221A610E4ADA601A6822F024
:108B280080421A601A685200FCD41A6842F00402A3
:108B38001A601A6842F008021A60FFF707FF00205F
:108B480010BD00BFC8AC040851770308EC0400202E
:108B5800000DF000BB7C0100000DF04010B51D4B6E
:108B680001461B68EFF31184102282F31288BFF3C9
:108B78006F8F5A68500605D45A68D2071DD46FF013
:108B88000A0015E01A6842F080421A601A6822F05A
:108B980080421A600A221868400005D458684006C6
:108BA80002D458684007E7D5013AF4D16FF00400C1
:108BB80084F31188BFF36F8F10BD5A689207F5D4FC
:108BC800586810F04000F1D19B680B60002BEFD182
:108BD800D5E700BFEC0400202DE9F347D8070F467E
:108BE800144605D42E48FFF7CDFE02B0BDE8F08745
:108BF800002A37D0EFF31185102383F31288BFF3CF
:108C08006F8F5E20FBF7E4F806465E20FBF7CCF892
:108C180085F31188BFF36F8FDFF88880FFF77EFE3A
:108C2800D8F800305A68510714D45B685A0611D432
:108C38004FF0804A2546DFF87090C9F888A1D8F827
:108C480000305B68DB070FD4BFF34F8F20BF40BFF6
:108C580020BFF4E701A8FFF781FF0024E6B15E20FA
:108C6800FBF794F82046C0E701A8FFF777FF002834
:108C7800C9F888A1E3DB6A1E291F019B17FA82F253
:108C880089B2013DADB202F801391B0A002DE5D0C9
:108C98008D42F6D10193D2E7FFF72EFEE2E700BF3F
:108CA80035050020EC04002000E100E02DE9F74341
:108CB80001A8FFF753FF002844DB0021042788465A
:108CC8000846264C019A94F84B3094F84CC094F816
:108CD8004AE0A3EB0E053CEA05055FFA82F91ED1CE
:108CE80094F8600094F85F6094F86150861B35EA48
:108CF80006062AD109B184F84B30B8F1000F00D02C
:108D080001925E20FBF750F8FFF7F6FD002384F888
:108D18004830134803B0BDE8F04304F03BB9E1180C
:108D280081F84E90012101330CEA0303013F4FF013
:108D380001084FEA1222CCD109B184F84B300192D4
:108D48000028E6D103B0BDE8F083261801300540BD
:108D580086F86390012084F86050E7E7EC0400206F
:108D68000C050020004870476CB40408044BB3F8A5
:108D7800A0379B020B60002318464B60704700BF6A
:108D88000000FA0B07B50346054A00910548012182
:108D98002CF07DFD6FF0150003B05DF804FB00BFFB
:108DA80056710508F4B0040873B50646642200231A
:108DB800684630F0F7FDDDE9004533691B681A6A3B
:108DC80012F0FA0212D01A6A02F0FA021A626FF06E
:108DD800040002B070BD22462B46684630F007FEFC
:108DE800DDE9003213430CBF0122002233691B68FE
:108DF800186A10F48030ECD0002AECD00A23012144
:108E0800024A03482CF039FDE1E700BF80710508EC
:108E1800F4B0040870B5036906461D6849B1FFF748
:108E2800C3FF044650B13069043004F0B3F820465B
:108E380070BDAB6A002B06DB0024F8E7AB6A43F091
:108E48000043AB62F8E7034BAB6003F18833AB60D8
:108E5800F2E700BF2301674573B5012306460D46B7
:108E680014462EF071FD50B90A482B4601210A4AD2
:108E780000942CF00CFD6FF0150002B070BD3CB1F1
:108E880022462946304602B0BDE870402EF00EBD9D
:108E98002046F2E7F4B0040894710508F7B51C46BB
:108EA80017460123224606460D462EF04DFD50B9C1
:108EB8000B482B4601210B4A00942CF0E8FC6FF07C
:108EC800150003B0F0BD44B123463A462946304662
:108ED80003B0BDE8F0402EF00EBD2046F1E700BF1C
:108EE800F4B00408BF7105082DE9F84F484B174640
:108EF8001B680D46834603F001080026FFF7B2FA07
:108F0800013FDFF81091DFF810A12F44AF420CD3D6
:108F1800DBF810301C68A36A002B0EDA01213F4AE7
:108F28003F482CF0A1FC6FF00406B8F1000F01D007
:108F3800FFF786FA3046BDE8F88F5846FFF734FF4A
:108F4800061EF2DBDBF810301B681B6C9B021AD57F
:108F58004FF6FF71B9F8A020236C8A4203F48013FE
:108F680007D1B5F5801F44D24BB1A36A43F400631F
:108F780008E0002AF5D0B5EB422F37D22BB9A36A07
:108F880023F40063A3626B0B09E0B5F5801FECD3F3
:108F9800A36A23F40063A362A5F580135B0BA26A9E
:108FA800584642F00202A262A26A22F47E72A262CB
:108FB800A26A42EAC303A362A36A43F48033A362AA
:108FC800A36AFFF7F1FEDBF8103006461B681B6C3E
:108FD80013F4001FA36A14BF03EA0A0323F0020371
:108FE8000028A362A1DB05F500558FE7B5F5801FC2
:108FF80005D3002BCCD1A36A43F40063CBE701214E
:109008002B46084A06482CF038FC6FF015068CE70A
:10901800000403400007FA0BFDF7FFFF1072050874
:10902800FCB004081D7205082DE9F84F0024984685
:10903800324B0D461F6806469146A346FFF712FAC3
:1090480007F0010705F10065D8450DD93369D3F854
:1090580000A0DAF82830002B0CDA0121284A294828
:109068002CF002FC6FF004040FB1FFF7E9F9204679
:10907800BDE8F88F3046FFF797FE041EF4DB2BF0AF
:1090880003024A44111F0B460C3253F8040F00BB6D
:109098009342FAD1DAF8283043F00103CAF82830AD
:1090A800DAF828302B4651F8040F914243F8040BA4
:1090B800F9D13046FFF778FEDAF82830041E23F09D
:1090C8000103CAF8283005F11005CDDB0BF1100BB0
:1090D800BAE7284600230468013408D005F178452A
:1090E8000121094A07482B442CF0C7FBBAE7013392
:1090F800042B00F10400EED1CCE700BF00040340CC
:1091080010720508FCB004083672050830B5104C1A
:10911800104D0C60236813B12B68136030BD0369D0
:109128001B68196C1B6C9B020FD54FF6FD700A4B20
:10913800B3F8A030591E89B281428CBF4FF48073B6
:10914800DB0823604FF40053636001232B60E4E7DE
:10915800D4350020D03500200007FA0B2DE9F8435C
:10916800D0F8049090460746D9F808000D461E46E8
:109178002DF0D4FDB8F5001F044616D12846D9F8BD
:109188000840FEF717FA84420CD129462DF0C6FD97
:109198000446FEF7ABF92046FEF7FAF9002120460F
:1091A800FEF7AEF90020BDE8F883B8F5800F20D0AF
:1091B800B6F1806F19D0B6F1C06F18D0B6F1007F44
:1091C8001AD102263A4620460E49FEF7C1F9B0B92F
:1091D8002846D9F808102DF0A6FD20463146FEF79E
:1091E8008FF92046FEF76AF9DCE70126EAE703264D
:1091F800E8E76FF08500D6E76FF01500D3E76FF06A
:109208000F00D0E7FB7B030808B5094A136943F050
:1092180000531361416807480C3183681B681BB110
:10922800984700EAE07008BD6FF05700F9E700BF03
:1092380000080246C8AC04080C291FB528BF0C2139
:109248000C460A4BD3F8082712BA0192D3F8042720
:1092580012BA0292D3F800370A461BBA01A903933F
:1092680041F053FB204604B010BD00BF0000FA0BCC
:1092780008B50121034A04482CF0F6FA6FF00400FF
:1092880008BD00BFE27205081CB1040898B5426821
:109298000369D26800AF83F8621029B9136823F410
:1092A80040131360BD4698BD6C468AB06A46036891
:1092B8000848D161C2E905034FF400731384064BD3
:1092C80042F8103F00234FF411510448F9F706FE05
:1092D800A546E7E700730508040000011CB104086F
:1092E800F7B500224368044606691C480F46DD6846
:1092F800596883680192DB684BB90121184A1948FB
:109308002CF0B2FA6FF00404204603B0F0BD01AAB5
:1093180098470028F1DB376306F118074FF0FF3252
:109328004FF0FF33384603F06FFE2B68204623F0DA
:1093380001032B6096F86210FFF7A8FF20460199F9
:1093480000F0A0F896F8613004461BB12B6843F092
:1093580001032B60384603F01DFED5E7C8AC0408AE
:10936800147305081CB1040870B5044646680569FD
:109378004FF0FF320021284630F01BF933682046B1
:109388009847002385F8603085F86230012205F19E
:109398001800114630F00DF9204600F03FF8316909
:1093A800184B994222D015D8174B994220D0174B09
:1093B800CB1A594259418900204641F01001FFF764
:1093C8008FFF041E18DA0121114A12482CF04CFABA
:1093D800204670BD104B99420CD003F5C31303F51A
:1093E800206399420CBF0A210021E5E70621E3E743
:1093F8000221E1E70821DFE70123002485F8603036
:10940800E6E700BF40420F00A0860100801A060070
:10941800427305081CB1040840E1330037B54568BC
:109428000021686901AA2EF09DFD041E07DB019B3F
:1094380000221979186800F0CBF8041E08DA012117
:1094480023460C4A0C482CF018FA204603B030BDCD
:109458000A48696883681B683BB90121084A0648BD
:109468002CF002FA6FF00404EFE79847044600284E
:10947800EBD0F2E7807305080CB10408C8AC040807
:109488009E7305082DE9F74F44680369002001938E
:10949800E369E568DFF81481DFF81491DFF814A1B7
:1094A800DFF814B10093009B8342019B1A6B0DD126
:1094B800C2F34202012A3BD0022A68D03F4A404800
:1094C80001212CF0D1F96FF015001FE00C2303FBEC
:1094D80000F7D4F818C0DFF8ECE00CEB0706736867
:1094E80073451DD015D853451CD05B4514BF0023C8
:1094F80001239B00C2F34202B2EB530F16D15CF872
:1095080007308B4212D1B36800202B6103B0BDE84D
:10951800F08F434508D04B450CBF0A230023E9E7E9
:109528000623E7E70223E5E70823E3E70130BAE784
:1095380041F25C2E4FF47A6C40F2E2474FF4FA762F
:109548000220214B421EB1FBF2F2B3FBF2F2BCFB4C
:10955800F2F4013CFF2C23D8BEFBF2F808F1FF38E7
:10956800B8F1FF0F1CD8B6FBF2F9B9F10F0F17D8F5
:10957800B7FBF2F2013A0F2A12D8023848EA094337
:1095880043EA007343EA025343EA0423BCE740F288
:10959800145E4FF4167C4FF4FA7740F27716CFE753
:1095A80001301128CED1094A89E700BF40E13300D4
:1095B800404B4C00A0860100801A0600CE730508B7
:1095C80014B1040840420F0000CA9A3B49740508C8
:1095D8002DE9F047044600251D4F00EBC106B442B3
:1095E80001D1002014E02068C30600F01F0911D43F
:1095F800656845F02005C0F3481AC0F344201928CF
:1096080023D857F82080B8F1000F0DD16FF0120061
:10961800BDE8F087B9F1100F04D0B9F1110FEAD104
:109628006568E8E73025E6E740462FF0C0FD0028EA
:10963800ECD04B462A4640460AF00F012EF0EFFACE
:10964800002804F10804CADAE2E76FF01500DFE742
:10965800B8B5040843681B6803F1080252E8002FF4
:1096680042F0010203F1080040E800210029F3D18B
:10967800174A93421ED002F1805293421AD0154ADB
:10968800934217D002F18052934213D0124A934268
:1096980010D002F1805293420CD0104A934209D064
:1096A80002F18052934205D00D4A934202D0B3F1A1
:1096B800502F03D15A6842F040025A6053E8002FF5
:1096C80042F4807243E800210029F7D1704700BFB7
:1096D800003801400044004000480040004C004071
:1096E8000050004043681B6803F1080252E8002F4D
:1096F80022F0010203F1080040E800210029F3D11B
:10970800174A93421ED002F1805293421AD0154A4A
:10971800934217D002F18052934213D0124A9342D7
:1097280010D002F1805293420CD0104A934209D0D3
:1097380002F18052934205D00D4A934202D0B3F110
:10974800502F03D15A6822F040025A6053E8002F84
:1097580022F4807243E800210029F7D1704700BF46
:10976800003801400044004000480040004C0040E0
:10977800005000400129034608461AD002290BD0A0
:10978800C9B91B680D4A934217D002F180529B1A3F
:1097980018BF0123180370471868084B98420AD06D
:1097A80003F18053984214BF4FF440504FF40050D7
:1097B8007047002070474FF400507047002400465F
:1097C80070B500261D46094B6C0833F81220334645
:1097D800F7F754FD090241EA1061000220182A46F1
:1097E800334641F10001F7F749FD70BD9054050873
:1097F8002DE9F04782B0436880460C461D6800AFEB
:10980800002944D0586819698368DB686BB13A1D30
:109818009847061E0CDA0121354A36482CF024F800
:1098280030460837BD46BDE8F0876FF05706F2E7C7
:10983800314B9D4203D003F180539D4249D100260C
:10984800D7F80490DFF8B4A0234648460021B2B206
:10985800FFF7B6FFA0F5407050451BD90136102E12
:10986800F2D16D468AB0D8F800306A462449D461EE
:10987800C2E905134FF400731384224B42F8103FDA
:1098880000234FF411511B48F9F728FBAD466FF040
:109898001506C5E7EB6A484623F00F033343EB622E
:1098A800194B33F8162000231946F7F7E7FC09028D
:1098B80041EA106163080002C01822464FF0000315
:1098C80041F10001F7F7DAFCC0F31300E860002665
:1098D800A6E72B6823F400432B607B6803EB540353
:1098E800B3FBF4F30F2BBCD99BB2EB60EFE700BFDF
:1098F800147305088CB1040800240046FFFC0F000F
:109908008D74050804000001905405082DE9F843FA
:1099180007460D7940683B69012D0E460468D3F867
:10992800008017D0AB1ED3F1000949EB03094FEAB9
:1099380089297179FFF71EFFB2790346022A0CD0F4
:10994800042A0ED0ADB1033D012D0CD86FF085006F
:10995800BDE8F8834FF4C069EBE73DB94FF080509C
:1099680008E0002DF2D14FF4805003E0033D012DB3
:10997800ECD90020B3F5805F4ED0B3F5405F4DD0F1
:10998800002B0CBF012303239942DFD149462EF057
:1099980034FB8242DAD1F37953B3012B40D1224B05
:1099A8009C4225D003F180539C4221D01F4B9C42FE
:1099B8001ED003F180539C421AD01D4B9C4217D0F5
:1099C80003F180539C4213D01A4B9C4210D003F1F0
:1099D80080539C420CD0184B9C4209D0B4F1502FB4
:1099E80006D0164B9C4203D003F180539C42ADD164
:1099F8002368314623F00103384623602EF081FCAA
:109A08000028A3DB236843F00103236096E80300E2
:109A180088E8030000209BE70023B5E70223B3E7AB
:109A2800032BBCD092E700BF00380140004400403F
:109A380000480040004C0040005000400024004610
:109A48002DE9F04383B0466805467068316983683C
:109A580000AF1B685BB90121724A73482BF004FF01
:109A68006FF0570420460C37BD46BDE8F083984791
:109A7800044630BB0021706A3A1D2EF073FA041EAA
:109A8800F0DB7B68002219791868FFF7A1FD041E36
:109A9800E8DBD5F804802B69D8F80040D3F80090AB
:109AA800236823F001032360D8F808002FF07FFB18
:109AB80078B901215D4A5C482BF0D6FE6FF012049C
:109AC800D0E70121574A58482BF0CEFE002CC9DBBD
:109AD800D0E7D8E902018368DB6803B1984754E806
:109AE800003F43F00C0344E80032002AF7D149460E
:109AF80028462EF006FC002802DA6FF01504B1E7BC
:109B080098F818301BB1A36843F00803A36098F8CD
:109B180019301BB1636843F40043636098F81A3046
:109B28001BB1636843F48033636098F81B301BB142
:109B3800636843F40033636098F81C30002B5AD0F4
:109B48003B4B9C423AD003F180539C4236D0394B70
:109B58009C4233D003F180539C422FD0364B9C4219
:109B68002CD003F180539C4228D0344B9C4225D002
:109B780003F180539C4221D0314B9C421ED0B4F15A
:109B8800502F1BD02F4B9C4218D003F180539C427E
:109B980014D06C4688B06A462B682B49C2E9051375
:109BA8004FF400739383294B42F8103F00234FF47E
:109BB800E2511D48F9F792F9A5469EE76B681A68C5
:109BC800936843F480439360236898F81D2023F03A
:109BD800787343EA42532360236898F81E2023F4DD
:109BE800F81343EA0243236098F81F301BB1A368B7
:109BF80043F40043A36098F820301BB1236843F076
:109C080000532360236843F001032360E3699A0249
:109C1800FCD5E3695B02FCD52846B36A9847002463
:109C280020E700BFA47405088CB10408C4740508B3
:109C3800003801400044004000480040004C00400B
:109C48000050004000240046DF74050803000001AE
:109C580038B50B68054698882EF020FC04280C4679
:109C680003468A6D1AD002280FD191F87010012985
:109C780002D9A16E012911D8002A49D0E16D01B19C
:109C8800118889B2298402250EE0012821D191F892
:109C98007010032918D9A16E032917D992B1E16D63
:109CA80001B1116829620425E26DB5FBF3F53AB1FB
:109CB8009542294619D901211B4A1C482BF0D4FD8D
:109CC800284638BD1146EDE7012902D9A16E0129C0
:109CD800D2D8FAB1E16D01B11178C9B285F8201076
:109CE800E26D0125002AEBD02946521AE2659AB99D
:109CF800A26C04F14C010832A264E26C04F1480041
:109D0800013AE26404F15C022EF0B2FBA065D7E7E9
:109D18001146B6E71146E0E7A26D002AD0D001FB54
:109D28000322A265CCE700BF3C75050864B10408AE
:109D380038B50B68054698882EF0B0FB04280C4609
:109D4800D1E91812034618D002280DD194F87000F2
:109D5800012802D9E06E01280FD8288E80B209B1F7
:109D680002B1088002250DE001281DD194F8700089
:109D7800032814D9E06E032813D9286B09B102B15E
:109D880008600425626EB5FBF3F59AB19542294641
:109D980018D90121184A19482BF066FD0AE0012854
:109DA80002D9E06E0128D8D895F83000C0B229B1A0
:109DB80012B90125284638BD0870626E002AF8D00D
:109DC80001252946521A62667AB9226D04F15401B6
:109DD80008322265626D04F15000013A626504F1AF
:109DE80064022EF045FB2066E4E7226E002AE1D0EB
:109DF80001FB03222266DDE73C75050864B104080F
:109E080038B50446006903691BB94360083003F09C
:109E1800C1F8012160682EF086FB002802DA10F1F3
:109E2800860F15D16568002128462EF07CFB041E9C
:109E38000CDB0948A96883681B6853B19847044636
:109E480020B10121054A06482BF00EFD04EAE47012
:109E580038BD6FF05704F4E7C8AC04085A75050814
:109E680064B104082DE9F04F87B081460E469B4641
:109E78009246046900AF32B92BB9002630461C3728
:109E8800BD46BDE8F08FB3889A042FD44FF0FF3257
:109E98004FF0FF3304F1080003F0B6F866600023C2
:109EA800C4E90F3384F84430D9F81030D9F8048065
:109EB800FB601B68D8F800509E4240F0B580B3881C
:109EC8001B0540F1AC81BAF1000F16D028464FF4BB
:109ED800C1212EF0BEFAB0882EF0E0FA0346DAF877
:109EE8000020A264A2B1DAF8042011E02369002B53
:109EF800CCD163689E42C9D1D1E728464FF4C0212E
:109F08002EF0A7FAB0882EF0C9FA03460022A26400
:109F1800E26404F14C0104F15C0204F14800FB60C6
:109F28002EF0A6FAFB68A065BBF1000F40F0938104
:109F3800C4F850B00022626504F1540104F16402CF
:109F480004F150002EF094FA00232066A3632A68D7
:109F5800EB6802F4006203F4C0231343FB6098F833
:109F68002130DB0728D5B288D9F80430D007BB6088
:109F78001B6821D41968D86801F4006100F4C02076
:109F88000143D9F8102040F07181D16D566E29B186
:109F9800002E00F069818E4228BF0E46002E56DB47
:109FA800B968C969B142C0F06F81C2E91A665A68D6
:109FB800120C120432435A60D9F804301B681A682C
:109FC80042F001021A60DA68510206D51A6842F4B2
:109FD80000721A601A689205FCD5E36D1BB9666EAB
:109FE800002E00F0F0812268D8F800609288D2072D
:109FF80040F150817269920740F15482002B00F0C1
:10A00800518221463046FFF723FE7369D80740F195
:10A018005F81236E002B00F05B81636E002B00F0E4
:10A028005781214630462EE2D8F81020B188022AFE
:10A03800C1F3451312D0032A13D0012A2CD1043BB3
:10A048001C2B8CBF002301237BB96FF085060023EE
:10A05800636004F1080002F09DFF0FE7043B0C2B3E
:10A06800EFE7082B01D0102BEFD1080448BFEB68AD
:10A07800A44842BF23F4601343F40023EB608368D1
:10A08800D8F80810DB686BB901219F4A9F482BF06C
:10A09800EBFB6FF00406DAE701219D4A9B482BF0A1
:10A0A800E3FBD2E707F1140298470028ECDB002213
:10A0B8007B69316823FA02F0884218D90132092AEB
:10A0C800F8D16D468AB06A46D3611B0A136205232C
:10A0D8009048C2E9050142F8103F00234FF421518E
:10A0E8008A48F8F7FBFEAD466FF01506AFE72B6818
:10A0F800894923F001032B60AB6851F8222023F033
:10A1080070431343AB6098F82130990700F19080B1
:10A11800B38813F0020FEB6814BF43F0007323F009
:10A128000073EB60B38813F0040FEB6814BF43F0BF
:10A13800807323F08073EB60B18811F4006104D060
:10A14800BAF1000F7BD04FF4C12128462EF081F9D7
:10A15800B38813F0100FEB6814BF43F4000323F423
:10A168000003EB60AB6823F48003AB60327DB388F7
:10A178001AB998F82120520764D5D80706D4EB6895
:10A18800D9005EBF2B6843F480532B60EB6823F043
:10A19800105343F08063EB60B388604913F0010FFC
:10A1A800EB6814BF23F4800343F48003EB60B288A8
:10A1B800AB68C2F34512043A51F8222023F01F037A
:10A1C8001343AB60EB68D8F8182023F00F03134350
:10A1D800EB60EB68D8F8142023F0F00343EA02138D
:10A1E800EB6098F821304E49DA0741BFB38898F8F8
:10A1F8002020C3F34513073343BFDB085B00B2FBE2
:10A20800F3F30123FA6882F87030AA68013B51F829
:10A21800233022F4F0721343AB60FB681E60B088F1
:10A228002EF03CF90346BAF1000F7FF458AE6DE604
:10A23800D8F80020D36843F40043D36068E74FF4AC
:10A24800C02182E713F0010FEB6823F0105308BF19
:10A2580043F000539FE7DBF800202265002A3FF413
:10A2680069AEDBF8042066E60E4697E6B1F5C12F25
:10A2780030460CBF51465946C7E900322EF031F935
:10A28800D7E90032064689E60121264A1F482BF005
:10A29800EBFA29E798F8213013F0010F3368F268D8
:10A2A80000F0E28003F4006302F4C022134354D1A7
:10A2B80073695B0738D47369D8073BD5E36E002B05
:10A2C80038D0214630462EF074F973691B0758D4EC
:10A2D800D8F80060736913F4787340F0E880FB687D
:10A2E800B3F5C12F7FF479AEE36D002B00F0FE804B
:10A2F8002B68EA6803F4006302F4C0221343FB608E
:10A308006BE600BFC8AC04089D75050864B1040875
:10A3180075750508C975050820B70408C0B704088D
:10A32800A0B70408F8750508A36E002BC3D0E36E28
:10A3380073B9736973699A07C7D5A36E002BC4D024
:10A34800E26E9342C1D1214630462EF01EF9BCE799
:10A35800214630462EF019F9B3E7B3F5C12FE9D0FD
:10A368007269D10702D5E26E002AAAD1B3F5C02FCF
:10A37800ABD0DFE721463046FFF7DAFCE36E1B1A65
:10A38800E366E36E002BF5D1E36D626E002B53D1CB
:10A39800C4E91A22002A9BD0B369304643F010035F
:10A3A800B361B36943F00803B3612EF0D1F8A26E2C
:10A3B800D8F81C309A4246D901218E4A8E482BF093
:10A3C80053FA6FF01506D9F80450D9F810802968A7
:10A3D8004B69D80700F1D380CB685A0240F1D2808C
:10A3E800DFF8189208462EF06EF8002800F0CA80B0
:10A3F8000B68D80740F1C68095F82130DA070DD4EC
:10A40800D8F800309B88C3F34513192B06D829FACE
:10A4180003F3DB0702D508462EF09AF80B68CA68E2
:10A4280003F4006302F4C0221343B3F5C02FD9D15B
:10A4380008462EF08DF8D5E712B1934228BF13468F
:10A44800C4E91A33A8E7736821461B0C1B0413439D
:10A458007360336843F001033360336843F4007377
:10A4680033602EF092F833E703F4006A02F4C02355
:10A478004AEA030ABAF5C02F08D1D8F800004369A0
:10A48800D907FCD52146FFF753FC21E773699807E4
:10A49800FCD521463046FFF7DBFBBAF5C12F3FF468
:10A4A80017AFEAE7336923F002033361ADE56D4680
:10A4B8008AB06A46524951615249C2E906134FF4BB
:10A4C80000731384504B42F8103F00234FF411518E
:10A4D8004948F8F703FD7369AD46590603D5B369D2
:10A4E80043F04003B3616FF004066CE7636E002B22
:10A4F8003FF4FEAE30462DF0E6FF03460028F9D1C2
:10A50800326822F00102326022689088C20712D4B1
:10A518001A46D4F854C0624527D12DF0BFFF93FBEB
:10A52800F0F200FB12323ABBB3FBF0F37268120C84
:10A538001204134373604FF4C02130462DF089FF95
:10A54800336843F001033360F3685B027FF5D0AEF4
:10A55800336843F400733360336898053FF5C8AE39
:10A56800736919073FF5C4AEF6E7216D01EBC20127
:10A57800496801320B44CEE72B68EB6821E791F874
:10A58800303025E74B699B0542BF8B6943F4007364
:10A598008B6195F821000B68C007CA6810D58B69D4
:10A5A80043F010038B618B6943F040038B618B6927
:10A5B80043F008038B614B681B0C1B044B6007E0DE
:10A5C80003F4006302F4C0221343B3F5C02FF2D0A2
:10A5D800D8F800309B88DB0402D408462DF0B8FF79
:10A5E80094F84430002B3FF432AD002E3FF445ACD4
:10A5F8002DE500BFF875050864B1040800020202E1
:10A60800247605082F760508040000014FF0E023A2
:10A6180010B50F499C691A6908689B690D4902F4CD
:10A62800803234B993B903464AB90A681044C01A4B
:10A6380010BD002B08BF03460AB9A342F5D90A6822
:10A6480002440A604FF0E0221269EEE70446F3E79D
:10A6580048370020443700201022094B002083F897
:10A6680023204FF47A52074B1A60074B43F67F6258
:10A6780018604FF0E0235A61072298611A61704709
:10A6880000ED00E04837002044370020684620F0FD
:10A6980007018D4619B5FFF7B9FF1149114B086835
:10A6A800D3E90042001942F10002C3E90002002385
:10A6B8000B604FF47A530C4AD2E90041001BB0FBFF
:10A6C800F3F043431B1941F10001C2E9003103F0E3
:10A6D800E5FBF9F77FF8BDE819408546704700BFEC
:10A6E80044370020882D0020802D00202DE9F041DE
:10A6F800DFF8E08099B1421C0BD14FF0E0221369DA
:10A7080023F0010313614FF07F43C8F80030BDE820
:10A71800F081D8F80060012807DC00270BE0431C13
:10A72800D8F80060F7D140F21740B0F5836FA8BFA2
:10A738004FF48360471EEFF31185102383F31288CB
:10A74800BFF36F8FFFF762FF4FF0E023224C996948
:10A75800D4E9002380184FF0000243F10003C4E954
:10A7680000031E4B1A601E4B1A68831A2ED44FF42E
:10A778007A5C0CFB073303F579533F33B3FBFCF7E3
:10A78800131A0CFB0733B3F5806F38BF4FF480639F
:10A79800144A934228BF13464FF0E022C8F800300D
:10A7A800013B90695361002381429361A1EB00034F
:10A7B80038BF9B19D4E900125B1842F10002C4E9C2
:10A7C800003285F31188BFF36F8FA0E74FF48063E1
:10A7D800E2E700BF48370020882D002044370020DA
:10A7E800802D0020809DFF0038B5EFF311851023E0
:10A7F80083F31288BFF36F8F084B1C68084B1B68E4
:10A80800E41AFFF703FF85F31188BFF36F8F4FF446
:10A818007A532044B0FBF3F038BD00BF882D0020E8
:10A82800802D002038B5EFF31185102383F31288AB
:10A83800BFF36F8F044B1C68FFF7E8FE85F31188A0
:10A84800BFF36F8F204438BD882D00202DE9F041DB
:10A858004B4AD369916A13F00C0342D00C2B52D1A6
:10A8680001F0030101293CD00024D369444EB36AA6
:10A87800B56A03F00308B06AB36BC0F30010C3F302
:10A88800CC035843F6F730FAC5F30325B8F1020FA5
:10A89800074605F1010542D0B8F1030F3FD0706BB0
:10A8A800C0F30800F6F720FA4FF064510646384620
:10A8B800F6F772FA01463046F6F766F94FF07E5120
:10A8C800F6F762F906462046F6F70EFA04462846D9
:10A8D800F6F70AFA01462046F6F712FB014630461B
:10A8E8003AE09168090254BFD2F8F42092682549E9
:10A8F80054BFC2F30332120F51F8224063B10C2B3C
:10A90800B4D0002408E0D26902F00C02042A35D041
:10A91800082B1D4C18BF00242046BDE8F081706B41
:10A92800C0F30800F6F7E0F94FF0645104463846E2
:10A93800F6F732FA01462046F6F726F94FF07E512F
:10A94800F6F722F904462846F6F7CEF901460F48ED
:10A95800F6F7D6FA01462046F6F71EFA084B0446E3
:10A96800586BC0F306600130F6F7BEF90146204681
:10A97800F6F7C6FAF6F712FC0446CDE7024CCBE729
:10A98800000C024634B804080024F4000024744B78
:10A9980008B5FFF75BFF054B054A1B6A03F00F0379
:10A9A800D35CD840034B186008BD00BF000C0246BA
:10A9B8005876050830060020F7B5044610B390F81D
:10A9C8009534056803F0FF021BB980F894242DF034
:10A9D8000BFE032384F89534324B20689D4204BF54
:10A9E8000023A3712EF027F8237C251D8DF8003055
:10A9F80095E80E0020682DF0DAFF014630B10223F9
:10AA080084F895340125284603B0F0BD20682EF05F
:10AA180018F80028F3D101270246267904F1140317
:10AA2800C1B28E4203F1240321D800210A4604F55D
:10AA38001573C8B2864203F1240326D8237C8DF807
:10AA4800003095E80E00206800F00AFC0546002852
:10AA5800D5D10123607484F89534237B012B02D16E
:10AA680020462DF090FF20682EF0F8F9CBE723F868
:10AA78000A0C43E9072203F8237C03F8241C03F893
:10AA8800202C43F8142C0130CAE743E9072203F8C5
:10AA9800232C03F8240C03F8202C43F8142C013140
:10AAA800C7E700BF000004422DE9F04F066889B0EF
:10AAB800044630462EF00EFA0390002840F06E81CE
:10AAC80020682EF0D9F9002800F06881D6F80838F7
:10AAD8002068C3F30D23C4F8D4342EF0CDF98707CA
:10AAE80048BF226806F5006542BF536903F00203B8
:10AAF800536120682EF0C0F9C0062CD522689369EE
:10AB080023F010039361D6F82080C8F34343022B47
:10AB180008F00F0740F0458147F6F07318EA030F75
:10AB280014D0242303FB0747C8F30A194A463046C2
:10AB3800D7F860122EF034F9D7F860324B44C7F8D2
:10AB48006032D7F868324B44C7F868322268936994
:10AB580043F01003936120682EF08EF9010300F191
:10AB6800328120682EF088F942030DD520682EF036
:10AB78008FF927464FF0000A049006F5106B049BE6
:10AB88002068002B40F0EA8120682EF075F9002833
:10AB980013DA6B6823F001036B6094F8CC34012B53
:10ABA80040F084820021204684F8CC142DF0FEFE6B
:10ABB8002268536903F00043536120682EF05CF962
:10ABC80001050AD5AB68DA0702D520462CF004FD4A
:10ABD8002268536903F40063536120682EF04CF92E
:10ABE800030115D52268536903F00063536194F893
:10ABF800CC34002B40F05E820121236884F8CC1409
:10AC08005B6D2046C3F38303C4F8D0342DF0CEFE29
:10AC180020682EF031F9C70433D56B68102123F072
:10AC280001036B6020682DF03AFF4FF67F3106F57F
:10AC3800106322790398824200F24082EB6943F064
:10AC48000113EB61E37B002B00F05682D5F88430CA
:10AC580043F00B03C5F884306B6C43F00B036B6453
:10AC6800D6F8003804F29C4223F4FE63C6F8003894
:10AC7800A179206800F0EEFC2268536903F4805340
:10AC8800536120682EF0F8F8800416D520682EF05D
:10AC980025F920682DF04EFFE0712768FFF778FE50
:10ACA800E2790146384600F06BFA20462CF05CFC4D
:10ACB8002268536903F40053536120682EF0DCF8CE
:10ACC800010707D520462CF0A5FC2268536903F03C
:10ACD8000803536120682EF0CFF8020600F11782AE
:10ACE80020682EF0C9F8C3020CD5A046012706F546
:10ACF80012692379BB4200F228822268536903F45F
:10AD08008013536120682EF0B7F8870229D52346AF
:10AD1800012206F53261207990421DD993F87C72A0
:10AD28000868012F40F02782002880F22482D4F896
:10AD3800D4C48CEA1040C00700F11D8283F87B72EE
:10AD4800B06940F08000B0617069000600F11382BC
:10AD58006B6843F400736B602268536903F4001353
:10AD6800536120682EF088F8410007D520462CF062
:10AD780027FC2268536903F08043536120682EF052
:10AD88007BF842070AD523685D686B0702D5204621
:10AD98002CF01CFC226853682B43536009B0BDE8B3
:10ADA800F08F062B7FF4D2AE0822304604F29C4185
:10ADB8002DF0F6FF242303FB0747D7F86832C8F3C2
:10ADC8000A184344C0E620682EF05AF8A246002725
:10ADD800049006F53068049B2068002B3FF4C1AE50
:10ADE800049BDB0765D55FFA87FB59462EF058F8B8
:10ADF80010F0010F81461ED00123C8F808302068E2
:10AE080094F806C000F5306303EB4713BCF1010F5B
:10AE1800016C9A687BD112F0080F07D0B4488142C0
:10AE280009D9120407D54FF4004203E012F0200FAD
:10AE380048D020229A6019F0080F0FD00823C8F8CC
:10AE480008302368AA49186C03F5306303EB4713ED
:10AE580088429A6870D82046FDF786FA19F0100FD4
:10AE68001CBF1023C8F8083019F0020F14D07369FA
:10AE78001A0642BF6B6843F480636B609AF85732D6
:10AE8800012B06D10023594620468AF857322DF067
:10AE980000FC0223C8F8083019F0200F1CBF20233B
:10AEA800C8F8083019F4005F1CBF4FF40053C8F805
:10AEB8000830049B01375B08049308F120080AF165
:10AEC800240A88E712F0280FB5D1DFF824C26145BB
:10AED80001D91204A7D41A69DAF87432C2F312023B
:10AEE8009B1ACAF868326FB9D4F864222AB90121CA
:10AEF80004F29C4200F0AEFB04E0D4F860221A444D
:10AF0800C4F8602259462046FDF7F4F993E7DFF8C4
:10AF1800E4C1614506D1110485D49006F2D52022FA
:10AF28009A60EFE7002FEDD1D4F86432002BE9D115
:10AF3800394604F29C42DDE7110448BF4FF4004251
:10AF4800204648BF9A60FDF70FFAA179012985D1FB
:10AF5800206804F29C4200F07DFB7FE7049BDB073E
:10AF680040F19B805FFA8AF3194607932DF0A1FF01
:10AF780010F0010F804620D001216B6B0AF00F0200
:10AF880001FA02F223EA02036B63CBF80810A179F5
:10AF980001290DD1D7E9072313443B62BAF1000F09
:10AFA80006D1636A23B9206804F29C4200F052FB80
:10AFB80020465FFA8AF1FDF7BBF918F0080F1CBFAD
:10AFC8000823CBF8083018F0100F1CBF1023CBF85B
:10AFD800083018F0400F1CBF4023CBF8083018F099
:10AFE800020F10D0514630462DF059FDFB7D012B44
:10AFF80006D100232046FB755FFA8AF12DF04AFB43
:10B008000223CBF80830236818F0800F059344D04A
:10B01800D7E909329A4240D8A3EB0208FB69984560
:10B0280028BF9846059B08F1030803F5106303EB56
:10B038004A134FEA98080693069B9969D7E909329B
:10B0480089B2414527D393420BD80121059B0AF0C9
:10B058000F00D3F83428814022EA0102C3F83428CB
:10B068001BE0A3EB0209FB69079A994528BF99469B
:10B07800A37905980093396A1FFA89F32DF07DFEAC
:10B088003B6A09F103084B443B62BB6A4FEA9808E4
:10B098004B44BB62D0E79342D7D9049B0AF1010A1B
:10B0A8005B08049324370BF1200B68E520462CF04D
:10B0B800A2FA7DE520462CF08FFAA9E599601A6876
:10B0C800203322F4001243F8202CC3F8E811D3F8F7
:10B0D800E02122F40012C3F8E021D3F8E02142F085
:10B0E8000062C3F8E021039A01320392A1E500BF90
:10B0F8000A30544F0A31544F6B6943F4005343F0FC
:10B108002B036B612B6943F00B032B61A8E501222C
:10B118002427B36904F2572023F08003B36106F5AE
:10B128003263217991427FF6DBAD07FB02F1415C86
:10B13800012907D1196841F000611960196841F0C7
:10B148008041196001322033EBE798F83C30D9F898
:10B158000020012B09D1002A07DA67F07F01204679
:10B1680088F83B30C9B22DF0BCFB013708F1240840
:10B1780009F12009BDE5013224332031CBE500BFB8
:10B18800022A4AD1274B284A0B44934239D9274BE4
:10B19800274A0B44934236D9264AA1F57403A3F5EE
:10B1A8001053934231D9244AA1F18373A3F5E7439D
:10B1B80093422CD3214B224A0B44934229D9214B49
:10B1C800214A0B44934226D3204B214A0B449342F5
:10B1D80023D3204AA1F1B773A3F5585393421ED342
:10B1E8001D4B1E4A0B4493422CBF06230723C268FB
:10B1F80022F47052C260C26842EA8323C36000200E
:10B2080070470F23F3E70E23F1E70D23EFE70C2335
:10B21800EDE70B23EBE70A23E9E70923E7E7082330
:10B22800E5E700BF405327FFFF340C00401E1BFF1B
:10B238003F420F007F4F120020D6130060B6E5FE94
:10B248005FE3160000D3CEFE40771B00C05BB3FE61
:10B25800C091210020753800E05459FEE09C41005F
:10B2680084B02DE9F041044607A880E80E000023C9
:10B2780019469DF81C709DF8268003F140020133A1
:10B2880004EB82020F2B5160F7D104F50066B8F188
:10B29800000F46D1736843F002037360A36B23F475
:10B2A8000013A363236843F040032360236843F03B
:10B2B80080032360002503212046C4F8005E2DF09A
:10B2C80032FC102120462DF0EAFB014620462DF0E5
:10B2D80009FC0843C0B2401B356118BF01207561E5
:10B2E80004F51063F561002F46D0D4F80029AA426E
:10B2F8001CDA4FF00062C4F8002900224FF67F31B3
:10B308000135AF421A61996003F1200311D9D3F8CE
:10B3180000C0BCF1000F09DA4FF0904CC3F800C030
:10B32800EEE7A36B43F40013A363C3E700221A609C
:10B33800E3E7D4F8002B04F53063002A18DA4FF05D
:10B348000062C4F8002B002200214FF67F3501323D
:10B35800974219619D6003F120030DD9D3F800C00D
:10B36800BCF1000F05DA4FF0904CC3F800C0EEE7CF
:10B37800002200211960E7E7336923F48073336101
:10B388000023A3616FF0804363619DF81E301BB9F1
:10B39800A36943F01003A361A2690B4B1343A36194
:10B3A8009DF822301BB1A36943F00803A361B8F1EB
:10B3B800010F01BFA36943F0804343F00403A36175
:10B3C800BDE8F04104B0704700383C8030B54A7899
:10B3D8000B78012A00EB431300F5006029D1D3F85C
:10B3E8000029002A0BDAD3F8002942F00062C3F8DA
:10B3F8000029D3F8002942F08042C3F8002901242B
:10B408000A78C56B02F00F0204FA02F225EA02027A
:10B41800C2630978C26901F00F018C4022EA040274
:10B42800C261D3F80019174A0A40C3F8002900205E
:10B4380030BDD3F8002B002A0BDAD3F8002B42F0EA
:10B448000062C3F8002BD3F8002B42F08042C3F807
:10B45800002B01240A78C56B02F00F0204FA02F2ED
:10B4680025EA0242C2630978C26901F00F018C40E3
:10B4780022EA0442C261D3F8001B034A0A40C3F817
:10B48800002BD4E7007833EC0078F3EFF7B54B786E
:10B498000F78012B6C4EDFF8B4C100EB471440F075
:10B4A80089800D6904F5106345BB1D6935401D6130
:10B4B8001D6945F400251D611D6905EA0C05012A71
:10B4C8001D614CD1CA6902B15A610B79012B0CD1AB
:10B4D800D0F8083813F4807FD4F800390CBF43F053
:10B4E800005343F08053C4F80039D4F8003943F0CE
:10B4F8000443C4F80039002003B0F0BD1D6905EA13
:10B508000C051D611D6935401D610D698E6867B99F
:10B51800B54288BF0E611D6945F400251D610D699E
:10B528001E69C5F312053543C9E73544013DB5FB2E
:10B53800F6F5474FD3F810C0AEB207EAC54545EA5D
:10B548000C051D610D79012DE9D11D6925F0C04556
:10B558001D611F69750705F0C0453D43DEE7D4F856
:10B56800003943F00443C4F800390B79012B0DD09E
:10B578000B69002BBFD001230A78D0F8344802F0B9
:10B588000F0293402343C0F83438B4E7D0F80838A2
:10B5980013F4807FD4F800390CBF43F0005343F014
:10B5A8008053C4F8003900920B8A0A78C9682DF0D4
:10B5B800E4FBA0E7D4F8105B04F5306305EA0C055A
:10B5C8001D611D6935401D610E698D683FBB06B15F
:10B5D8000D610D621E69C5F3120535431D611D69B4
:10B5E80045F40025012A1D6102D1CA6802B15A61D9
:10B5F8000B79012B0CD1D0F8083813F4807FD4F8DC
:10B60800003B0CBF43F0005343F08053C4F8003BA9
:10B61800D4F8003B43F00443C4F8003B6BE7002E2A
:10B62800D8D02E44013EB6FBF5F6B6B275430D628E
:10B63800074D1F6905EAC6453D431D610D6A1E6930
:10B64800C5F312053543CDE7FFFF07E00000F8FF1B
:10B658000000F81F30B5114C056C00F53063A542A9
:10B6680003D9D0F8004B002C16DB00241C611C69A0
:10B67800012944F400241C611C6944F018041C616D
:10B688001C6944F0C0441C6101BF5A61D0F8003BFA
:10B6980043F08023C0F8003B002030BD0A30544FEF
:10B6A800A8B1304BDA6802F44032B2F5403F10D10D
:10B6B8002D4B984251D92D4B984250D92C4B98423A
:10B6C80035D92C4B984216D92B4B984231D90120A9
:10B6D8007047DA6802F44032B2F5003F0DD1274BCB
:10B6E80098423AD9264B984239D9264B98421ED9C6
:10B6F800254B9842EBD803201CE0DB6803F4403369
:10B70800B3F5803F0AD1214B984226D91B4B98426A
:10B7180025D91F4B98420AD9194BEAE71D4B984285
:10B728001BD91D4B98421AD91C4B9842CFD80220DE
:10B7380000E004201A4A136823F00F030343136040
:10B74800136803F00F0398420EBF0346136803F013
:10B758000F03C01A18BF012070470020EAE7012034
:10B76800E8E700BF000802460048E8010090D0035F
:10B7780000D8B8050020A1070068890940787D0134
:10B7880080F0FA02C068780400E1F50520BCBE002C
:10B7980060343C0200127A000024F40000366E0186
:10B7A8000020024010B50A46044619B1024B002198
:10B7B8001B68984710BD00BF3406002003460020D0
:10B7C800094AC3E900009A6002F18832DA6002F19E
:10B7D8002942A2F59612A2F68B621A61A2F188326A
:10B7E8005A61024A9A61704701234567F0E1D2C362
:10B7F8002DE9F04F4B68AFB01BBA08930B69D1F82D
:10B8080000E093FA83F84B698E6893FA83FA8B69A0
:10B81800CD681BBA0A93CB6901901BBA12930B6AC5
:10B828009EFA8EFE93FA83FB4B6A36BA1BBA0B93C9
:10B838008B6A2DBA1BBA0C93CB6A1BBA0D930B6B90
:10B848001BBA0E934B6B1BBA03938B6B1BBA0493F7
:10B85800CB6B1BBA059383680F93C3680293036984
:10B868000F9906934369029F10938369109A139363
:10B87800069B83EA0200029B18405040DF4B139A54
:10B8880003EBB7071A4402EBF16210440299069AD7
:10B89800704482EAB1020F992F440A4006998EEA51
:10B8A800060E4A4010998EEA0B0E19440A4408996C
:10B8B8000A440F9902EBF0624FEAB10C02998CEA44
:10B8C800B104044084EAB1040699194431440C4493
:10B8D8008CEAB001114004EBF26481EA0C014FEAF2
:10B8E800B202394482EAB00727409C4401EBF46174
:10B8F800C44482EAB40987EAB007674409EA01093F
:10B908000AEB030C07EBF1670CEBB00C4FEAB10143
:10B918000A9889EA0209E14481EAB40C0CEA070CA6
:10B92800184410448CEAB40C129A09EBF769844461
:10B9380081EAB70000EA09001A4402EBB402484061
:10B9480010444FEAB9020CEBF96C82EAB7040BEB2E
:10B95800030904EA0C0484EAB704894404EB0901E6
:10B96800DDF82C9000EBFC6082EABC0404409944AA
:10B9780001EBF06109EBB7094FEAB0000C9F5440A6
:10B988004C4480EABC0909EA01091F44174489EAC2
:10B99800BC090D9A04EBF164B94480EAB107274069
:10B9A8001A4409EBF46902EBBC024FEAB404DDF86F
:10B9B80038C04740174484EAB10202EA09029C44AD
:10B9C800844482EAB1026244DDF80CC007EBF967EF
:10B9D80084EAB90038409C4402EBF7620CEBB10CE6
:10B9E8004FEAB70704996040604487EAB90C0CEA4B
:10B9F800020C194421448CEAB90C059C00EBF26056
:10BA08008C4487EAB20101401C4404EBB904794034
:10BA18000CEBF06C214401EBFC6903994FEAB00090
:10BA28008EEA010103EBF17E07910899BE4481EA91
:10BA380005070B9980EAB2044F40049904EA0C0404
:10BA4800794084EAB204744403EBF17E0EEBB20E43
:10BA58000C9A86EA080680EABC075640059A07EA67
:10BA6800090756404740774403EBF67E86440D9815
:10BA780085EA0A054540079804EBF96485EAF07001
:10BA88001190119D08914FEAF0704FEAB90107EB48
:10BA9800F467159081EAB400384003EBF57303EBC3
:10BAA800BC03484018440A9B4FEAF67288EA030828
:10BAB8000E9B149288EA0308089B81EABC0288EA74
:10BAC800F3730993099D4E4B224082EABC0203EBB3
:10BAD800F57C8C441299039D724402EBF7628AEA62
:10BAE80001014FEAB70787EAB409694081EAF671AC
:10BAF80089EA0209E14403EBF17C0CEBB40C0A9CE3
:10BB080000EBF26084EA0B08049C87EAB20A88EA30
:10BB18000408119C8AEA000A88EAF478E24403EBF4
:10BB2800F87C129DBC440B9F09EBF06985EA070E6F
:10BB3800059D4FEAB0008EEA050E099D4FEAF8749C
:10BB48008EEAF57E03EBFE7716944FEAFE7580EADF
:10BB5800B20407EBB2070C9A1295079D84EA090410
:10BB68008BEA02020AEBF96A644482EAF57280EA17
:10BB7800B90C04EBFA6482EAF1728CEA0A0C4FEA17
:10BB8800BA0A0A9203EBF27BBC440B9A8AEAB90719
:10BB98000D9D6740834407EB0B0082EA0507089A6E
:10BBA8000E9D87EAF27787EAF8720B9203EBF27B35
:10BBB8000C9A0BEBB90B82EA050989EAF67686EA54
:10BBC800FE760CEBF46C8AEAB4074FEAF6750D9A28
:10BBD800179587EA0C07039D5F4403EBF67BD34474
:10BBE80082EA050A119A00EBFC608AEAF2754FEACC
:10BBF800BC0C0A9A8CEAB40904E000BF9979825A0D
:10BC0800A1EBD96E85EAF27589EA000907EBF067BE
:10BC18008CEAB00AD94403EBF57B4FEAF5728AEA5D
:10BC2800070A0BEBB40B0D920AEB0B040E9ADDF826
:10BC380010A009EBF76982EA0A0A099A4FEAB707DE
:10BC48008AEAF27A0B9A04EBF9648AEAF27203EB55
:10BC5800F27B87EAB00A8AEA090AE3440C920AEB03
:10BC68000B0C039ADDF814A00CEBF46C82EA0A0AB8
:10BC78008AEAF17A8AEAF67203EBF27B039287EAA0
:10BC8800B90A049A0BEBB00B07988AEA040ADA445B
:10BC98004FEAB40B82EAF07484EAF87484EAF57423
:10BCA8008BEAB90003EBF4784FEAF47280EA0C00EF
:10BCB800B8440E9200EB0807059A08980AEBFC6A4C
:10BCC80082EAF0700C9A80EAFE7080EAF2708BEAE1
:10BCD800BC0E03EBF0784FEAF07208EBB9088EEA75
:10BCE8000A0E1192C644149ADDF81C8007EBFA6715
:10BCF80082EAF8780A9A4FEABA0A88EAF278039A46
:10BD08000EEBF76E88EAF27203EBF2798AEABC0866
:10BD1800D94488EA07080492C844159ADDF82090A7
:10BD280008EBFE6882EAF9790B9A89EAF27989EADE
:10BD3800F47203EBF27B8AEAB70989EA0E090BEB86
:10BD4800BC0B059209EB0B0C149ADDF824904FEA12
:10BD5800BE0E82EAF97989EAF67989EAF0794FEA3A
:10BD6800F97214928EEAB706159A03EBF97B86EA04
:10BD78000806D34406EB0B0A82EAF176049A86EAAF
:10BD8800F57686EAF2764FEAF67203EBF67B1592C1
:10BD98000BEBB70B169A099F0CEBF86C82EAF77756
:10BDA8000C9A8EEAB80587EAF277059A85EA0C05B7
:10BDB80087EAF27207925D4403EBF27B129A0AEB70
:10BDC800FC6A82EAF1714FEABC0C039A8CEAB80764
:10BDD800F34481EAF27187EA0A075F4481EAF97B52
:10BDE80005EBFA658CEABA0E03EBFB7101EBB801BF
:10BDF8008EEA050E169A8E440A9907EBF56782EAD1
:10BE0800F17181EAF47484EAF6744FEAF47203EB90
:10BE1800F4781692E044129ADDF82CC04FEAB50582
:10BE280082EAFC7C079A8CEAF07080EAF2700EEBEA
:10BE3800F76E85EAB70C03EBF0734FEAF07203EB89
:10BE4800BA038CEA0E0C12929C440A9A179B85EA54
:10BE5800BA0183EAF272049B794082EAF37282EAB9
:10BE6800FB730893089AE74B414401EBFE6103EB2F
:10BE7800F272154441EABE020CEBF16C01EABE080D
:10BE880002EAB70205EBFC6542EA08022A44DDF83B
:10BE98002C800D9D85EAF875DDF8148085EAF87523
:10BEA80085EAF4754CEAB108099508EABE080CEA77
:10BEB800B10548EA0505DDF8248003EBF87808EBBE
:10BEC800B70805EB0807179DDDF8308007EBF26728
:10BED80085EAF87888EAF97888EAF0784FEAF87518
:10BEE8000B9503EBF87505EBBE0E42EABC0502EABA
:10BEF800BC0905EAB10545EA09050EEBF76EAE4443
:10BF0800DDF80C900D9D85EAF97585EAF676089DB1
:10BF180047EAB20986EAF5764FEAF6750D9509EA19
:10BF2800BC0907EAB20549EA050503EBF67909EB0E
:10BF3800B1094D440E99DDF8309005EBFE6581EAB4
:10BF4800F971DDF81C9081EAF971DDF8249081EA35
:10BF5800F9710A9103EBF17101EBBC0C4EEAB701E0
:10BF68000EEAB70901EAB2010CEBF56C41EA0901E6
:10BF78006144DDF80C90DDF844C08CEAF97C8CEA69
:10BF8800FB7C8CEAF87C45EABE09CDF80CC009EACE
:10BF9800B70905EABE0C49EA0C0CDDF80C9003EB76
:10BFA800F97909EBB209CC440E9ADDF810900CEB44
:10BFB800F16C82EAF97282EAF47484EAF6744FEA60
:10BFC800F4720E9203EBF47202EBB70741EAB50282
:10BFD80001EAB50902EABE0242EA090207EBFC6778
:10BFE8001744DDF81490119A82EAF97282EAF07027
:10BFF8000A9A4CEAB10980EAF2704FEAF07211929B
:10C0080009EAB5090CEAB10249EA020203EBF07940
:10C0180009EBBE094A44DDF850E0DDF8109002EB68
:10C02800F7628EEAF97EDDF820908EEAF97EDDF877
:10C038000C908EEAF97E03EBFE7909EBB50947EA25
:10C04800BC05CDF810E005EAB10507EABC0E45EAE3
:10C058000E0509EBF269A944DDF814E0159D85EA9F
:10C06800FE75DDF824E085EAFE7585EAF475059528
:10C0780042EAB70505EABC0502EAB70E45EA0E0E24
:10C08800059D03EBF57505EBB105AE441499079DC5
:10C098000EEBF96E81EAF57181EAF87888EAF078B2
:10C0A8004FEAF871149103EBF87101EBBC0C49EA03
:10C0B800B20109EAB20501EAB70129430CEBFE6CAB
:10C0C8008C4415990EEAB90581EAFB7A04998AEA43
:10C0D800F67A8AEAF17A4FEAFA7115914EEAB901CD
:10C0E80001EAB2010D4303EBFA7101EBB701079EB8
:10C0F8000D44169905EBFC6581EAF6710A9E81EA02
:10C10800F671059E81EAF67103EBF17707EBB2074A
:10C118004CEABE02079102EAB9020CEABE010A43E0
:10C1280007EBF5671744129A05EABC0182EAFB7B24
:10C13800039A089E8BEAF27B45EABC028BEAF87BFD
:10C1480002EABE02114303EBFB7202EBB90211448F
:10C15800169A01EBF76182EAF67686EAF47686EAC1
:10C16800FA764FEAF672169203EBF67447EAB502CE
:10C1780004EBBE0402EABC0207EAB50E42EA0E026C
:10C1880004EBF1641444DDF824E0129A82EAFE72AA
:10C1980082EAF070079A41EAB70E80EAF2720C92CE
:10C1A8000C984FEAF27212920EEAB50E01EAB70243
:10C1B8004EEA020203EBF07E0EEBBC0E089802EB8F
:10C1C8000E0C0B9A0CEBF46C82EAF072049804EAF9
:10C1D800B10E82EAF07282EAFB72089203EBF27205
:10C1E80002EBB50244EAB10505EAB70545EA0E05D2
:10C1F80002EBFC622A440D98099D0CEAB40E80EA11
:10C20800F57501E0DCBC1B8F059885EAF07585EAB9
:10C21800F6704CEAB40505EAB10545EA0E0E03EBE3
:10C22800F07505EBB7050990AE44DDE90A5080EAE0
:10C23800F5750C9885EAF87585EAF0754FEAF57793
:10C24800179703EBF57707EBB10742EABC010EEB52
:10C25800F26E02EABC0801EAB40141EA080107EB00
:10C26800FE670F4403980D994EEAB20981EAF0710E
:10C27800089881EAFA7181EAF07109EABC090EEAC4
:10C28800B20803EBF1734FEAF17049EA080803EBCF
:10C29800B4030D9008EB03040A980E9B4FEABE0AFC
:10C2A80083EAF07307988AEAB20E83EAF073099872
:10C2B8008EEA070E83EAF0730A930A98DF4B04EBC1
:10C2C800F76403EBF07808EBBC081198DDF80CC0B4
:10C2D800C64480EAFC7C8CEAFB7C8CEAF57003EBB4
:10C2E800F07C0B900CEBB20C04980E9A8AEAB70813
:10C2F80082EAF07989EAF67989EAF1790EEBF46E47
:10C308004FEAF97288EA04084FEAB4040E92E0444E
:10C3180003EBF97284EAB70C52448CEA0E0C0598C8
:10C328009444119A08EBFE6882EAF0760C9A0CEBBA
:10C33800F86C86EAF2760A9A86EAF2764FEAF6729C
:10C348000C9203EBF67084EABE0200EBB70082EAB7
:10C358000802149F02444FEAB800DDF8108080EA12
:10C36800BE0A87EAF877DDF820808AEA0C0A87EAAD
:10C37800F877DDF82C8002EBFC6287EAF8774FEA61
:10C38800F777039719971F442744BA44159C059FCC
:10C398000AEBF26A84EAF774099F84EAF77484EA7C
:10C3A800F9744FEAF4740494049F1A941F4480EAC1
:10C3B800BC0407EBBE0754404FEAB20205923C4466
:10C3C800149A079F04EBFA6482EAF77888EAF5780A
:10C3D800059A88EAF6784FEAF87882EABC0508EB0D
:10C3E8000307159A074485EA0A053D4482EAFB7764
:10C3F80087EAF1770399059A4F404FEAF77782EA7F
:10C40800BA00F91801EBBC016040169A0844079974
:10C4180005EBF46582EAF1710A9A4FEAB40481EAFD
:10C42800F271049A84EABA0E51404FEAF171059A02
:10C4380001EB030C94448EEA050E129AE644DDF8EB
:10C448002CC082EAFB7282EAFC7282EA08024FEA96
:10C45800F27200EBF56084EAB50C02EB030B0BEB10
:10C46800BA0B8CEA000CDDF858A0DC44DDF820B0EB
:10C478000EEBF06E8AEAFB7A8AEAF97A8AEA070A08
:10C488004FEAB0004FEAFA79CDF81490CDF87C90D5
:10C4980080EAB50A9944A1448AEA0E0A129CCA4461
:10C4A800DDF824900CEBFE6C84EAF97484EAF674E7
:10C4B8004C404FEAF4740794209480EABE061C446A
:10C4C80004EBB50486EA0C062644179C039D84EA0F
:10C4D800FB746C4054400AEBFC6A4FEAF4744FEA70
:10C4E800BC0C8CEABE09E518054489EA0A09CDF8AE
:10C4F8006C801C971D911E92A9442194099D0D984A
:10C5080006EBFA6680EAF570049D09EBF669684067
:10C51800059D68404FEAF0708CEABA0500EB030B02
:10C528000BEBBE0B7540DDF85CE05D44DDF828B030
:10C538004FEAB6068EEAFB7E8EEA080EDDF81C800E
:10C5480005EBF9658EEA080E4FEAFE7E0EEB030B4B
:10C5580086EABA08E34488EA0908DDF834C0D84412
:10C56800DDF82CB008EBF5688CEAFB7C8CEA070C4C
:10C578008CEA040C4FEAFC7786EAB90407EB030C53
:10C588000CEBBA0C6C40DDF828A06444DDF838C028
:10C598004FEAB5058CEAFA7C8CEA010C8CEA000CAF
:10C5A8004FEAFC7101EB030CB4440C9E229086EA1E
:10C5B800FB76564086EA0E0685EAB9004FEAF6761B
:10C5C80004EBF864269685EAB80280EA08001E445F
:10C5D80006EBB9066044624000EBF460324402EBBB
:10C5E800F06C039E0E9A4FEAB4045640059A2497BD
:10C5F80056407E404FEAF67627961E440C9A2E4403
:10C60800049D84EAB8075540079A474055404D4075
:10C618004FEAB00018954FEAF5752591289584EAF8
:10C6280000011D4481EA0C01374405EBB80507EB0E
:10C63800FC674B190F994FEABC0201E0D6C162CAE8
:10C6480003EBF763CDF88CE02D942A972C9029936F
:10C658002B920B4401998B60029B1F44069BCF6071
:10C668001A44109B0A611844139B48611C448C614E
:10C6780018A85821FFF796F800202FB0BDE8F08FD2
:10C6880003460846C1B9C3E910110D4A0D49DFF840
:10C6980038C0C3E912120D4A0D49C3E914C20D4A44
:10C6A800C3E916120C4A1A6602F17452A2F5230263
:10C6B800A2F692425A6670476FF07300704700BF47
:10C6C80085AE67BB67E6096A72F36E3C3AF54FA51B
:10C6D8007F520E518C68059BABD9831F2DE9F04F13
:10C6E8000446CFB0039100F1480346AD00F1680657
:10C6F8002A4618685968083303C2B3421546F7D169
:10C70800DDE94883DDE94B96DDE946154FF0000C7D
:10C7180001933E4BDDF834B14A9804AA0293BCF168
:10C728000F0F5BD8039B53F82C301BBA4FEAF02E3F
:10C7380086EA0907DDF808A08EEAB01E07408EEAEF
:10C74800706E774077445AF804EB936077443B4423
:10C7580045EA010E4FEA7137CDF808A087EAB1071C
:10C768000EEA080E05EA010A4EEA0A0E87EAB157F0
:10C7780077440CF1010CDDF804E05B44BCF1400F98
:10C788009E44B3463B4402F10402CDF804801ED116
:10C79800CDE94C96CDE94AE0CDE94858CDE9463196
:10C7A800CDE9043745A904F14403643453F8042F50
:10C7B80051F8040FA34202441A60F7D104A84FF4B9
:10C7C8009471FEF7EFFF00204FB0BDE8F08FA84648
:10C7D8004E460D46814619467046A0E7136852F842
:10C7E80034AC4FEAF34E8EEA734E52F8387C8EEA38
:10C7F800932E52F8143C3B444FEABA4787EAFA179B
:10C80800734487EADA073B4490E700BF74B804082A
:10C8180010B50446F6F792FA03480121034A29F0B5
:10C8280023F820462CF0CEFC54B10408687605089D
:10C838002DE9F84304460D4600AFEFF311881023A5
:10C8480083F31288BFF36F8F0428294A98BF294BB6
:10C85800E9468AB09668117C98BF53F820306A463A
:10C8680088BF254BC2E9073140F20133234893843E
:10C87800234BC2E9050442F8103F00234FF431511D
:10C888002048F6F72BFBCD4645B1EB69C3F3080307
:10C8980023B101211C4A1B4828F0E6FF2EB130467F
:10C8A8002CF017FF08B1037803B91848E9468AB095
:10C8B8006A46174BD061C2E9053640F2013313844A
:10C8C800144B42F8103F00234FF411510D48F6F76E
:10C8D80005FB2946CD462046FFF79AFF88F31188C5
:10C8E800BFF36F8F3046F7F7E1F9BD46BDE8F8832F
:10C8F8004C37002074B90408777605088D7605084A
:10C908000500000154B10408B576050885760508C8
:10C91800D67605080400000138B50A4B53F82040C4
:10C92800013053F82050A54200D838BD606830B1B6
:10C93800037EDB0701D42CF022FC0834F3E72368DC
:10C948009847FAE788B90408012270B5294B0320F3
:10C9580086B01A70FFF7E0FF01F028FC0420FFF70B
:10C96800DBFF254C254D2646AE4204F1300410D39A
:10C9780000F072FF204C224EAC4226D300F080FF1C
:10C9880027F0E1FF1F4A938923F00103938106B042
:10C9980070BD54F80C3C059354F8103C049354F8BB
:10C9A800143C039354F8183C029354F81C3C01932C
:10C9B80054F8203C009354E90A2354E90C0100F090
:10C9C80035FD54F8303C5E65CDE7D4E90A23B3F170
:10C9D800FF3F08BFB2F1FF3F05D052EA03012068CC
:10C9E80003D101F01FF83034C6E73146183001F0A2
:10C9F800C5F9F8E73E3F002050AF040880AF0408AF
:10CA0800BB970308302E0020A02370B5134E0122D7
:10CA180003FB0066002386B0CDE904230F220193AF
:10CA2800CDE9023214234FF4A0720D4D0D4903FBDA
:10CA38000055044602FB00110B4B3046009500F0F0
:10CA4800F5FC337C2C7423F004033374074B013456
:10CA580003EBC423EE606B6006B070BD902D002020
:10CA68004C370020C05E002055930308C0560020B4
:10CA7800BFB50020FFF750FF294B03F5006282F392
:10CA8800088883F30A880024F023264D264F85F86A
:10CA98002230EC772C766C76AC7685F820406B6A81
:10CAA80043F4E0236B62F7F7BBF8F7F707FA4FF0A8
:10CAB800FF33AB62EB62F7F7ABFBF7F729FAF6F750
:10CAC800A3F81A4800F034FDF5F750FF0120FFF7EE
:10CAD80023FF0220164DFFF71FFF00F005FF154B3F
:10CAE80015495D61154B45F6E0620593012328461B
:10CAF800CDE90343CDE901443B46009400F096FCA0
:10CB080006462A7C284622F004022A742CF01DFED0
:10CB18002046FFF779FF3A4631462846F7F7ACF941
:10CB2800C056002000ED00E051C90008D02E0020BA
:10CB3800302E00204C37002000600020D45B050810
:10CB480038B5064C064DAC4201D3002038BD20460E
:10CB5800D4E901122CF080FB1434F4E7AC0F002068
:10CB6800C00F002030B5054B85B0DDE908450293BC
:10CB7800CDE900452CF02EFB05B030BD234E03084F
:10CB8800002038B5054C064DAC4200D338BD2046D0
:10CB98002CF086FB0028F9DB1C34F5E7900F002009
:10CBA800AC0F002073B50C46EFF31181102585F307
:10CBB8001288BFF36F8FC5685DB125602B68C360AD
:10CBC800836901338361002081F31188BFF36F8F7C
:10CBD80011E052EA030603D16FF00B002560F3E77A
:10CBE800CDE900230246083000F07CFD18B9034B5C
:10CBF8009B685B69236002B070BD00BF4C370020A2
:10CC08002DE9F34104460E469DF8200004F108087A
:10CC1800EFF31187102181F31288BFF36F8F256A14
:10CC2800E1688D4247D22568AC4218D0BDB128468C
:10CC38002CF097FB05F118002CF086FE3146A2680F
:10CC480068693DF062FE00232846C5F898302CF04C
:10CC58007CFD4046394600F0D9FD002038E0A26846
:10CC6800D8B13146E0693DF050FEE369A26813444B
:10CC78006269E361934201D12369E361236A102168
:10CC88000133236204F124002CF03DFF0028E0D199
:10CC980087F31188BFF36F8F1AE0A169236999425E
:10CCA80008BF6369314608BFA361A069801AA06103
:10CCB8003DF02BFEE2E752EA03010CD0074940465B
:10CCC80089684E61CDE900233946224600F00AFD05
:10CCD80002B0BDE8F0816FF02200D9E74C370020A0
:10CCE800F7B50446084604F10807EFF3118610214A
:10CCF80081F31288BFF36F8F216A00293AD0A268A6
:10CD0800A1693DF002FEA369A2682568134462691F
:10CD1800A361934204BF2369A361236AAC4203F170
:10CD2800FF33236234D02846002D32D02CF019FB73
:10CD380005F118002CF008FEA2686969E0693DF069
:10CD4800E4FDE369A268284613446269E3619342FB
:10CD580004BF2369E361236A013323620024C5F811
:10CD680098402CF0F2FC3846314600F04FFD204642
:10CD780003B0F0BD52EA030110D00A49896848613E
:10CD8800CDE9002331462246384600F0ABFCEFE7F8
:10CD9800002086F31188BFF36F8FE9E76FF0220058
:10CDA800F7E700BF4C3700202DE9F341044617464A
:10CDB8001E46EFF31188102383F31288BFF36F8F99
:10CDC800C368314A7BB180689168884219D057EAB4
:10CDD800060318D188F31188BFF36F8F6FF00F0027
:10CDE80002B0BDE8F081916891F90E100133E3605B
:10CDF80093682161A36088F31188BFF36F8F0020C7
:10CE0800EEE72169F2E790F90E3091F90E10994298
:10CE1800A8BF19468B422DDD2CF00DFB0546224696
:10CE28004146CDE90076194800F05CFC0028E6D0C0
:10CE3800EFF31186102383F31288BFF36F8FA06876
:10CE4800D0B1236821699C420AD04BB193F90E30C6
:10CE58009942A8BF19466FF07F039942B8BF194697
:10CE68002CF0E9FA40B13146084800F0CFFC6FF0E9
:10CE78000A00B5E70025D2E7002DF4D186F3118822
:10CE8800BFF36F8FF3E700BF4C3700203F3F002010
:10CE9800F8B583680546002B40D0234A9268934230
:10CEA8003FD1C368012B03D9013BC3600020F8BD03
:10CEB800EFF31187102383F31288BFF36F8F016993
:10CEC80080682CF0B8FA2C68AC4207D10023C5E979
:10CED800023387F31188BFF36F8FE7E7002CF5D093
:10CEE800D4E90032002613605A60237CC4E9006646
:10CEF80023F002032374A66004F118002CF024FD2B
:10CF0800AC6094F90E3020462B61C4F898602CF080
:10CF18001CFC3946054800F079FCC7E76FF015009E
:10CF2800C5E74FF0FF30C2E74C3700203F3F0020F5
:10CF380037B51146EFF31185102282F31288BFF33B
:10CF48006F8F04689CB12368426823F003039442FE
:10CF5800036008BF4360012120462CF0F9FA04461B
:10CF680085F31188BFF36F8F204603B030BD51EAB7
:10CF78000302F5D000F10802CDE900131046294656
:10CF880000F0B0FB0028EFD1014B9B685C69EBE730
:10CF98004C37002070B5EFF31186102383F3128805
:10CFA800BFF36F8F0468A0421BD0D4B1D4E900321C
:10CFB800002513605A60237CC4E9005523F002035E
:10CFC8002374A56004F118002CF0BEFC2046C4F8B8
:10CFD80098502CF0BAFB3146BDE87040094800F083
:10CFE80015BCD0E902329A4218BF0133022183608E
:10CFF80010302CF088FD0028EDD186F31188BFF39E
:10D008006F8F70BD3F3F002013B5EFF311811024DF
:10D0180084F31288BFF36F8F846844B1013C846045
:10D0280081F31188BFF36F8F002002B010BD52EA60
:10D03800030406D181F31188BFF36F8F6FF00F00DF
:10D04800F3E7CDE900230246014800F04BFBECE78B
:10D058003F3F00202DE9F8430546EFF311881023E0
:10D0680083F31288BFF36F8F00266FF00A093746E3
:10D078002C68A54216D0ACB1D4E9003213605A60CE
:10D08800237CC4E9007723F002032374A76004F12A
:10D0980018002CF059FC2046C4F898902CF055FB49
:10D0A8000126E5E700230221AB6005F110002CF012
:10D0B8002AFD30B92EB988F31188BFF36F8FBDE808
:10D0C800F8834146BDE8F843014800F09FBB00BF24
:10D0D8003F3F00202DE9FF41044610274E4EEFF355
:10D0E800118887F31288BFF36F8FD4F8A450F5B96D
:10D0F800022104F1BC002CF06CFA002868D004F17D
:10D10800B4050022012128462CF0B3FB0028F8D1F1
:10D1180000234FF0FF3202934FF0FF334146CDE931
:10D1280000233E4804F1AC0200F048FDD7E7D4F8EC
:10D13800A8202B689542C4F8A43008BFC4F8A830CA
:10D14800D4F8BC3043F00203C4F8BC30EB6823F0D9
:10D15800040343F00103EB606B6888F31188BFF3A5
:10D168006F8F28469847EFF3118887F31288BFF32B
:10D178006F8FEB68D80623F0010236D4EA60EB68BB
:10D188009A0716D5306823F00203EB6088B10021B6
:10D19800036870B14268954235D1036869BB72680B
:10D1A8003360824200D17360002340F8083BFFF7E8
:10D1B800F1FED4F8BC3023F00203C4F8BC3088F385
:10D1C8001188BFF36F8FDB0589D400F0ABFB86E7CE
:10D1D800D4F8BC30D9069BD5C4F8BC0088F31188B4
:10D1E800BFF36F8F04B0BDE8F08123F01103EB604B
:10D1F80005F11000FFF7CEFEC1E70B6073688342AC
:10D2080008BF7160D0E723B11A6801461846134673
:10D21800BFE71A46F9E700BF703700203F3F0020FC
:10D22800F8B5C36804469A070F46C3F340062ED4E0
:10D238005B071CD40B680BB983680B60E368DD07D8
:10D2480042BFA36802263B603D6858BF0126002DF7
:10D258003CD0204B9A68D5F8A0309A420AD0D5F82D
:10D26800BC30D807C3F3800214D46FF01206002331
:10D278003B6025E02CF024FAD5F8BC300028F0D12A
:10D28800D907C3F3C002F0D552B15B0708D46FF0D9
:10D298000F06ECE7002AFAD1C3F3C003002BF6D13E
:10D2A80000232360D5F8A83063B9C5E92944284686
:10D2B8002CF0A9F9E36843F00403E3603B68A3603A
:10D2C8003046F8BD1C60C5F8A840F0E76FF01506B9
:10D2D800CDE700BF4C370020014601482CF0D4B9F7
:10D2E800902F0020F0B50446002089B0C4E9290039
:10D2F8000E9D04F1AC00C4E92B0004F1B400C4E9AC
:10D308002D0055B32879002840F2011008BF0120EC
:10D31800C4F8BC0000204FF0FF364FF0FF37CDE9CE
:10D328000330CDE90100CDE9066720460C4B009497
:10D3380000F0D2F855B1296811B120462CF0C6F991
:10D348006B791BB1A38943F00103A381204600F048
:10D3580069FBC4F8A04009B0F0BD0120D8E700BFC0
:10D36800DDD0000837B501900846EFF3118410218D
:10D3780081F31288BFF36F8FC16811F01E0F16D1A9
:10D3880053EA020508D101A9FFF74AFF84F311887F
:10D39800BFF36F8F03B030BD41F00801C160019940
:10D3A80010308161034900F0E9FC0120EEE700201C
:10D3B800ECE700BF1D96030801460148FFF7D2BFFE
:10D3C800902F0020F7B50C4616461D460190EFF346
:10D3D8001187102383F31288BFF36F8F08462CF050
:10D3E80003F955EA060309D1204601A9FFF718FFFA
:10D3F80087F31188BFF36F8F03B0F0BDE36832463F
:10D4080043F00803E360019B0449A36204F11000A0
:10D418002B4600F0B3FC0120EAE700BF1D96030885
:10D4280001460148FFF7CEBF902F00202DE9F04FAD
:10D43800984685B000F15803C0E91633129B0026C0
:10D4480083810423073222F0070A0374119B01EB3E
:10D458000A090F46C0E90666494686608373C673A3
:10D468000446DDF838B0F6F795F9109BC51D25F090
:10D478000705C4F88850C4E9207A02930F9BA9EBEA
:10D488000505CDE900B32A46434639462046F6F756
:10D49800D7FC0F9BC4E91B8B6367109B6665A3676A
:10D4A800EFF31182102383F31288BFF36F8F094BB8
:10D4B800196A1C62E16782F31188BFF36F8F9B685A
:10D4C8000BB1D3F88C302846C4F88C3005B0BDE8D1
:10D4D800F08F00BF4C370020F0B5002587B00595C8
:10D4E800109DDDE9127604950F9D044603950E9D67
:10D4F80002950D9D01950C9D0095FFF797FFB6F1DC
:10D50800FF3F08BFB7F1FF3F05D056EA070305D133
:10D51800204600F087FA204607B0F0BD3A46334669
:10D5280004F11800014900F029FCF4E7BB9703084F
:10D538000123037483810023C0E92033C0F88C30B1
:10D54800014B9860704700BF4C3700206FF00A010C
:10D55800094A9368C3F898100849C3F894004B68BF
:10D5680043F080534B60002383F31188BFF36F8F20
:10D578009368D3F8980070474C37002000ED00E01E
:10D5880070B590F91020037C002A36DBD90634D117
:10D598001B4C63F07F032246037452F8183FE1697D
:10D5A800934207D1C0E900210860E06111E0994287
:10D5B800F8D01B68002BF5D090F90E5093F90E6047
:10D5C800B542F4D0AE42F2DD5968C0E900310860D6
:10D5D8005860A569954200D005B9E568A3681A7C2A
:10D5E800D20604D1DA897F2A01D9AA6932B1AB42BD
:10D5F80002D0284600F024FB656170BD6361FCE73A
:10D608004C37002038B590F910200146002A037CD9
:10D6180004DA03F07F0303742CF05DF80D4D2A46FD
:10D6280052F8184FAB68944200D004B9EC688B42AA
:10D6380007D01A7CD20604D1DA897F2A01D9A269D7
:10D648002AB1A34202D0204600F0FAFA23466B61C1
:10D6580038BD00BF4C370020B3F1FF3F08BFB2F11F
:10D66800FF3F03D00249183000F088BB704700BF65
:10D67800BB97030838B5194CA168E0690B6881426B
:10D6880014BF1A46002249680B605960A368E16913
:10D698002AB9134AC3E900210B60E3610CE093F94E
:10D6A8000E0092F90E50A84214D0854212DD51683E
:10D6B800C3E900210B605360A569094B9D4200D066
:10D6C80005B9E568A3689D4202D0284600F0B8FA7B
:10D6D800656138BD9142DCD01268D9E74C3700202B
:10D6E80064370020F8B5DDE906670D4B0C469868ED
:10D6F80011460C4A1060EFF31182102282F312884F
:10D70800BFF36F8F9D6828462BF0F7FF28463246F7
:10D718003B46FFF7A1FF2046BDE8F840FFF716BFDC
:10D728004C37002078370020F8B50446EFF311870E
:10D73800102383F31288BFF36F8F037C49B203F081
:10D748001F02002A0CBF0126002639D103F07F03EF
:10D758002D4D03742BF0BFFF2A46037C817363F0C1
:10D768007F03037452F8183F934227D1E869C4E94C
:10D7780000200460EC610FE09842F8D01B68002B91
:10D78800F5D093F90EC06145F6D08C45F4DD5968A3
:10D79800C4E900310C605C60AC69944200D004B903
:10D7A800EC68AB689C4202D0204600F049FA6C61F4
:10D7B80087F31188BFF36F8F3046F8BDE869DEE75D
:10D7C8009B071ED585682BF086FF81732B689D42C9
:10D7D80009D16B68C4E900531C606C60E8E76A68AB
:10D7E8009342F6D01B68002BF3D093F90E20914298
:10D7F800F5D08A42F3DD5A68C4E9003214605C60EF
:10D80800D6E78173D4E700BF4C37002049B9EFF35E
:10D81800058030B9054B5A699B689A4201D0FFF7D9
:10D8280095BE81F31188BFF36F8F70474C37002086
:10D83800034648B9EFF3058232B9064A516992683E
:10D84800914201D0FFF782BE83F31188BFF36F8F37
:10D85800704700BF4C370020EFF31181102383F38A
:10D868001288BFF36F8F054B9A68D37B013BD37344
:10D8780081F31188BFF36F8F704700BF4C370020CA
:10D8880070B5EFF31186102383F31288BFF36F8FFF
:10D89800144DAB68DA7B0132DA732A4652F8184F16
:10D8A800944200D004B9EC681A7CD20604D1DA8913
:10D8B8007F2A01D9A2692AB1A34202D0204600F0EA
:10D8C800BFF923466B6186F31188BFF36F8FEFF3BF
:10D8D8001180102383F31288BFF36F8FBDE8704067
:10D8E800FFF7A6BF4C370020024B03F11802C3E92B
:10D8F800062270474C37002008B5FFF715FF70B1B6
:10D90800074B9B68DB7B53B9EFF31180102383F33C
:10D918001288BFF36F8FBDE80840FFF789BF08BDC5
:10D928004C37002070B5EFF31186102383F312886B
:10D93800BFF36F8F1B4CA168E0690B68814214BF6D
:10D948001A46002249680B605960A368E1692AB940
:10D95800154AC3E900210B60E3610CE093F90E005E
:10D9680092F90E50A84218D0854216DD5168C3E9D5
:10D9780000210B605360A5690B4B9D4200D005B98F
:10D98800E568A3689D4202D0284600F059F9656110
:10D998003046BDE87040FFF7D9BD8A42D8D012683A
:10D9A800D5E700BF4C37002064370020F8B550EAAF
:10D9B800010306460C4603D1FFF7B4FF0020F8BD6B
:10D9C800EFF31187102383F31288BFF36F8F124D83
:10D9D800124BA8681860FFF715FEA8682346324660
:10D9E8000F49183000F0CAF9AA680446137C384673
:10D9F80043F004031374FFF7A9FDAB68D3E90A23C6
:10DA0800B3F1004F08BF002AD8D12BF0C5FF201A68
:10DA180020EAE070D3E700BF4C37002078370020B9
:10DA2800BB97030838B50446EFF31185102383F339
:10DA38001288BFF36F8F037C5B070FD518302BF06C
:10DA480083FF237C204623F004032374FFF798FD0B
:10DA58002946BDE838400448FFF7D8BE85F3118849
:10DA6800BFF36F8F38BD00BF3F3F0020014B986860
:10DA7800704700BF4C3700202DE9F84304468789DA
:10DA8800EFF31185102383F31288BFF36F8F037CA4
:10DA9800190705D585F31188BFF36F8FBDE8F883A3
:10DAA800D90943F0080260D10274A36813B1204673
:10DAB8002BF019FE04F118002BF046FFA66D04F1B7
:10DAC8005808B04511D04FF0000976B130462BF018
:10DAD8000AFE06F118002BF037FF3046C6F898907A
:10DAE800FFF74EFDA66DB045EFD1DFF8C480D8F83A
:10DAF80008309C4241D1EFF30589B9F1000918BFFC
:10DB08004FF00109D8F818602A4A964200D00EB999
:10DB1800D8F80C60B34202D0304600F091F82046A5
:10DB2800C8F8146028F055F8204600F0DBF8B9F181
:10DB3800000F02D02048FFF7FBFCD8F808309C42C1
:10DB480031D1EFF3058373BBA289D20718D42846D5
:10DB5800FFF7FCFCFB07A1D5002383F31188BFF373
:10DB68006F8F0423184602DF98E703F07F0343F022
:10DB7800080303742BF0AFFD97E74FF00009C1E7E6
:10DB880085F31188BFF36F8F83F31188BFF36F8F0D
:10DB98000423184602DFEFF31180102383F3128861
:10DBA800BFF36F8FD4E785F31188BFF36F8FD1E789
:10DBB8004C37002064370020D02E0020D3B5DDE993
:10DBC8000667089CCDE90067FFF78CFD1CB1034B85
:10DBD8009B685B69236002B0D0BD00BF4C37002052
:10DBE800027C034612F01F0210D10A4988420DD068
:10DBF8000949086868B1D9897F2909D893F90E209D
:10DC0800064B1B689A42B8BF002070470020704737
:10DC180010467047902D0020380600207C370020E1
:10DC28000122044BC01A044BC0105843034B1A542A
:10DC3800704700BF702F0020ABAAAAAA3F3F002060
:10DC480070B50D4B0D4D1E7CFFF7CAFF06EB460362
:10DC580005EBC305044628462BF076FE0022084B48
:10DC68009A553CB1621E2846BDE870400549D31755
:10DC780000F084B870BD00BF4C370020702F002022
:10DC88003F3F002029DC000838B5EFF31185102349
:10DC980083F31288BFF36F8F0F4B104A9C6810688C
:10DCA800A04206D1FFF7CCFF85F31188BFF36F8F31
:10DCB80038BD00211B7C1160094AD35C002BF3D0CE
:10DCC8002046FFF78DFF0028EED0237CDB0601D12C
:10DCD800FFF7D0FC2046E5E74C37002078370020D6
:10DCE8003F3F0020EFF31181102383F31288BFF325
:10DCF8006F8F0A4A136A834207D1DB6F136281F37D
:10DD08001188BFF36F8F70471346002BF7D0DA6F77
:10DD18008242F9D1C26FDA67F1E700BF4C370020C1
:10DD2800024B1868984208BF002070473C06002044
:10DD3800034B1B680BB9FCF757BD0020704700BFA9
:10DD48008037002030B570B10B4B5B6898420AD021
:10DD5800036843B1D3E90421D0E90445121941EB22
:10DD68000501C3E90421D0E9003213605A60002399
:10DD7800C0E9003330BD00BF3C060020B3F1FF3FCF
:10DD880008BFB2F1FF3F2DE9F84F04469946154602
:10DD98001F467AD08160EFF31188102383F312882D
:10DDA800BFF36F8FB9F1000FDFF8E4A020DBFFF7B6
:10DDB800BFFFDAE90027013549F100092D1849EBC1
:10DDC800E07306464FF00109C4E90453AD1843EB6C
:10DDD8000707FFF7A5FF0346DFF8B8E0DEF804A061
:10DDE800EBB9C4E900EACAF80040CEF8044028E0DC
:10DDF8006FF00103DAE900125B1A4FF0FF3161EBB3
:10DE080002025B1B62EB0902012B72F10001BCBF2D
:10DE1800012300224FF00009C0E90432D9E7D3E911
:10DE2800041CD4E904208A4270EB0C0B24DA891A0A
:10DE38005A686CEB0000C3E90410C4E900321460AE
:10DE48005C60FFF76DFF84420ED1134B1B685BB912
:10DE5800B9F1000F02D1FFF76BFF064630462BF0F1
:10DE68005CFD0021FCF742FC88F31188BFF36F8F3B
:10DE780028463946BDE8F88F521A60EB0C009A45DF
:10DE8800C4E90420ADD01B68AAE700252F46EFE7B8
:10DE9800882F00203C060020803700202DE9F0471D
:10DEA800EFF31185102383F31288BFF36F8FDFF828
:10DEB800A0900026C9F800000027FFF731FFDFF81F
:10DEC8009480D9F80030D8E900ECD91750B1D0E9DE
:10DED8000442A34271EB020A1BDAE41A62EB010264
:10DEE800C0E90442002413EB0E034CEB0101204669
:10DEF800C8E90031C9F800402BF00FFD2146FCF7B6
:10DF0800F5FB85F31188BFF36F8FBDE8F047FFF786
:10DF1800BBBE14EB0E024CEBE473C0E90467C8E91E
:10DF28000023FFF70FFF85F31188BFF36F8F836816
:10DF38009847EFF31185102383F31288BFF36F8F8F
:10DF4800D9F800301B1BC9F80030FFF7E9FEB8E725
:10DF580080370020882F002010B5EFF3118410239C
:10DF680083F31288BFF36F8FFFF7E2FE0346054A7B
:10DF7800D2E90001181841EBE37184F31188BFF36B
:10DF88006F8F10BD882F0020F8B50646EFF3118774
:10DF9800102383F31288BFF36F8F026822B187F3CF
:10DFA8001188BFF36F8FF8BDD0E90A54691C44F19A
:10DFB8000003022973F1000334D3013D44F1FF3417
:10DFC800002CBCBF15462C462BF0EAFC013041F171
:10DFD8000001401944EB0101012871F100014ADBFD
:10DFE8002BF0DEFC6FF00203013041F10001401913
:10DFF80044EB010183426FF000438B4140DB2BF07F
:10E00800CFFC6FF001024FF0FF33013041F1000106
:10E01800401944EB0104121A63EB040330461A4911
:10E02800FFF7ACFE336B01333363336A6BB187F3AD
:10E038001188BFF36F8F3046336A9847EFF3118723
:10E04800102383F31288BFF36F8F334653F8184FAA
:10E058009C42A4D0002CA2D020462BF085FB0023A4
:10E06800C4F8983087F31188BFF36F8F2046BDE856
:10E07800F8402BF06ABB6FF001024FF0FF33CDE799
:10E0880000224FF00043C9E791DF00082DE9F04175
:10E0980005461C4690461F46EFF31186102383F36E
:10E0A8001288BFF36F8FB4F1FF3F08BFB2F1FF3F93
:10E0B80005D186F31188BFF36F8FBDE8F081002C7E
:10E0C80009DB012A74F10003BCBF0122002412F10C
:10E0D800FF3844F1FF3728462BF036FCDDE906010E
:10E0E8000023C5E90A012B6342463B4628460249FC
:10E0F800FFF744FEDDE700BF91DF000838B50346AF
:10E10800EFF31185102282F31288BFF36F8FC1607D
:10E11800012181600068834206D185F31188BFF32D
:10E128006F8F0024204638BDD0E9003213605A6052
:10E138000023C0E900332BF0A3FC2946044602481B
:10E14800FFF764FBEEE700BF403F0020F8B5074645
:10E158000C4616462BF0B4FA08B10020F8BD0E4B59
:10E168009B68D3F88C50002DF7D0221DF5D2EFF321
:10E178001184102383F31288BFF36F8F284647F06A
:10E188000401B04784F31188BFF36F8F0028E4D0EF
:10E1980040F8045BE2E700BF4C3700200146024A22
:10E1A8000020FFF7D3BF00BF1D4E0308014826F02B
:10E1B80098BF00BF3877050807B5074B4FF4806252
:10E1C800009306494FF0FF330548FFF78BF800200E
:10E1D80003B05DF804FB00BFA0B90408E0BE00204E
:10E1E800902F0020F0B5042804468BB02BD0344D76
:10E1F800286818B113F0ECF800232B601CB3314BDE
:10E208009C4220D0002601AB02932F4B214602A846
:10E21800039301962FF019FE01983146013013F04F
:10E22800B7F80246286070B106AF3846019932F057
:10E238007FF8264B214604A8059304972FF005FE86
:10E248002A68019BD65402F0D9FC32F0F5F92BF07C
:10E25800AFFD01F059FC00221D4D1E4BD5F8F040D2
:10E268001A7084B1204611F0CBFF30B3A06804F0D7
:10E2780093FBD5F8F040002CF4D1D5F8F0301C46CB
:10E28800DB68002BFBD1C5F8EC400025124C02F0EE
:10E2980061F804F039FC12F0A5F8206813F098F83A
:10E2A80025600E4C206813F093F825602BF086FC4F
:10E2B8000BB0BDE8F0402BF006BDE468DBE700BF1B
:10E2C800DC38002070390020759B0308B10204086F
:10E2D800F8380020403F0020C0370020BC3700201D
:10E2E800002270B50446154B00EB8105C3E90022F6
:10E2F8009A60264630682DF0FAFA022804F10404E0
:10E3080018D130680E4C206098B10E482BF031FFC0
:10E3180020682BF07BFC0C4802F018F901F03AFC5D
:10E32800064920682BF06DFC0023236001F032FCC5
:10E33800012070BDA542DCD10020E3E7883700202A
:10E34800B8370020C07805084DCD050810B504463B
:10E3580008482BF05BFC01F077FD40B1064802F05D
:10E36800F5F834B1BDE81040044802F0EFB80448AD
:10E37800F5E710BDC07805083CCB05081FC60508A1
:10E3880069CB050873B506462BF09DFC0CF024FFFD
:10E3980012F00AFF054612F013FF0446641B00251D
:10E3A8000CF022FFA4F580600CF024FF01F0ACFB18
:10E3B80000F05CFC6B464FF4006230461F49009544
:10E3C8002BF0D8FB01461E4B1E4C1860009B1944CD
:10E3D80005F030F84FF4005201AB30461A49019568
:10E3E8002BF0C8FB0146194B1860019B194411F02A
:10E3F800D9FE06F02BFC2946D4F8E8000DF078FE8B
:10E408001621D4F8E80030F056F96621D4F8E8006F
:10E4180030F051F940F6B651D4F8E80030F04BF935
:10E42800294604F1D8000DF063FE094804F02AF8E3
:10E438000122084B1A7002B070BD00BF6F77050843
:10E44800BC370020F838002086770508C037002040
:10E45800955C0508403F00202DE9F047092804464F
:10E46800A4B000F08F8001F069FB00287FD0002C59
:10E478007DD1464BD3F8F030002B78D0204602AD42
:10E48800DFF80C81FFF77EFF2BF07DFE01F0ECFB3F
:10E498004FF40071284631F030FFC8F8005001F001
:10E4A80055FB0121064600F180072BF03AFC394B59
:10E4B800394A3A493A482FF024FE06A800F040FBB2
:10E4C800384937482FF042FEDFF8DCA0DFF8D0905B
:10E4D80006AD5146484615F8012B01342FF036FE9B
:10E4E800202CF6D131492E482FF00BFE32F0A5F83A
:10E4F80002212F48FFF7F4FE0023C8F8003001F08E
:10E50800B9FB012338462B4A0EA933F02EF8A0B9DF
:10E5180002982DF08CFA039A0446014601AB0132A9
:10E528000EA833F047F940B9039A019B9A4204D1E7
:10E53800214604983CF018FAA0B14FF47A702BF0F9
:10E548004CFE0A231B4A0EA9384633F00EF8DDE9C3
:10E55800032101AB0EA833F0DFF90EA833F045FB19
:10E5680001F0D2FA002130462BF0DBFB04E0204614
:10E57800FFF708FF2BF007FE0F4C6068FFF732FE2D
:10E588000023636024B0BDE8F08700BFF83800209E
:10E5980084370020A0770508B377050801780508B7
:10E5A800E8E104080FC505083BCD0508BDB7050817
:10E5B800DCB9040811780508883700202DE9F04FE8
:10E5C80089B007462BF0AEFD804640B1B1482BF02C
:10E5D800D0FD3846FFF7BAFE384601F037F9DFF8C4
:10E5E800B892CDF80880002F40D0D9F80030B3F5A4
:10E5F800007F40F0D780002520262C464FF00209E6
:10E608004FF4401B2BF0E5FD4FF4C87303FB09F3EF
:10E61800049303F59C53083303900093002C40F0B7
:10E628007681A2464FF0010901F062FE01F030FC4C
:10E6380005460190002800F0BD8046F0100601F064
:10E64800DBFB964C206828B103781E4002D112F0FB
:10E65800BFFE2660BAF1000F04D0002001F028FBAD
:10E6680001F020FB284609B0BDE8F08F01F04CFA14
:10E6780001F02CFC0546002840F08680874EFFF705
:10E6880081FE2BF082FD3368002B5CD01A7822F0D3
:10E6980020021A7033689A681C78127892B1586808
:10E6A80008B103F0EFFE336801219B6807A80793C0
:10E6B800FFF716FE98B9336898682BF05AFD78482A
:10E6C80001F044FF04217748FFF70AFE38B9082112
:10E6D8007548FFF705FE10B1744801F037FFD9F807
:10E6E80000301B0531D501F00DF801282DD17048F7
:10E6F8004FF0000A01F02AFF6E4BD9F8040083F8A6
:10E7080000A0FFF76FFD3268C9F804A02AB113789A
:10E71800980644BF43F020031370D9F80030190558
:10E7280015D500F0EFFF441E18BF01243026D9F894
:10E738000030DA051BD5B3F5007F4FF001043FF434
:10E748005DAFA1462BE03C46BCE75B48D0E71BB970
:10E75800242604F00104EAE714F0020418BF83F445
:10E7680080634FF0280618BFC3F38024DFE7B3F5B2
:10E77800007F254615BF4FF001094FF002094FF4FD
:10E78800405B4FF4401B3DE7D9F80030B3F5007FFC
:10E798003FF431AF3D463C4620264FF001094FF487
:10E7A800405B2FE7002520262C464FF00309DFF8B1
:10E7B8000CB127E72BF0B6FC059080B12BF0D1FC0B
:10E7C80068B101F083FB054648B92BF0B8FC042872
:10E7D8007FF437AF032000F09BFF059D31E7CCB9EC
:10E7E8002BF0A0FC0546A8B101F070FB90B9B8F178
:10E7F800000F02D13846FFF7A9FD029B13B938462E
:10E8080001F024F82C4623482BF0B3FC2C4801F0E7
:10E818009DFE02952BF086FC0546002814BF454650
:10E828002C46B9F1000F05D001F050FB10B902F0E9
:10E8380035FF81462BF0CDFC039B049AC31A9A42FC
:10E8480080463FD94FF4C871B3FBF1F201FB12388F
:10E85800B8F1630F11D9BAF1000F04D0002001F00C
:10E8680027FA01F01FFAC8F5C870B9F1000F47D1AF
:10E8780012F0CAFC12F012FD2CE0BAF1000F04D11C
:10E8880001F030FA584601F013FA0123C8F1640088
:10E898000193EAE73B79050888370020D83800203B
:10E8A80053CD0508CCB90408ACB9040840C4050820
:10E8B800B4C30508403F0020CDC305080030300030
:10E8C800A0C60508009A9A4208D22BF082FCCDF81F
:10E8D80004A00390A846DDF804A0A5E6BAF1000F4D
:10E8E80004D0002001F0E4F901F0DCF9009B039A60
:10E8F8001344A3EB0800B9F1000F05D00028E9D0B4
:10E90800484528BF4846B3E70028E3D0B0E74FF0B2
:10E91800000A96E607B5114A114B1068596820B1EC
:10E9280003B05DF804EB2BF024BC1A6892050ED5F1
:10E938009A68002A0BDD51B109680C33C988094867
:10E94800009109492FF0DDFB03B05DF804FB07488F
:10E9580003B05DF804EB01F0F9BD00BFB837002043
:10E9680088370020E8E104081F780508D5C905089C
:10E978002DE9F74312F0FCFB00F0D6FE2BF01EF950
:10E9880012F0AEFC2BF010FA01F048FC53482BF0C3
:10E998003DF900F0C3FE18B900F0CCFE00F0C4FE4B
:10E9A8002BF007FA01F070F900F0B8FEB0FA80F029
:10E9B8000021400900F0DCFF10B9082000F0B4FE87
:10E9C80031F03AFE2BF0F4F92BF0F1F902F050FA9D
:10E9D80042482BF01BF9002000F09AFE00F09EFE42
:10E9E80008B901F00FFA0125012001F0A1F8012072
:10E9F80001F098F800F092FEFFF72EFD2BF064F975
:10EA0800012001F0BBF84FF480742846344E354F8E
:10EA1800DFF8D48014F4106957D015B9384601F0DE
:10EA280095FD3578002D3ED100F078FEFFF7C6FD44
:10EA38000028EFD100F072FE044601F065F8204688
:10EA4800FFF7A0FC2BF0A1FB012001F0EDF900F08D
:10EA580065FE28B9254B012101A80193FFF740FC69
:10EA680001F040F9404601F023F901F01BF9337831
:10EA7800012B1AD101F0F8F800F0C0FC044601F0AF
:10EA8800F9F80420FFF7AEFB01F02CF9002001F0A3
:10EA98000FF901F007F9012001F0CEF9032000F089
:10EAA80037FE0020B6E70025C4E7114BDFF8449095
:10EAB800C9F8003001F06EF800F030FD002304467C
:10EAC800C9F8003001F066F8DBE7002CB0D02DF073
:10EAD800BCFD484603B0BDE8F08300BFC078050818
:10EAE800413F0020FDBB050830303000287805087C
:10EAF80030780508B837002008B511F091FB00F010
:10EB080037FB0421064831F016FD2BF0B0FB01F06D
:10EB180055FC02F0EFF8BDE8084011F095BB00BFC6
:10EB2800E8390020014B1878704700BF403F0020AB
:10EB380000487047006889090048704733335340DC
:10EB480038B505462021FAF777FB041E11DA21466D
:10EB5800094826F0C6FA002421462022074826F054
:10EB6800C0FAC4F1200228190021BDE838403BF062
:10EB7800F3BE1F2CF0DD38BDC9780508E378050819
:10EB88000428034607B506D801460F4803B05DF8C8
:10EB980004EB01F06DBC062168460C4A23F016FD13
:10EBA800011E0DDD052901DD27F04CF8442201F195
:10EBB80008036B446846013103F8082C01F058FC3F
:10EBC80003B05DF804FB00BF0A7905080F79050852
:10EBD800F8B5244DAB7DDB0732D52E687068012867
:10EBE8002ED9B168431ECA5C0A2A29D14A1E002BB5
:10EBF80001DC1A4608E0D45C0A2CFAD0013BF6E79F
:10EC08008C5C202C02D101329042F9D8002B0CDD0B
:10EC1800541CA04209D15C1E0C44A14205D014F832
:10EC2800017D0A2F0CD0202FF7D00144D21A11F8F9
:10EC3800023C94083A2B0C4F08BF0134013C00D227
:10EC4800F8BD04223946304631F02EFB04213846FF
:10EC580001F00EFC2B6904332B61AB7D43F00203FA
:10EC6800AB75EBE7C437002096D0050820220021B9
:10EC780001483BF071BE00BFB0390020002238B512
:10EC88000B4C0546A26062754FF0FF326B68084670
:10EC9800C4E9032363602560A1612AF0B7FF6B68AC
:10ECA8000BB90123A375BDE83840FFF791BF00BF3A
:10ECB800C4370020F8B503780446DBB10E4FD7F807
:10ECC800B80018B12146F2F733FB98B12046F2F7A5
:10ECD80041FB461C30462CF0ADFE054650B132468D
:10ECE80021463BF012FE05491C22081D3BF01AFE86
:10ECF800C7F8B850F8BD00BFF8380020B039002078
:10ED08002DE9F347AC4C06462368D3E901102DF0F2
:10ED1800DEF9A5680746002D40F03A81731E042BE2
:10ED28001AD8D4E900325B689A4279D0012E15D1FD
:10ED3800236865689868D4F8108000EB08012844B7
:10ED4800A8EB050800252AF044FFA8450646A5605B
:10ED580040F3BC80A946AAE00D2E13DC022E40F336
:10ED6800B580F31E0A2B00F29180DFE813F05900FA
:10ED78008F00CF018F008F0060008F008F008F0001
:10ED88003E004E001B2E4FD07F2E50D0A37D9907FA
:10ED980000F181801F2E40F39980206821698368E3
:10EDA8005A5C06F0C003802B0CBF237DF2B202F13F
:10EDB800400508BF0133EDB214BF0023DBB2372D85
:10EDC80097BFE5250025D20802F0060298BF154135
:10EDD80019443246237598BF05F0030531F04EFB00
:10EDE800237DAB4272D1013597E074482AF00EFFBB
:10EDF800A0692AF00BFF2268636821699068C91A24
:10EE0800184401F035FB002587E06D482AF0FEFE26
:10EE1800206831F0C2FA636800261844FFF74AFFF9
:10EE2800304602B0BDE8F0870123A3604EE02269B6
:10EE380061688A424AD900232068561AD0F808E047
:10EE4800B34203EB010C18D1032BCCBF04260126D7
:10EE5800961B33461EF803C019460CF0C00CBCF1D3
:10EE6800800F03F1FF33F5D0A2EB01084246761A72
:10EE780031F011FB4FF0010919E01EF80CC0BCF18C
:10EE8800200F01D10133DBE70126E1E7A37D9A07D3
:10EE980023D5092E18D0202E7FF47CAF002603211D
:10EEA8002068A675B14631F0EFFA4FF00308A8EBD9
:10EEB8000600FFF765FE2369A3EB08032361B9F198
:10EEC800000F00F0298128E00023A375A37D4FF0EF
:10EED800FF3623F00203A375A2E7092E7FF45AAF89
:10EEE80022682169D2E90123002A40D00B4413F893
:10EEF800010C04F0E9FA002839D00425314B0193BC
:10EF08000026019B21695A1C019231441A78206815
:10EF1800013631F0ADFAB542F3D12368D3E90110D7
:10EF28002DF0D5F8B84203D20321274801F0A0FA02
:10EF380023682769D3F80880D3F80490781908EB78
:10EF4800090140442AF045FE0646A9EB070108EBF3
:10EF5800070001F08DFA236822695B689B1A5B1B26
:10EF6800981BFFF70DFE23692B442361AEE7236846
:10EF780060689D682169154A091A01AB284410F098
:10EF8800CBFC05460028A1D0431C3FF431AFB7E7BE
:10EF9800013D032D00F2E880DFE815F004001A00B7
:10EFA800A000E1004F2E04D05B2E40F0DD8002234C
:10EFB8003BE7042339E700BFC4370020147905086C
:10EFC8003B79050896D005081D790508E8E104088D
:10EFD800A6F13003092B03D803236675A36075E7F0
:10EFE8000023412EA3602ED1E368062B3FF76EAFB6
:10EFF8005E4D03F1010A2D3305EB8305AB68002B49
:10F008003FF464AFD4F80080D4F80490D8F808002E
:10F018002169014448442AF0DCFD06464046C8F808
:10F028000490A968C4F80CA031F015FA6368226945
:10F03800A2EB03082268B8F1000F5568A5EB030599
:10F048007FF76BAF16E7423E062E3FF63FAF01A3B0
:10F0580053F826F079F00008BFF00008CFF0000858
:10F06800D5EE000815F10008D5EE000839ED0008C6
:10F07800E568002DFFF62AAFD4F80080D4F8049094
:10F08800D8F808002169013D014448442AF0A1FD4F
:10F09800D8F804100646A1EB09014046E56031F0B6
:10F0A800F3F9E268002AC1DB304B206803EB8203E6
:10F0B800D3F8B810B8E7236822695B689A42BFF4AE
:10F0C80005AF01252BE0226963689A427FF6FEAE00
:10F0D80000254FF00108A9462E46E8E67E2E43D1CA
:10F0E800637D312B3FF424AE333B052B3CD801A282
:10F0F80052F823F037F1000815F1000871F1000803
:10F1080071F1000839ED000815F1000823685D6801
:10F118002369ED1A0023A360002D7FF7D7AE23687B
:10F12800294698682369184401F0A2F91BE720686A
:10F1380021694368994217D2012285685B1A0D44F8
:10F1480015F8016F06F0C006802E01D19A4204D14D
:10F1580031F0A1F90023A36055E60132F0E7462E0D
:10F16800D4D0482E3FF4E4AD00235EE6F838002002
:10F178002DE9F04F8BB068460A4BCDE90045196878
:10F18800CDE90267091A8908CDE90489CDE906ABFA
:10F19800CDF820C0CDF824D031F0CDF90BB0BDE8C2
:10F1A800F08F00BFF838002070B5067804461EB10D
:10F1B8004FF0FF35284670BD2BF05AF8C31E012BBF
:10F1C80005460CD801210C48217001F051F9032D96
:10F1D800EED10A48836E60309E6010F031FAA38841
:10F1E800013B9BB2A380002BE4D10121044801F02C
:10F1F8003FF96388A380DDE721790508F838002006
:10F208003F7905082DE9F0431D46002391B00446D7
:10F2180003A817460493884610F0FEF907F0010684
:10F22800034600285BD1F90641D5D4E90121DC2049
:10F238002EF09FFD0446B8F1010FD4F8009007D1D5
:10F248004FEA09114FF4347041F0060105F066FDEC
:10F258002146424601A80DF087FD4946C7F38002C2
:10F2680001A808F081FFB8F1010F044601D1FFF7AA
:10F2780043FC380602D4032000F0FCF914B1204600
:10F288002DF01BFA4FF0FF3000F0F4F9012004F0E4
:10F29800B7F809F003FFEEB9CDB900241EB101217A
:10F2A800474801F0E5F8204611B0BDE8F0837A063A
:10F2B80005D594E80E00DC202EF013FDBAE7BB0656
:10F2C800B9D520462CF061FB2EF061FDB2E7002392
:10F2D8002B60E2E701213A4801F0CAF8DCE74FF079
:10F2E800FF3000F0C7F9022004F08AF8790602D549
:10F2F800A368206898471EB10121314801F0B8F889
:10F30800049C20460AF0ACFA2E4905F039FA002888
:10F3180041D004982EF091FF0E283AD0C20705D4A8
:10F3280083072BD10268284B9A4227D12CF0C9FFBA
:10F3380040F48074002DB1D04FF0FF33049F2C604F
:10F3480038466F60AB602EF063FF0028A6D0694690
:10F35800384601AA2EF08BFF019B002B9ED05A68DD
:10F36800AA60002285F82C2018682CF02EFB202299
:10F37800014605F10C003BF026FB8FE70146002211
:10F3880012480AF089FA124910482EF036FE012078
:10F39800CEE70020CCE70F4B9C420DD004990B48D8
:10F3A8002EF053FD049B0C49186805F0E9F908B1E3
:10F3B8008224BFE70124BDE74FF40064BAE700BF29
:10F3C80021790508B8E60408C4E00408E8E104085F
:10F3D800BDB705087039002094E6040808B503781D
:10F3E8004BB901210170044801F042F82AF040FFAE
:10F3F80003380128FAD808BD217905082DE9F0431A
:10F408008BB0202106A830F078FF0026DFF8E880CE
:10F418003A4F40462AF0FAFB384607962AF0F6FBA0
:10F428002AF026FF0128044635D107990229F0D190
:10F43800089B1A78052AECD193F80190B9F1410F8D
:10F4480006D02F4801F014F800232C480793E5E76D
:10F4580080252C4801F00CF803216846ADF80050CF
:10F468008DF8024001F004F8002301AA0392264A0D
:10F4780021460492254A03A805924A468DF804308D
:10F48800ADF80650ADF80850FFF7BCFEC305DBD554
:10F498000BB0BDE8F083022809D11D482AF0B6FB5D
:10F4A80006A830F04CFF00201A4B1870F0E703282C
:10F4B80002D100230793B3E7042804D0C1B206A8F9
:10F4C80030F07AFFACE714482AF0A0FB079B43B959
:10F4D8000F482AF09BFB06A830F031FF4FF48070EC
:10F4E800D6E700231122012106A8FFF78BFE10F4AE
:10F4F800106F91D0CCE700BF23790508B7B5050890
:10F508001CB204083E790508B1F10008E5F30008CB
:10F518003B790508413F0020417905082DE9F04174
:10F5280092B0202101A830F0E8FE494EDFF824818E
:10F5380030462AF06BFB48482AF068FB30462AF030
:10F5480065FB464FBA8A002302B1BB8205A8029325
:10F55800069310F061F8044690B9414901A82AF0D1
:10F5680046FB012805462CD139482AF04FFB01A853
:10F5780030F0E5FE20463B4B1D7012B0BDE8F0812F
:10F58800022003F03DFF30462AF040FB069936483A
:10F598002EF05BFC029B002BD4D001A830F0FDFEBE
:10F5A80010F0F6F858B10A2101A830F005FF4146DD
:10F5B80001A82AF01CFB03280BD00428EDD1002158
:10F5C8002CE0022803D122482AF020FBB0E70328C8
:10F5D80001D1304619E0042808D11D482AF016FB4D
:10F5E80001A830F0ACFE4FF48070C6E70528D1D1F1
:10F5F8001E482AF00BFB02941D4C2AF039FEC1B2BA
:10F6080003298DF8031003D111482AF0FFFA99E76E
:10F6180004290CD10E482AF0F9FA012100231622F8
:10F6280001A8FFF7EFFD10F4106F8BD0A5E701A834
:10F6380030F0C2FE9DF803300D2B03D120462AF08E
:10F64800E5FADAE701210DF1030000F011FFD4E734
:10F658003B79050880790508B3770508F838002054
:10F6680044790508413F0020E8E104084979050884
:10F6780079790508014B1860704700BF44060020DF
:10F68800024B986A003818BF01207047F8380020EC
:10F698002DE9F04106460D4600270DB9BDE8F08179
:10F6A80033780A2B16D1AFB90121104800F0E0FEDB
:10F6B800012406EB040843461FB998F800200A2ADB
:10F6C80001D0A54208D13046214600F0D1FE464679
:10F6D8002D1BE2E70024ECE71F7808F10108A7F1E9
:10F6E8000D035F425F410134E5E700BF85790508F6
:10F6F800024B034819782EF0E3B900BF423F0020BF
:10F7080054C30408014B1878704700BF423F0020DB
:10F71800014B1870704700BF423F0020014B18781A
:10F72800704700BF433F0020014B1870704700BF6F
:10F73800433F00202DE9F04130F081FF294B04467A
:10F7480020F47F0020F47F409842274E0AD114F419
:10F758007F4FC4F3072505D030F070FF3570284679
:10F76800BDE8F081002333702AF031FA28B1062869
:10F7780033D85423C340DB072FD51C4830F05EFF35
:10F7880000F0B0FA2AF016FD064600200F460146A2
:10F79800DFF85C80FA220023F1F770FD7D2A73F10F
:10F7A800000334BF4046002000F082FA2AF05DFDD5
:10F7B800054648B92AF0FEFC801B61EB0701B0F54D
:10F7C8007A7F71F10003E5D3002000F071FA00F0B0
:10F7D80069FA25B9204630F031FF0025BFE7112529
:10F7E800BDE700BFAF0000AD433F0020AF1100AD43
:10F7F80000303000024B43EA002030F01FBF00BF4A
:10F80800AF0000AD0D4D08B52B780446012B0FD97C
:10F8180001280DD90A4825F064FC2146094825F03D
:10F8280060FC2978084825F05CFC26F0DCF9FCE748
:10F838002046FFF7DFFF30F0FBFE00BF433F00200C
:10F84800877905089D790508A979050810B5044642
:10F85800002838D01C4800F079FE631E112B12D8FE
:10F86800DFE803F02D1111111111112B11291111BC
:10F8780027212523091F154800F068FEBDE8104020
:10F88800134800F063BE023C1248E4B200F05EFE8A
:10F898000A2C16D8104B53F8240000F057FE0F48D6
:10F8A800EAE70F48E8E70F48E6E70F48E4E70F48BC
:10F8B800E2E70F48E0E70F48DEE70F48DCE70F48CC
:10F8C800DAE70F48E9E710BD5FC30508E7C3050895
:10F8D80073C305084BCA05084CBB040884C3050854
:10F8E800A7C8050807CB0508DFC40508F5C405083F
:10F8F800E0C50508C3C50508AACA0508C1C60508A4
:10F908009CC4050800B597B002460A236946044816
:10F9180031F02BFE684632F068F917B05DF804FB49
:10F92800C012002010B5064C23783BB14FF47A7210
:10F93800044B1A6000F01CFA0023237010BD00BFAE
:10F94800443F002048060020074B1A685AB11A683D
:10F95800012A09BF05491A680A704FF47A7218BF5C
:10F9680002F1FF321A60704748060020443F002029
:10F978002DE9F0414FF00008514EADF5287D0746BE
:10F98800504C30460D46A6F8048000F0FFF906F109
:10F998008000C4F8048031F0E4FD0D2806D147B991
:10F9A8003DB900200DF5287DBDE8F081002D00F05F
:10F9B80084804FF40073002200930721424828AB4B
:10F9C80012F034FE0028ECD100F0D2F93F493E484D
:10F9D80012F046FD0028E4D13D493B4832F0B4FC22
:10F9E8000028DED13B48FFF78DFF3B48FFF78AFF31
:10F9F8003A48FFF787FF3A48FFF784FF394932480A
:10FA080032F0A2FC384B03AA03F1380715461868F0
:10FA18005968083303C5BB422A46F7D11B88334AC5
:10FA28002B80392312A9029327480A2331F09DFD20
:10FA3800029A02AB03A912A831F06EFF12A832F0A5
:10FA4800D4F82B48FFF75EFF2A4B03AA03F11007EF
:10FA5800154618685968083303C5BB422A46F7D1CA
:10FA6800186899889B792860AB711623A980224A67
:10FA7800029312A90A23144831F077FD02AB03A9B7
:10FA88001A6812A831F048FF12A832F0AEF81B49E4
:10FA98000D4832F059FC002883D100F069F9184B61
:10FAA800012523600023E360164BC4E90156C3E92E
:10FAB8003B442BF082FA284674E70028EFD070E721
:10FAC80040120020E0370020C0120020678505089A
:10FAD800C0790508CC790508DF790508F6790508A5
:10FAE800007A05080D7A0508427A0508117A050892
:10FAF800257A05087C7A0508347A05083D7A0508D0
:10FB0800955C0508F83800204FF47A7208B5044B64
:10FB18001A6000F02DF9BDE8084011F0DBB900BF0C
:10FB280048060020014601482AF0D5B840120020B6
:10FB3800014601482AF0EBB840120020024B5868F1
:10FB4800003818BF01207047E0370020034B0448F5
:10FB58005B68002B08BF0020704700BFE03700201B
:10FB680040120020034B1B7813B903482AF001BB4D
:10FB7800704700BF453F0020937A050810B1012265
:10FB8800024B1A70024800F08FBB00BF463F0020AE
:10FB9800F0370020F8B5254B1D7825B1BDE8F840B1
:10FBA8000120FFF7EBBF224B22481D702BF04BFBC7
:10FBB80020482BF02EFB58B91E482BF03CFB80F058
:10FBC8000104012000F060FB01270546E4B20AE0C9
:10FBD8002AF0A8FA0028EFD016482BF02CFB2F4665
:10FBE80080F00104E4B2F4B1012000F055FB0646B0
:10FBF80011482AF0BEFA11482AF0BBFAFEF78AFE2D
:10FC08000F482AF0B6FA0F482AF0B3FA0E482AF03D
:10FC1800B0FA17B1284600F037FB34B13046BDE8DA
:10FC2800F84000F039BB2646E2E7F8BD453F002022
:10FC3800463F0020080700209A7A05089F7A0508A1
:10FC4800A47A0508A87A0508977A0508044B1B7852
:10FC580023B9044B1B780BB1FFF79CBF704700BF5B
:10FC6800453F0020463F00200122014B1A70704793
:10FC7800453F00200022024B02481A7000F014BBD6
:10FC8800453F0020F0370020034B044A04481A601F
:10FC980000225A602BF0D1BAF037002055FC00083A
:10FCA8000807002001482AF02DBB00BF04380020B7
:10FCB80038B5094D04462B6883420CD0074B197898
:10FCC8002AF05BF82C60011E18BF0121BDE83840FE
:10FCD800034800F0D3BE38BD00380020DF0A0020FA
:10FCE8000438002070B50B4C257895B901260A49CF
:10FCF8000A48267000F0A6FE2A46314607482AF030
:10FD080029FB4FF08072064B18681A60FFF7D0FF86
:10FD1800257070BD473F0020A80F05080438002053
:10FD280000380020014B1870704700BFDF0A002020
:10FD3800014B1878704700BFDF0A0020F8B50E465F
:10FD48001C4615466AB1094F3B781BB900F06AFB9F
:10FD580001233B7022463046691EBDE8F84011F089
:10FD680043B9012B94BF00200120F8BD483F002073
:10FD780010B5054C11F096F823780BB100F064FB30
:10FD88000023237010BD00BF483F002010B50F4B63
:10FD980004460360838843F00503838030F03CFC0D
:10FDA80001230E220A4984F88430231DC4E908235C
:10FDB800C4E90D2323616161064B0749A060C4F8BB
:10FDC8008040E260A162E36310BD00BF80F60408D2
:10FDD800C19D03081F9F030845FD000808B5FFF7EC
:10FDE80097FC044B03F178029A62BDE8084011F0D1
:10FDF800D5B900BFF83800200022014B1A607047BF
:10FE0800103800200122034B1A700022024B1A609E
:10FE1800704700BF493F0020103800200022014BE6
:10FE28001A707047493F0020024A13680343136061
:10FE3800704700BF14380020024A136823EA000301
:10FE48001360704714380020014B1878704700BFC2
:10FE5800493F002038B50B4B1B7893B10A4B1B6800
:10FE68007BB90A4C25682AF0B4F92060236813B9D5
:10FE780023680133236025B9BDE838400120FFF726
:10FE8800ADBF38BD493F002014380020103800208D
:10FE980010B50C4C206890B10B4B1B6883B92AF045
:10FEA80098F9236883422368A0EB030040F2EE230D
:10FEB80088BF00F1FF30984294BF0020012010BD98
:10FEC8000020FCE71038002014380020024B186886
:10FED800003818BF0120704710380020012910B5DC
:10FEE80002460C4617D9042915D00B490B482EF0A9
:10FEF8002DF9022C03D0052C0BD0094900E0094943
:10FF080006482EF023F9BDE81040074903482EF0B3
:10FF1800F8B80649F4E710BD75CB0508E8E1040810
:10FF2800B8C8050868C80508BDB7050873C8050836
:10FF38002DE9F04F9DB000AF80460C469246FFF782
:10FF480005FE28B9012528467437BD46BDE8F08F5F
:10FF580001239F4A07F11801803031F006FB002881
:10FF6800F0D1D7E91402D7E90A139A4208BF8842A8
:10FF780000F02B8197F84930002B40F0268107F1DB
:10FF8800180029F0F7FF5B28064606D1D7E90A23AF
:10FF980007F1180031F0FEFEE3E7002EF6D008F175
:10FFA800FF3919F8015F2DBB304603F08DFA20B1F7
:10FFB80007F1180029F0DEFF06463D2E1CD107F197
:10FFC800180029F0D7FF22280CBF012300238AF844
:10FFD800003040F0CA8007F1180029F0BCFF222841
:10FFE8002AD016D830B30A2824D0C1B2204629F026
:08FFF800D9FFF0E7B54206D085
:020000040801F1
:100000000A2EB2D007F1180029F0C7FFADE707F1BB
:10001000180029F0A4FF0646C7E75C28E9D107F1DC
:10002000180029F09CFF7628E3D861281DD80A28FB
:1000300004D0552800F089800028DAD1052509E090
:1000400007F1180029F09AFF0A2803D0232807D0C7
:100050000028F3D1EDB207F1180031F0CAFD76E7C0
:1000600007F1180029F099FFF4E7A0F16203142BBF
:10007000BFD801A252F823F06F010108F3FF000876
:10008000F3FF0008F3FF0008DD000108F3FF00089C
:10009000F3FF0008F3FF0008F3FF0008F3FF000878
:1000A000F3FF0008F3FF0008D1000108F3FF000888
:1000B000F3FF0008F3FF0008CD000108F3FF00087C
:1000C000D5000108E1000108D90001080D2090E7E2
:1000D0000A208EE709208CE70B208AE70C2088E7AE
:1000E0003B1D6E469B464FF00409D84609EB0B0AB0
:1000F00007F1180029F033FF08F8010BD045F7D1BC
:10010000002339460BF809301022584622F002FB32
:100110003B680146434528D1B0F5881F22D27F288D
:100120001AD9B0F5006F19D3B0F5803F34BF03235F
:100130000423227B22B16268134422689A420FD9B9
:10014000204630F044F9B54649E707F10C036E4606
:100150009B464FF00809C8E70123EAE70223E8E7D6
:100160006360F0E70225B54674E7B54666E7082008
:100170003FE70A283FF462AF00283FF45FAF002555
:100180000D281CD009DC092819D00A2800D040B954
:1001900063685B1B636000255CE720280FD0232881
:1001A00005D0C1B2204629F001FF00250CE06368AC
:1001B00007F118005B1B636029F0EFFEEBE7C1B2AB
:1001C000204629F0F3FE013507F1180029F0C7FE9B
:1001D000D6E704253FE700BF257A050870B586B04D
:1001E0000E4610220DF1070302A929F0EAFE04468B
:1001F00048B99DF807507DB9084902A8F1F79CF865
:1002000020B901253570204606B070BD044902A80A
:10021000F1F792F80028F5D00524F4E7AF7A050845
:10022000B47A050810B5054C23782BB929F06EFF78
:1002300030F02EFA0123237010BD00BF4A3F00208A
:1002400073B505460C46C1B10E4B1B78C3B90A46BF
:1002500001AB01460C482BF00DF906460B4B1B7801
:1002600053B902F0D7FA40B12146284629F056FF8B
:100270002146284611F062F93446204602B070BD8E
:100280000E46EBE74B3F0020500700204C3F00207C
:10029000024B1A7818701046704700BF4C3F002080
:1002A000024B1A7818701046704700BF4B3F002071
:1002B00010B5044601F03EFFE3681BB90C4A116813
:1002C000A14203D1BDE8104001F04EBFA360094B2D
:1002D0001968E160196809B119688C60116801B981
:1002E00014601C6001F040FF10F05CFF10BD00BF07
:1002F000203800201C3800202DE9F041144E32F047
:1003000086FE33680BB3134D01F014FF2C681CB14B
:10031000BDE8F04101F028BF01230F4A2B6033688C
:10032000346014601BB92B68013B2B60F0E79F68B9
:10033000C3E90244D3E9006801F016FF0EB140465C
:10034000B04701F0F7FE3B46ECE7BDE8F08100BFA7
:1003500020380020183800201C3800202DE9F743F1
:100360000025A846144E019501F0E4FE346801AF63
:1003700054B9019B3360114B1D60114B1C6003B0DD
:10038000BDE8F04301F0F0BED4F808902046C4F870
:1003900008800FF039FF18B10023E3604C46E7E70F
:1003A00060680FF031FF0028F6D12B463C602546EF
:1003B00004F10807F1E700BF203800201C380020B6
:1003C0001838002010B5044B1C6804B910BD6068D3
:1003D00030F0E9F8A468F8E72038002008B532F0DA
:1003E00013FE29F0ECFC00F087FBFFF79FFA32F0D8
:1003F0000DFE29F0E4FC002030F027F9034BC3E99F
:100400000001BDE8084032F000BE00BF50300020BF
:1004100008B5FFF79DFABDE80840002201490248EF
:1004200029F0B8BEDD0301082838002010B5074CBC
:1004300001F080FE23680BB910F0D6FE236801336B
:100440002360BDE8104001F08FBE00BF24380020BB
:1004500008B501F06FFE074B1A6812B11A68013A2D
:100460001A601B680BB910F0CDFEBDE8084001F022
:100470007BBE00BF243800202DE9F843DFF87C80E4
:1004800000AF05460E4629F095FCD8F8003043B37E
:100490001B4829F00AFFC0F500720446D8F8000096
:1004A00043689919914223D90734D21A294624F076
:1004B00007042FF0FDFEE946ADEB040D6946104838
:1004C000D8F8004000F050F8014620462FF0C7FF52
:1004D0000A21D8F800002FF073FF0023C8F800307D
:1004E000CD4631462846FFF7ABFEBD46BDE8F88352
:1004F000324629462FF0DCFEF3E700BF84370020A8
:10050000DAC30508A1F18003532B70B5064618D84D
:10051000194602230D480E4C10F8012B914205DAC2
:1005200003FB0144E518A54205D870BD03FB024456
:10053000891A0133F0E7304614F8011BFFF7E2FF98
:10054000F1E7BDE870402FF042BF00BFBD7A05085B
:10055000C77A05080246024902482DF0D6BD00BF01
:10056000BA7A050810E804082DE9FF410546802401
:100570000A4615F8011B684601312FF0DDFE009E8A
:10058000254FDFF89880013E019B9E4205D86846C2
:100590002FF007FF04B0BDE8F0810023184619468C
:1005A0001A4695F800C0520014EA0C0F14BF4FF021
:1005B000010C4FF0000C64084CEA020204BF8024D6
:1005C000013501318242C9B205D317F801C00CEBE5
:1005D00040006344E5E71B1A4244D15C012917D16E
:1005E0000B2300202A784000144214BF012200226D
:1005F000640804BF80240135013B40EA0200F1D1C8
:1006000001302BF0E6F9014668462FF028FFBBE7E2
:100610006846FFF777FFB7E7037D0508597C0508B3
:1006200008B5024824F061FD002008BD107D0508D2
:1006300038B5FFF78FFA044620B90D4824F055FD70
:10064000022038BD29F05EFB20B90A4824F04DFD98
:100650000420F6E7084D2B782BB9204629F088FBBB
:1006600008B90648F2E7012300202B70E9E700BF34
:10067000237D0508357D05084E3F0020487D05088F
:10068000F8B514460E461F46FFF764FA05460420E7
:10069000FFF7CEFB3B4622463146284632F0DDF8D6
:1006A000D5F8CC30A34207D134B14FF400723146B3
:1006B00005F580703AF02DF9D5F8BC300020A34242
:1006C0009EBF0122014B1A70F8BD00BF4D3F0020B4
:1006D00038B50C461546FFF73DFA022C03D0052C21
:1006E00007D0012C15D12A46214612F081FD0020A9
:1006F00038BD2A4600210A4C12F07AFD0420FFF78B
:100700009FFB2378002BF2D0FFF7A8FB0023237078
:10071000EDE70448214624F0E8FC6FF08500E7E7A8
:100720004D3F0020587D050808B5F4F75DF830B15D
:10073000BDE808400121024A024825F099B808BDE9
:10074000757D0508D4B0040838B504460D4625F07B
:100750005AFB90B12B7843B92046F3F7FFFF20B145
:100760000121064A064825F083F82B78012B04D195
:100770002046BDE83840FFF7D7BF38BD967D050855
:10078000D4B0040837B5844824F0AFFC834824F083
:10079000ACFC8349834825F096FB034638B1824A76
:1007A0000121824803B0BDE8304025F06AB8804995
:1007B0007C4825F088FB034608B17E4AF0E77E4975
:1007C000784825F080FB034608B17C4AE8E702F050
:1007D00021F898B90E2002F06FF802F021F8D8B98C
:1007E0000E2002F077F87648F2F722FF014608B3B0
:1007F000744803B0BDE8304024F077BC012180206C
:1008000010F0CAFD03460028E4D080226E496F48EC
:1008100002F022F86D48DEE70121802010F0BCFDD7
:1008200003460028DCD0802269496A4802F014F8A7
:100830006848D6E75B4825F0A6FA0128044640D16F
:10084000654824F052FC2146644A5648F5F796F96B
:1008500038B1634A0121554803B0BDE8304025F066
:1008600007B8604824F041FC01F0D4FF48B15E496C
:10087000234622464B48F5F7B1FA014608B15B48DA
:10088000B7E701F0CDFF40B1012359491A46454869
:10089000F5F7A4FA01460028F1D1012355491A467B
:1008A0004048F5F79BFA014608B15348A1E7534881
:1008B00024F01BFC01210223EF223A48009125F08D
:1008C00069FA4F4824F011FC00214E4A3548F5F7EB
:1008D00055F9044608B14C4ABCE701F09BFF78B1DA
:1008E0004A4824F002FC012322463F492D48F5F7EF
:1008F00075FA28B1464803B0BDE8304024F0F5BB96
:1009000001F08EFF50B1414824F0EFFB012300229B
:1009100037492448F5F762FA0028EBD10123002279
:1009200034492048F5F75AFA044608B10146BCE7B5
:1009300001250223EF22014600951A4825F02AFAE4
:10094000344824F0D2FB2146164825F047FA3248B5
:1009500024F0CBFB3149134825F033FD08B1304A70
:1009600078E7304824F0C1FB0E48F3F7B9FE08B130
:100970002D4A6FE72D4824F0B8FB0A4825F043FACA
:1009800038B90848F3F7EAFE08B1294A62E729486E
:10099000B1E703B030BD00BFB67D0508C87D0508CE
:1009A000EC0600200C110020E47D0508D4B00408FA
:1009B000D4060020127E0508BC060020447E0508EF
:1009C0004C060020717E050834AE0408A8300020D3
:1009D00018AE040858300020947E050864060020F4
:1009E000B57E0508DC7E0508B36A0508027F0508A8
:1009F000936A05084B6B0508257F05084A7F0508A3
:100A00006F7F050878060020907F0508B77F0508EE
:100A1000DD7F0508FD7F05081380050849070108EB
:100A2000298005084D800508588005087C80050848
:100A3000967D05088D80050808B501F0EBFE0028BD
:100A4000014808BF002008BDA830002038B50C467A
:100A50000546084629F0BAF86C60606828F0ABFBE0
:100A600020B9074824F041FB012038BD4FF4803203
:100A7000217A606829F039FC0028F5D12872F4E762
:100A80000681050838B50C460121436805465868BB
:100A90001B7A994003691B6819420CBF234684F0F6
:100AA00001034BB18368DB689847014610B10448E5
:100AB00024F01BFB6C7238BD83681B69F4E700BF30
:100AC0001D81050838B543680129094A04460D46C9
:100AD00018BF4FF40032197A586829F006FC014615
:100AE00020B1044824F001FB012038BDA572FCE7C9
:100AF000060002003581050808B5FEF7C5FD10B9EE
:100B0000FFF7CAF970B108BD0D4A934203D1BDE8A1
:100B100008402AF051B80B4A9342F4D1BDE808408E
:100B200000F058BD08480368002BECD0074A9342F8
:100B3000E9D0074A9342E7D1BDE8084032F096BDBC
:100B4000C8BE0408A0BC0408F830002020EE040849
:100B5000641D05084FF0FF3370B5204E204C336004
:100B600023682BB93368E3B9BDE8704013F008BFC0
:100B70001C4DAB42F6D01C4A934204D1204632F0C1
:100B80008EFD2560EEE7194A934203D1204600F01E
:100B900051FDF6E7164A9342F3D1204601F0ACF836
:100BA000EFE7144C2368002BDED00E4DAB42DBD0B8
:100BB000114A934204D1204629F0DBFC2560D3E79B
:100BC0000E4A934203D1204601F010FAF6E70C4A90
:100BD0009342F3D1204601F019FDEFE7040700200E
:100BE000F830002020EE0408641D0508A0BC0408AD
:100BF000C8BE04083838002040BE040844C00408B9
:100C000094C20408F8B5334C334E23680BB1B34299
:100C10000DD1266031480368002B59D0B34257D01C
:100C20002F4A934246D1BDE8F84015F08BB92D4AC2
:100C3000934216D16568A54203D304F198039D42FF
:100C4000E8D928460FF0E0FA0028E3D0264B6C22C2
:100C50002946184639F05DFE6060284632F09DFD59
:100C6000D8E7224A93421ED16568A54203D304F116
:100C700098039D42CED928460FF0C6FA0028C9D065
:100C8000194A2B46944605F1200E174618685968F4
:100C9000083303C773453A46F7D12846C4F804C061
:100CA00032F0BCFEB6E7124A9342B3D120462AF096
:100CB0000AFAAFE70F4A934203D1BDE8F84000F0CB
:100CC000E5BC0D4A934203D1BDE8F84001F026B8D7
:100CD000F8BD00BF3838002020EE0408F8300020AE
:100CE000641D050840BE04084038002044C00408C4
:100CF00094C20408A0BC0408C8BE040808B514487F
:100D000003681BB9134803684BB908BD124A9342E4
:100D1000F8D0124A9342F5D12AF068FAF2E70E4A67
:100D20009342F2D00E4A934203D1BDE8084032F01C
:100D3000C5BC0C4A934203D1BDE8084029F055BF19
:100D4000094A9342E1D1BDE8084029F0A8BB00BFA1
:100D500038380020F830002020EE040894C204083F
:100D6000641D0508C8BE0408A0BC040810B5084BE3
:100D7000084C1B68A34200D043B9074BB4220021A2
:100D8000184639F0EDFD40F8044D10BD0020FCE799
:100D9000F830002020EE0408FC30002008B5FFF7F2
:100DA000E5FF10B9014804F0E3F808BD2DC50508BA
:100DB00010B5084B084C1B680BB1A34208D1074B78
:100DC00094220021184639F0CBFD40F8044D10BDA7
:100DD0000020FCE73838002020EE04083C380020D2
:100DE00008B5FFF7E5FF10B9014804F0C1F808BDE8
:100DF00033C50508094B1B685A1C0DD0002B0BDCB2
:100E0000B8225343064A9818D358064A934203D04F
:100E1000002B08BF0E2070470E20704704070020EB
:100E2000F830002020EE04080E2807B513D00E4A33
:100E30009042136803D10D4A934200D093B908F051
:100E400013FDC388E922009340F2151140F25713B5
:100E5000074804F0C9F84FF0FF33064A136003B0A7
:100E60005DF804FB0023F8E7F830002020EE0408CA
:100E7000DBCC050804070020074A1368013304D1BE
:100E8000064B07491B688B4200D17047002BFCD0F2
:100E900000231360704700BF04070020F8300020D3
:100EA00020EE04082DE9F04F04461F464FF00008DD
:100EB00085B0CDE9021200F15009B84502D305B062
:100EC000BDE8F08F039B03EB080694F8B530757806
:100ED00096F901B0002B37D0B57806F1030A4846E1
:100EE00017F094F9A8B3012300930021334694F836
:100EF000B620206DD4F860C0E0470095534601212C
:100F000094F8B620206DD4F860C0E047484633F02E
:100F1000BEFDBBF1000F23DB00202AF038FC029B52
:100F20003BB1D4F88430164A934202D0204629F0CF
:100F300045FAFEF7A9FB0028C1D194F8B530454425
:100F4000DBB905F10208B8E706F1020A05F07F05F2
:100F5000C5E7FEF799FB0028C5D1FFF7CDF9BEE73D
:100F60006B1C94F8B520DDB256FA83F3134458781D
:100F7000FF2808BF4FF4FA70CFE705F103089CE79C
:100F800020EE0408F0B54B6B05460C468BB0002BE9
:100F900000F0C980012380F84030486B33F0B8F886
:100FA00085F83C00636B002B00F0C080A36B002B26
:100FB00000F0BC804FF48073A5F84030A06B33F094
:100FC000A7F885F83D00B4F85630002B14BF012374
:100FD000002385F8B43094F8573018BF042185F801
:100FE000423094F8563085F8433094F855600CBF81
:100FF00001230026626B0CBF194633460AB9A26B67
:1010000032B1228EB2F5807F02BF00260221334624
:1010100001220027CDE90422CDE90222CDE9001307
:1010200005F10800638C228BE18A33F048FC94F8C8
:1010300059300897099394F8543005F15000CDE9E0
:101040000673638D0593238D0493E38C0393A38C24
:101050000293B4F920300193B4F91E300093628BEF
:10106000A38B216817F04AF8A38D3249A5F8AA305E
:1010700094F82E3085F8B030238EA5F8AC3094F873
:10108000323085F8B130606CEFF78AFEF0F78AF8FD
:10109000A5F8A80094F84C3085F8B27085F8AF3008
:1010A000206D2449EFF77CFEF0F77CF8C5F890003E
:1010B00094F8543085F8B36085F8B63063681D49FC
:1010C000C5F894302389A5F8A030E068EFF768FEF2
:1010D000F0F768F8A5F8A6002369C5F89830A38A48
:1010E000A5F8A230E36BC5F89C30B4F84030A5F801
:1010F000A430114BC5F8843094F8583085F8B530D9
:10110000A36C4BB128460D4B40F8843FA16CFFF710
:101110009DFCA06C28F058FD284609490BB0BDE89D
:10112000F04029F090B980F840303BE7002385F883
:10113000413048E700007A4420EE0408BC2205084C
:101140005C09002010B50B680446C0F894304B6869
:101150000549A0F8A0301046EFF722FEF0F722F87C
:10116000C4F8900010BD00BF00007A4410B5038F92
:1011700004465A2B02D0B3F5877F19D15A2902D0E1
:10118000B1F5877F19D104F1080033F057FB0E4BFE
:101190009C4205D113F0F4FBE18EA08E13F092FA7D
:1011A000A06878B104F11801BDE8104032F065BEC6
:1011B0005A2902D0B1F5877FE5D1A38EE28EE3866E
:1011C000A286E0E710BD00BFF83000202DE9F04F07
:1011D00097B090F8B230044602AFE3B1D0F8842063
:1011E000B14B9A4217D1843029F09BF894F8AF3074
:1011F000834204D100205437BD46BDE8F08FFFF78D
:1012000027F900212046B4F8A230D4F8982084F8B9
:10121000B210FFF747FEA368002B00F0BF81204605
:1012200029F01AF90028E5D104F1500A504633F0AC
:1012300023FC0028DED094F84810002900F09A80A2
:101240000023236304F12803FB6294F8B430002BDD
:1012500040F0A180FEF718FA78610028CAD1204634
:1012600029F0BEF804F1080B5846F96A07F1380274
:10127000C7F810D033F0C1FB002800F0848107F1DB
:10128000380033F0EBFD202594F83A30064607F19C
:101290003800B5FBF3F533F0E6FD814607F1380081
:1012A00033F0E1FDB0EBC51F4FEAC51800F2CA806C
:1012B00001233B6280231FFA89F09B004009BB6138
:1012C0000130073323F007037863ADEB030D7B6B2D
:1012D0000DF108089B00073323F00703ADEB030D66
:1012E00002ABBB62B4F8AC300025B3F5807F14BF0D
:1012F00002230123BB60BB694344FB6007F1380054
:1013000033F0ACFDB4F87A307862B3F5807F05D065
:101310005946504607F1380233F0BCFBB4F8AA3006
:1013200087F833301DB1B4F8AC3087F8333050460D
:1013300016F06CFF002800F02681012394F8B620F7
:101340000093002107F13303206DD4F860C0E0471B
:10135000504633F09CFB00239946FB61BB8B3A6AF5
:101360009A4200F2A380BA686B1C9A424FF00105C2
:10137000C4D808E1A068002800F0108116F0DCF85D
:10138000F862002800F00A81B4F87A30B3F5807F63
:101390007FF45BAF54E7204604F1080629F020F8FB
:1013A0003046C7F828D033F0EDFA0546304633F022
:1013B000EBFAC5F34F05EB1D23F00703ADEB030D6F
:1013C0000DF108092A4677218046484639F0C8FAC7
:1013D000B4F8AA30504687F8443016F017FF834619
:1013E00088B12046D7F828D029F019F894F8B230FF
:1013F000002B3FF42FAFFEF747F900287FF42AAF08
:10140000FEF77AFFF2E70123014694F8B620009335
:10141000266E07F14403206DB047504633F037FB8A
:101420001FFA8BF39845DCD9504616F0EFFE0BF10E
:10143000010B0028D5D094F8B62000954B46012129
:10144000266EE8E707F1380033F003FDB8FBF0F053
:10145000002808BF012086B207F1380033F0FEFCF7
:10146000B0FBF6F083B207F138003B6233F0F6FCD4
:10147000B0FBF6F303FB160080B218B13B6A0133F0
:101480009BB23B6207F1380033F0E3FC16FB00F03F
:1014900080B2B0FBF5F293B205FB1202002A3FF4D2
:1014A0000CAF01339BB208E7BC2205087B69786A60
:1014B0007A8FFB643B8F8642A7F8443002EB090326
:1014C00088BF7A6A9BB298BF9219A7F8463095BF39
:1014D0004A449B1813B21BB2A7F84A307B6AB7F98B
:1014E0003C109B1B9BB2A7F8481007F144007B629D
:1014F00033F0B9FC082294F83A300021B2FBF3F340
:10150000B0FBF3F37A6BB86A92007B6039F028FA8B
:1015100000214046BA6939F023FA94F8B43013B97F
:1015200040F20713E387D5B194F8B33063B10623D3
:1015300084F83E3043465846BA6A07F1440133F016
:101540004FFA94F8B13013E094F8402012B184F8C7
:101550003F30EFE7B4F84230002BF2D0EAE74346E1
:101560005846BA6A07F1440133F03AFA94F8B030B9
:10157000B3B9504616F04AFEFB69B1440133FB6132
:101580001FFA89F9A8B9FB6AD7F810D09B68FB62EB
:10159000002B7FF467AE204628F041FF01202AE6A9
:1015A0004346FA689342E4D01A68D24343F8042BC6
:1015B000F7E7BB8894F8B620009301214346206DDD
:1015C000D4F860C0E047504633F061FAFEF794FE6D
:1015D000C4E600BF10B590F8B23004463BB3D0F873
:1015E0008420134B9A4214D1843028F09AFE94F848
:1015F000AF3083421BD0FEF72BFF002184F8B210DE
:101600002046B4F8A230D4F89820BDE81040FFF787
:1016100049BC28F0D3FDD4E90432C01AB4F8A8308C
:1016200061EB020183424FF000038B41E3D310BD15
:10163000BC22050810B590F8B230044693B1D0F83A
:101640008420104B9A4201D028F0B8FEFEF700FF2C
:1016500000212046B4F8A230D4F8982084F8B210C3
:10166000FFF720FC04F1080033F0AEF9D4F8842031
:10167000054B9A4205D104F18400BDE8104028F0E2
:1016800045BE10BD20EE0408BC22050810B5044973
:101690000446083033F048F9012384F8483010BD7F
:1016A0005C09002010B50B4C0B4B22689A420ED1FE
:1016B000A2680A4B9A420AD1204628F0CDFE28B9EA
:1016C0002046FFF783FD80F00100C0B210BD00206E
:1016D000FCE700BFF8300020A0BC04085C09002033
:1016E00008B5014803F03CFCA4CB050810B504493B
:1016F0002AF0ECFE044603F029F8204610BD00BF96
:10170000A0BC0408F0B50C4689B0064654F8040B9A
:101710001746FFF7EBFF03AB01930C4B05463A4628
:1017200021460093701E022307F064FB05A90522E1
:10173000039808F045FC049808F048FA05A9024609
:101740002846FFF7FFFC0E2009B0F0BD90BC04084E
:1017500008B5FFF7CBFFFFF739FD10B9024803F0DA
:1017600007FC0E2008BD00BF55C6050810B5FFF7E1
:10177000BDFF28F071FEA0B16430EEF79FFE00229D
:101780000A4BEFF73FF8EFF7ADF901460446EFF7E4
:10179000CDFC40B924F0030040F00200A0F1FF406E
:1017A00010BD0348FCE70348FAE700BF00408F4044
:1017B00002008080020040002DE9F04FCBB00846C7
:1017C00011461A462AAB01936A4B009320232CF052
:1017D000D7F92A9B05220AA92B98039308F0F0FB5E
:1017E00005220DA92C9808F0EBFB40F21931409826
:1017F00029F0FEFA5A22339F049097FBF2F302FB82
:10180000137313B15C4803F095FBFFF7C7FA054665
:101810003F9808F0DBF98346429808F0D7F98246F2
:10182000489808F0D3F93C9B80463A9805933D9B35
:101830000E28069300F08C802CF00EFB06463E9C92
:1018400009A920469DF81C9108F042F9002800F0F3
:10185000828003202AF0F7F8099B044603700023D6
:101860004370837009F10203444A00212A600DF19C
:1018700056005222079339F073F80A9A039B149288
:101880000B9A1393ADF854200D9ACDF85880179207
:101890000E9AADF86E70ADF860202D9A2846ADF81E
:1018A00062202E9A13A9ADF864202F9AADF8662015
:1018B000309AADF86820319AADF86A20329AADF8C6
:1018C0006C20349AADF87020359AADF87220369AB3
:1018D000ADF87420379AADF87620389A059BADF8AC
:1018E00078202093069B9DF8E420CDE92134079BC6
:1018F0008DF87A20ADF88C30049B9DF8EC20259370
:101900009DF80431ADF87C608DF898309DF80C316D
:101910008DF87E208DF8A0309DF81031CDF890B074
:101920008DF8A1309DF81431CDF89CA08DF8A2302F
:101930009DF818318DF8A4908DF8A3309DF82431CE
:101940008DF8A530FFF71EFB28464BB0BDE8F08FA1
:101950004FF4807673E70122204610A908F030FB8F
:1019600010B1DDE910437FE740F25241044803F033
:1019700027FB00BF90BB0408D9C90508A0BC040818
:1019800089C8050870B58AB004AB01931B4B0C469F
:10199000009304310323013807F02CFAFF220021C1
:1019A00040F23533049807F0C1FA05228DF80F0094
:1019B00007A90598246808F003FB204628F096FE46
:1019C000C0B101259DF81860204632460DF10F0385
:1019D0000021009528F0AAFE089B324629462046A1
:1019E0000093079B28F0A2FE204628F020FF0E203F
:1019F0000AB070BDFEF780FCDFE700BF28BE040818
:101A000070B58CB0084611461A4605AB0193184BC9
:101A1000009307232CF0B4F840F2A742154905982B
:101A200007F0BCFA0646FFF7DBF9134B04460360E8
:101A3000012240F2334300210A9807F077FA4FF46D
:101A400085630546012200210B9807F06FFA099B78
:101A5000C0B20193089BEDB2039000932046DDE9EC
:101A600006233146029528F0CDFD20460CB070BD0E
:101A7000F0BD0408A81F050840BE040808B528F0FA
:101A8000A5FD20B940F25D41024803F079FA0E202D
:101A900008BD00BFC9C70508436DDB6B0BB1006D06
:101AA00018470148704700BF000080BF10B5038F82
:101AB00004465A2B02D0B3F5877F19D15A2902D098
:101AC000B1F5877F19D104F1080032F0B7FE0E4B53
:101AD0009C4205D112F054FFE18EA08E12F0F2FD6F
:101AE000A06878B104F11801BDE8104032F0C5B922
:101AF0005A2902D0B1F5877FE5D1A38EE28EE38625
:101B0000A286E0E710BD00BFF8300020F8B590F8DD
:101B1000783004460D46174643B10023204684F82A
:101B2000793028F094FE01263046F8BD90F87960AF
:101B3000002EF2D14B1CF0D028F040FB2369C31AD1
:101B4000BB4202D90D4803F013FAA26EC4E91A0190
:101B5000821A9542E8D3B3FBF5F205FB1233ED1A76
:101B600028F02CFBD4E91A32C01A61EB0201A8421A
:101B700071F10001D1D2FEF7BFFBF1E72CCB0508D4
:101B80002DE9F04F1F460023044680F878300165A8
:101B90008BB040F23B40904601F06EFC6065C3693B
:101BA000002B00F09180206D984786B2636D206D08
:101BB0001B69984783B20793636D206D5B699847F3
:101BC00083B20893636D04F1080B5B6A002B7DD030
:101BD000206D98478146636DDD6A15B1206DA84779
:101BE0000546636D9B69002B77D0206D98475FFA9F
:101BF00080FA636D1B6B13B1206D98470346626DCD
